:100000000C941F2D0C9424300C944F300C947A30A7
:100010000C94A5300C94D0300C94FB300C94263109
:100020000C9451310C94502D0C94502D0C94502D57
:100030000C94502D0C94502D0C94502D0C94502D4C
:100040000C94502D0C94EDCC0C94502D0C94502D00
:100050000C94502D0C94502D0C9492BD0C94522D58
:100060000C94502D0C94CAA70C9476A80C94502D87
:100070000C94502D0C94502D0C94502D0C94502D0C
:100080000C94502D0C94502D0C94502D0C94502DFC
:100090000C94502D0C94502D0C94502D0C94502DEC
:1000A0000C94502D0C94502D0C94502D0C94502DDC
:1000B0000C94502D0C94502D0C94502D0C94502DCC
:1000C0000C94502D0C94502D0C94502D0C94502DBC
:1000D0000C94502D0C94502D0C94502D0C94502DAC
:1000E0000C94502D9A2E9F2EA42EAE2EB82E312F6A
:1000F000C22ECA2ED22EDC2EE62EF02EFF2E092F77
:10010000312F132F1D2F272F552F582F472F4B2FB0
:10011000512F8F2F5C2F602F662F6A2F6E2F742F19
:10012000782F7C2F8F2F822F862F8A2FD866B86644
:10013000BE66BB66C166C466C766D366CA66E56648
:10014000CD66D06605A503A527A524A522A559A59A
:1001500056A554A5B2A580A57DA57BA5FDA703A89E
:1001600014A81FA827A83CA82BA83CA82FA833A8F0
:100170003CA839A839BE45BE49BE5CBE60BE73BE50
:100180007EBE29BE084AD73B3BCE016E84BCBFFD74
:10019000C12F3D6C74319ABD56833DDA3D00C77F57
:1001A00011BED9E4BB4C3E916BAAAABE00000080F0
:1001B0003F05A84CCDB2D44EB93836A9020C50B97F
:1001C000918688083CA6AAAA2ABE000000803F00AB
:1001D0000D947B500D94A12A0D943A550D94ED0A7F
:1001E0000D9429414E414E494E495459494E46CDF0
:1001F000CCCC3D0AD7233C17B7D13877CC2B3295DE
:1002000095E6241FB14F0A000020410000C84200BB
:10021000401C4620BCBE4CCA1B0E5AAEC59D740085
:10022000000A0B02090C0D0E080703040100000070
:1002300000000000000000000000000000000000BE
:10024000000000000000000000000012111000007B
:10025000000000000000000000000000000000009E
:1002600000000000000102102020080810204010AB
:10027000204080020102010804020101020408106A
:100280002040808040201008040201800402018088
:1002900040201008040201080402010102040810B1
:1002A0002040800102040810204080050505050754
:1002B0000508080808020202020A0A0808040404E1
:1002C000040101010101010101030303030303030D
:1002D00003040707070C0C0C0C0C0C0C0C0202029C
:1002E0000206060606060606060B0B0B0B0B0B0B8F
:1002F0000B000020002300260029002C002F0032D4
:100300000000010000030106010901000022002590
:100310000028002B002E00310034000201000005EF
:100320000108010B0100002100240027002A002DF4
:10033000003000330001010000040107010A01013F
:10034000060D00FE09016602D620FFFE0BFE0AFE26
:100350000D00602219698080808080808000801874
:100360003363A0A0A00357675050F850F8505002D4
:1003700059692078A0A0702828F02002596948A85F
:100380005010204050A89002586840A0A040A0986B
:100390009068281363808080113B6B2040408080F0
:1003A000808080404020113B6B80404020202020F6
:1003B0002040408006556520A870A820045565207F
:1003C00020F82020113363604080065161F811331A
:1003D0006340E040025969080810102040408080C6
:1003E00002596920508888888888502002596920DD
:1003F00060A02020202020F8025969708888081009
:10040000204080F8025969F80810207008088870A8
:10041000025969101030505090F81010025969F8C4
:100420008080B0C80808887002596970888080F0A0
:1004300088888870025969F80810102020404040D0
:100440000259697088888870888888700259697034
:10045000888888780808887011386840E040000073
:1004600040E04011386840E04000006040800259A0
:1004700069081020408040201008045464F80000EF
:10048000F802596980402010081020408002596904
:100490007088880810202000200259697088889888
:1004A000A8A8B080780259692050888888F8888880
:1004B00088025969F048484870484848F00259692C
:1004C000708880808080808870025969F048484830
:1004D00048484848F0025969F8808080F080808060
:1004E000F8025969F8808080F08080808002596924
:1004F0007088808080988888700259698888888888
:10050000F888888888123969E0404040404040407F
:10051000E0025969381010101010109060025969EB
:10052000888890A0C0A090888802596980808080C7
:1005300080808080F80259698888D8A8A88888882F
:100540008802596988C8C8A8A898988888025969F3
:10055000708888888888888870025969F0888888B7
:10056000F080808080015A6A70888888888888A88E
:100570007008025969F0888888F0A090888802592C
:1005800069708880807008088870025969F8202096
:10059000202020202020025969888888888888881F
:1005A00088700259698888888850505020200259E4
:1005B0006988888888A8A8A8A8500259698888509E
:1005C0005020505088880259698888505020202037
:1005D0002020025969F808101020404080F8113B93
:1005E0006BE0808080808080808080E0025969801C
:1005F0008040402010100808113B6BE02020202094
:100600002020202020E0085363205088015161F809
:100610002A226280400256667008788898680259DB
:1006200069808080F088888888F0025666708880AB
:100630008088700259690808087888888888780254
:1006400056667088F880887002596930484040F0DA
:100650004040404000586870888888780888700258
:100660005969808080B0C8888888881238684000BE
:10067000C040404040E0004A6A10003010101010A6
:1006800090906002596980808090A0C0A0908812EC
:100690003969C040404040404040E0025666D0A822
:1006A000A8A8A888025666B0C888888888025666B6
:1006B000708888888870005868F0888888F0808002
:1006C000800058687888888878080808025666B0DC
:1006D000C8808080800256667088601088700258DA
:1006E000684040F04040404830025666888888881C
:1006F0009868025666888888505020025666888816
:10070000A8A8A85002566688502020508800586833
:100710008888889868088870025666F8102040809B
:10072000F8015B6B1820202020C0202020201822F8
:100730001969808080808080808080015B6BC02010
:100740002020201820202020C008536348A890FFB4
:10075000FFFFFFFFFFFFFFFFFFFFFFFFFFFFFFFFA9
:10076000FFFFFFFFFFFFFFFFFFFFFFFFFFFFFFFF99
:100770000D00602219698000808080808080800365
:1007800058682070A8A0A0A870200259693048407D
:1007900040E0404048B00356668870505070880270
:1007A000596988885050F820F820202219698080E3
:1007B00080800080808080124A6A60908060909083
:1007C000601090601A3262A0A00359697088A8D89E
:1007D000C8D8A88870045767700878887800F8032C
:1007E00056662850A0A05028045363F80808163114
:1007F00061E00359697088E8D8D8E8D888700A5150
:1008000061F8174464609090600357672020F820D7
:100810002000F807356540A02040E007356540A07E
:100820004020C02A226240800058688888888898C2
:10083000E8808002596978E8E8E8E86828282826EE
:100840002161C0202262408007356540C04040E001
:10085000045767708888887000F8035666A050288F
:100860002850A0025A6A40C04040E00818283808C2
:10087000025A6A40C04040E01028081038025A6A04
:1008800040A04020A04818283808025969200020BC
:10089000204080888870025A6A4020002050888852
:1008A000F88888025A6A10200020508888F88888C2
:1008B000025A6A30480020508888F88888025A6AAC
:1008C00028500020508888F88888025A6A505000C2
:1008D00020508888F88888025A6A20502020508842
:1008E00088F8888802596958A0A0A0B0E0A0A0B8F4
:1008F000005B6B7088808080808088702040025A06
:100900006A402000F88080F08080F8025A6A102047
:1009100000F88080F08080F8025A6A304800F88041
:1009200080F08080F8025A6A505000F88080F08091
:1009300080F8123A6A804000E04040404040E012B7
:100940003A6A204000E04040404040E0124A6A607D
:100950009000E04040404040E0123A6AA0A000E031
:100960004040404040E0025969F0484848E8484863
:1009700048F0025A6A2850008888C8A898888802D7
:100980005A6A40200070888888888870025A6A10E5
:10099000200070888888888870025A6A3048007001
:1009A000888888888870025A6A28500070888888E9
:1009B000888870025A6A50500070888888888870C9
:1009C0000355658850205088015B6B08709898A883
:1009D000A8A8C8C87080025A6A4020008888888801
:1009E000888870025A6A10200088888888888870F1
:1009F000025A6A30480088888888888870025A6A53
:100A000050500088888888888870025A6A102000B0
:100A10008888502020202002596980F0888888F03A
:100A2000808080025969609090A0A0908888B00270
:100A30005969402000700878889868025969102028
:100A40000070087888986802596930480070087802
:100A50008898680259692850007008788898680258
:100A60005969505000700878889868025A6A30486E
:100A70003000700878889868025666702870A0A8C0
:100A80005000586870888080887020400259694002
:100A900020007088F88088700259691020007088E2
:100AA000F88088700259693048007088F880887032
:100AB0000259695050007088F88088701239698036
:100AC0004000C040404040E0123969204000C04032
:100AD000404040E0124969609000C040404040E022
:100AE000123969A0A000C040404040E0025A6A505C
:100AF000206010708888888870025969285000B07A
:100B0000C888888888025969402000708888888849
:100B100070025969102000708888888870025969AD
:100B200030480070888888887002596928500070A1
:100B30008888888870025969505000708888888831
:100B400070035767202000F80020200158680870C3
:100B500098A8A8C8708002596940200088888888B1
:100B60009868025969102000888888889868025916
:100B70006930480088888888986802596950500010
:100B8000888888889868005B6B102000888888981F
:100B900068088870005A6A8080B0C88888C8B080A9
:100BA00080005B6B505000888888986808887001C6
:100BB000050700FE0500FB01F220FFFE05FE05FE15
:100BC0000200400215258080800080053242A0A0EE
:100BD00002556550F850F8500146562070C030E07C
:100BE000200255659010204048025565608068904D
:100BF00068051222808002253540808080400225D1
:100C0000358040404080043343A040A0033343403C
:100C1000E0400122324080043141E0021121800293
:100C20005565081020408002455560909090600204
:100C30002535C040404040024555E0106080F0023C
:100C40004555E0106010E00245552060A0F02002FC
:100C50004555F080E010E00245556080E09060026C
:100C60004555F0102040400245556090609060026C
:100C70004555609070106003132380008002142497
:100C8000800080800235452040804020033343E0CF
:100C900000E00235458040204080024555E010606C
:100CA00000400255657088B8A87002455560909064
:100CB000F090024555E090E090E00235456080807C
:100CC0008060024555E0909090E0023545E080E07C
:100CD00080E0023545E080E080800245557080B0BC
:100CE00090700245559090F09090023545E040405C
:100CF00040E0024555301010906002455590A0C06C
:100D0000A09002354580808080E002556588D8A893
:100D1000888802455590D0B09090024555609090DB
:100D20009060024555E09090E080014656609090BA
:100D3000906010024555E09090E09002455570801B
:100D40006010E0023545E04040404002455590903B
:100D50009090600245559090A0A04002556588A8EB
:100D6000A8A85002455590906090900245559090EB
:100D7000701060023545E0204080E0022535C080DB
:100D80008080C00255658040201008022535C04093
:100D90004040C005324240A0024151F0052232805D
:100DA000400244547090907002455580E09090E06D
:100DB000023444608080600245551070909070024B
:100DC000445460B0C0600235452040E040400046D9
:100DD0005670909070106002455580E0909090029F
:100DE000152580008080800027374000404040402B
:100DF000800245558090A0E090021525808080807B
:100E000080025464F0A8A8A8024454E09090900294
:100E1000445460909060004656E09090E0808000DE
:100E20004656709090701010023444A0C08080022A
:100E3000445470C030E002354540E0404020024458
:100E400054909090700244549090A040025464A832
:100E5000A85050023444A04040A0004656909090C4
:100E6000701060024454F02040F00235456040802C
:100E700040600215258080808080023545C040207A
:100E800040C005425250A0FFFFFFFFFFFFFFFFFFE2
:100E9000FFFFFFFFFFFFFFFFFFFFFFFFFFFFFFFF62
:100EA000FFFFFFFFFFFFFFFF020040FFFFFFFFFF0D
:100EB000FFFFFFFFFFFFFFFFFFFFFFFFFFFFFFFF42
:100EC000FFFFFFFFFFFFFFFFFFFFFFFFFFFFFFFF32
:100ED000FFFFFFFFFFFFFFFFFFFFFFFFFFFFFFFF22
:100EE000FFFFFFFFFFFFFFFFFFFFFFFFFFFFFFFF12
:100EF000FFFFFFFFFFFFFFFFFFFFFFFFFFFFFFFF02
:100F0000FFFFFFFFFFFFFFFFFFFF01050800FF06D8
:100F10000121023520FFFF07FF06FF0900502216BE
:100F200056808080800080153353A0A0A0025757C0
:100F30005050F850F850500257572070A070287049
:100F40002013355580A040A02002475740A0A04064
:100F5000A0A05025135380808012265640808080A8
:100F600080401226568040404040800245559060A7
:100F7000F060900255552020F82020113353604036
:100F800080044151F011335340E0400246561010A6
:100F90002040808012365640A0A0A0A040123656B5
:100FA00040C0404040E00246566090106080F00231
:100FB0004656F020601090600246562060A0F02057
:100FC00020024656F080E01090600246566080E0B5
:100FD000909060024656F010202040400246566035
:100FE000906090906002465660909070106012255C
:100FF00055C0C000C0C0113656606000604080120D
:101000003656204080804020034353F000F01236D3
:101010005680402020408012365640A0204000409C
:10102000015858304898A8A8904030024656609021
:1010300090F09090024656E090E09090E002465684
:10104000609080809060024656E090909090E00220
:101050004656F080E08080F0024656F080E08080C6
:1010600080024656609080B090600246569090F0A4
:10107000909090123656E040404040E00246567054
:10108000202020A04002465690A0C0A0A09002467A
:10109000568080808080F002465690F0F0909090CC
:1010A00002465690D0F0B0B09002465660909090B4
:1010B0009060024656E09090E08080014757609033
:1010C00090D0B06010024656E09090E090900246BA
:1010D00056609040209060123656E04040404040BC
:1010E0000246569090909090600246569090909054
:1010F0006060024656909090F0F0900246569090B4
:1011000060609090025656888850202020024656F3
:10111000F010204080F0123656E080808080E0029F
:101120004656808040201010123656E020202020A5
:10113000E016325240A0014151F016225280400286
:101140004454709090700246568080E09090E01277
:101150003454608080600246561010709090700287
:10116000445460B0C060024656205040E040400108
:10117000455560907010600246568080E0909090D7
:101180001236564000C04040E01137572000202062
:1011900020A040024656808090E09090123656C0C3
:1011A00040404040E0025454D0A8A8A8024454E073
:1011B00090909002445460909060014555E090E01A
:1011C00080800145557090701010024454A0D0806A
:1011D0008012345460C020C00246564040E0405067
:1011E0002002445490909070123454A0A0A0400269
:1011F000545488A8A850024454906060900145550A
:101200009090709060024454F02040F002475730B4
:101210004020C0204030221656808080808080028E
:101220004757C02040304020C006425250A0FFFF28
:10123000FFFFFFFFFFFFFFFFFFFFFFFFFFFFFFFFBE
:10124000FFFFFFFFFFFFFFFFFFFFFFFFFFFFFF09A4
:101250000050221656800080808080014656207003
:10126000A0A070200246562050E04050A0025555E4
:1012700088705070880256568850F820F82022173F
:1012800057808080008080800247577080E0907097
:1012900010E0173151A002565670A8C8C8A87014A3
:1012A000355560A06000E003435350A05012335303
:1012B000E02020143151E002565670E8D8E8D8708A
:1012C000173151E015335340A04012355540E040EE
:1012D00000E014355540A02040E0143555C020C032
:1012E00020C01622524080014555909090E0800227
:1012F000565678E8E8682828241151801122524077
:101300008014355540C04040E014355540A04000A1
:10131000E0034353A050A0024757808080A060F0B4
:10132000200247578080A0D010207002475780408D
:101330008060A0F02012365640004080A040024756
:101340005740206090F0909002475720406090F006
:10135000909002475760906090F0909002475750ED
:10136000A06090F0909002475790006090F09090AD
:1013700002475760906090F0909002465670A0A08F
:10138000F0A0B001475760908080906040024757BE
:101390004020F080E080F00247572040F080E0805D
:1013A000F00247576090F080E080F00247579000CD
:1013B000F080E080F01237578040E0404040E0127B
:1013C00037572040E0404040E012375740A0E0400F
:1013D0004040E0123757A000E0404040E00256563F
:1013E0007048E848487002475750A090D0B090909D
:1013F000024757402060909090600247572040601D
:101400009090906002475760906090909060024783
:101410005750A06090909060024757900060909065
:101420009060123353A040A002465670B0B0D0D0A6
:10143000E00247574020909090906002475720402C
:1014400090909090600247576090909090906002CA
:101450004757900090909090600257571020885006
:1014600020202002465680E09090E08002465660A0
:1014700090A0A090A002475740200070909070026A
:1014800047572040007090907002475720500070DE
:1014900090907002475750A000709090700246568E
:1014A00050007090907002475760906070909070FC
:1014B000025454F068B07811355560808060400265
:1014C000475740200060B0C060024757204000608E
:1014D000B0C06002475760900060B0C060024656DE
:1014E000500060B0C060123757804000C04040E0FC
:1014F000123757204000C04040E012375740A0004C
:10150000C04040E0123656A000C04040E0024757BD
:10151000A040A01070906002475750A000E090904B
:10152000900247574020006090906002475720404B
:101530000060909060024757609000609090600259
:10154000475750A00060909060024656900060900F
:1015500090601235554000E0004002445470B0D015
:10156000E00247574020009090907002475720407B
:101570000090909070024757609000909090700299
:1015800046569000909090700148582040009090EE
:101590007090600147578080E090E080800147575D
:1015A000900090907090602020202000202020202B
:1015B0002020200025753A253032750025303275FF
:1015C0003A253032750025756420253032753A256C
:1015D00030327500A2167216BA168A163FFFF0381E
:1015E00000703186302387102787902F87D02F03F4
:1015F000D02030102078102078102030102F03D009
:101600002F87D02787902387103186303800703F8E
:10161000FFF03FFFF038007030FC3020FC102078E5
:10162000102030102C00D02E31D02F7BD02F7BD02B
:101630002E31D02C00D020301020781020FC10301B
:10164000FC303800703FFFF0041040020820020810
:101650002004104008208010410010410008208024
:101660000410400000001FFFF81FFFF81FFFF81FC5
:10167000FFF81FE020102310249010A0112022104A
:10168000241037B00840048003001FE03FF03CF016
:101690003B701F601EE03DF03BF038700FC00780CC
:1016A00003001FE02010211023101520112021100D
:1016B000211031300840048003001FE03FF03EF06D
:1016C0003CF01AE01EE03EF03EF03EF00FC0078016
:1016D00003004572723A207574663820666F6E7426
:1016E000206E6F7420696E697469616C697A6564D3
:1016F0002E004572723A207574663820666F6E74DB
:10170000206E6F7420696E697469616C697A6564B2
:101710002E004572723A207574663820666F6E74BA
:10172000206E6F7420696E697469616C697A656492
:101730002E00506C6561736520726573657400508E
:1017400052494E5445522048414C544544007F80F4
:10175000FFC0FFC0FFC07F807F80FFC0FFC0FFC011
:101760003F001E000C00FFFFFF0E000E000E000EDB
:10177000000E000E000E000E007FC03F801F000E06
:1017800000040004000E001F003F807FC00E000E0A
:10179000000E000E000E000E000E000E0000FE00F7
:1017A00003FF800783C00E01C00E00E01C00E07F35
:1017B00000E03E00E01C00E00800E00000E0000166
:1017C000C00E01C00F078007FF0001FC0001FC00F4
:1017D00007FF000F07800E01C00001C00000E008F5
:1017E00000E01C00E03E00E07F00E01C00E00E0096
:1017F000E00E01C00783C003FF8000FE0000060C5E
:1018000000FE07022603BC017FFE08FE08FE050855
:101810000806000040F0C888889878100508080677
:101820000000C0F88888888888F80505050600014A
:101830002030F830200508080600002070F820202D
:101840002020E00509090600FF2070A8A8B88888B4
:101850007020050606060001E08CEA8C8A0A05095C
:10186000090600FFF8A88888888888A8F8050A0A69
:101870000600FE205050505088A8A888700303032B
:1018800006000340A040FFFFFFFFFFFFFFFFFFFF39
:10189000FFFFFFFFFFFFFFFFFFFFFFFF000000064E
:1018A00005FF01070706020080808080800080031A
:1018B0000303060105A0A0A005060606000050F8D7
:1018C0005050F8500509090600FF2070A8A07028A4
:1018D000A87020050707060000C8C8102040989887
:1018E00005070706000040A0A040A8906801030378
:1018F0000602058080800309090601FF2040408020
:1019000080804040200309090601FF8040402020DC
:101910002040408005070706000020A8702070A81E
:10192000200505050600012020F8202002030306FB
:1019300001FFC04080050101060003F80202020613
:101940000100C0C005070706000008101020404035
:1019500080050707060000708898A8C888700307EC
:101960000706010040C040404040E0050707060070
:1019700000708808102040F8050707060000F808E6
:10198000103008887005070706000010305090F8E6
:101990001010050707060000F880F0080888700599
:1019A0000707060000304080F088887005070706AA
:1019B0000000F8081010202020050707060000701E
:1019C0008888708888700507070600007088887806
:1019D000081060020505060100C0C000C0C0020674
:1019E000060601FFC0C000C04080030505060101D6
:1019F0002040804020050303060002F800F803059C
:101A000005060101804020408005070706000070A0
:101A10008810202000200507070600007088B8A85D
:101A2000B88070050707060000708888F8888888E5
:101A3000050707060000F04848704848F00507070A
:101A40000600007088808080887005070706000007
:101A5000F04848484848F0050707060000F880802D
:101A6000F08080F8050707060000F88080F080808D
:101A70008005070706000070888080988870050739
:101A800007060000888888F8888888030707060109
:101A900000E04040404040E00507070600003810E5
:101AA00010101090600507070600008890A0C0A0E5
:101AB0009088050707060000808080808080F805F8
:101AC000070706000088D8A88888888805070706C1
:101AD00000008888C8A89888880507070600007055
:101AE000888888888870050707060000F08888F0D5
:101AF00080808005070706000070888888A89068A5
:101B0000050707060000F08888F0A0908805070701
:101B100006000070888070088870050707060000BE
:101B2000F82020202020200507070600008888884C
:101B300088888870050707060000888888885050C4
:101B40002005070706000088888888A8A850050790
:101B5000070600008888502050888805070706007F
:101B60000088885020202020050707060000F8087C
:101B700010204080F80309090601FFE08080808082
:101B8000808080E00507070600008040402010109C
:101B9000080309090601FFE020202020202020E082
:101BA0000503030600052050880501010600FEF824
:101BB00003030306010580402005050506000070AB
:101BC000087888780507070600008080F0888888F4
:101BD000F00505050600007080808870050707067F
:101BE00000000808788888887805050506000070D8
:101BF00088F08070050707060000304840E040404C
:101C0000400507070600FE70888888780870050779
:101C1000070600008080F08888888803070706018F
:101C2000004000C0404040E00409090601FE1000E9
:101C300030101010109060050707060000808088A3
:101C400090E09088030707060100C04040404040F4
:101C5000E0050505060000D0A8A8A8A8050505060A
:101C60000000B0C8888888050505060000708888CF
:101C700088700507070600FEF0888888F0808005D8
:101C800007070600FE788888887808080505050695
:101C90000000B0C8808080050505060000788070CF
:101CA00008F00507070600002020F820202018056E
:101CB0000505060000888888986805050506000067
:101CC00088888850200505050600008888A8A85047
:101CD0000505050600008850205088050707060006
:101CE000FE88888850204080050505060000F81011
:101CF0002040F80309090601FF2040404080404091
:101D000040200109090602FF808080808080808059
:101D1000800309090601FF80404040204040408088
:101D200005030306000248A890FF1FFFFFFFFFFF07
:101D3000FF600000000001FF400000000000FF8085
:101D400000000000007F83CF00000C303F87FF8041
:101D5000000C301F867980000C000F8C30C7838CFC
:101D600030E78C30CFC7CC31F38C30DCECEC33B9BE
:101D70008C30D86C6C33198C30D06C0C33198C309F
:101D8000D86C0C33198C30DC6C0E3B198C30CF7C4A
:101D9000079F198C30C77C038F194000000000009A
:101DA00002600000000000061FFFFFFFFFFFF800B9
:101DB0000000000000000000000000000000000023
:101DC0000000000000000000000000000000000013
:101DD00000000C000000000000000C0000000000EB
:101DE00000001200000000000000230000000000BE
:101DF000000021000000000000004C8000000000F6
:101E000000005E8000000000000092400000000022
:101E10000000A1400000000000012120000000009F
:101E200000027F900000000000020010000000008F
:101E30000007FFF800000000000400080000000098
:101E40000008000400000000000800060000000078
:101E5000001000020000000000301E010000000021
:101E600000207F81000000000041FFE080000000B2
:101E70000043FCF08000000000873B784000000039
:101E8000018EDBFC60000000010FEBCC20000000A5
:101E9000021FEDB610000000021FDEB610000000A9
:101EA0000439CD7F080000000436E0FF0800000080
:101EB000087EC0BB84000000187F005D8600000023
:101EC000107FC0ED82000000203CC07301000000C4
:101ED000203B337F01000000701BE77E0380000081
:101EE000C81DEEDE04C00000880FDEDC04400001E7
:101EF000240FDF3C092000012607DBF8192000022F
:101F00007203E7F0139000025101FFE022900004F9
:101F100089007F802448000904801E004824000BAB
:101F2000FE400000DFF40010004000008002001FAF
:101F3000FFFFFFFFFFFE00000000000000000000A8
:101F40000000000000000000000000000000001081
:101F500022103C3C0E1F001022100422110400101D
:101F600022100822110400102210083C1104001055
:101F70002210102211040010221020221104001E31
:101F80001C1E3C3C0E04000000000000000000008D
:101F90000000000000000000000000000000000041
:101FA0000000000000000000000000000000000031
:101FB0000000000000000000000000000000000021
:101FC0000000000000000000000000000000000011
:101FD0000000000000000000000000000000000001
:101FE00000000000000000000000000000000609E2
:101FF00000FE06018902FE20FFFE07FE06FE00002D
:10200000000600070106060602008080808000802E
:10201000030303060103A0A0A00507070600FF5065
:1020200050F850F850500509090600FE2070A8A08D
:102030007028A870200608080600FF40A848102055
:102040004854080507070600FF6090906098906864
:102050000103030602038080800207070602FF4097
:102060008080808080400207070602FF8040404059
:102070004040800505050600008850F85088050599
:10208000050600002020F820200204040602FEC0FD
:10209000404080050101060002F80202020602002B
:1020A000C0C004060606010010102040808004060F
:1020B00006060100609090909060030606060100FD
:1020C00040C0404040E00406060601006090102039
:1020D00040F0040606060100F020601010E005063E
:1020E0000606000010305090F810040606060100A5
:1020F000F080E01010E00406060601006080E09029
:102100009060040606060100F0101020404004060E
:1021100006060100609060909060040606060100CB
:10212000609090701060020505060200C0C000C0FB
:10213000C00207070602FEC0C000C040408005057F
:10214000050600001860806018050303060001F80A
:1021500000F8050505060000C0300830C004070778
:102160000601006090106040004005060606000071
:102170007090A8B08070050606060000205088F810
:102180008888050606060000F088F08888F00406B6
:10219000060601006090808090600406060601003B
:1021A000E090909090E0040606060100F080E08048
:1021B00080F0040606060100F080E08080800406BE
:1021C00006060100609080B09060040606060100DB
:1021D0009090F0909090030606060100E040404089
:1021E00040E0050606060000381010109060040656
:1021F0000606010090A0C0A090900406060601000B
:102200008080808080F005060606000088D8A8A897
:10221000888804060606010090D0B09090900506CC
:10222000060600007088888888700406060601008B
:10223000E09090E080800407070601FF609090D056
:10224000B06010040606060100E09090E090900453
:102250000606060100609040209060050606060014
:1022600000F820202020200406060601009090900F
:10227000909060040606060100909090F060600562
:1022800006060600008888A8A8D888050606060065
:1022900000885020205088050606060000888850D7
:1022A000202020040606060100F010204080F003E4
:1022B0000606060100E080808080E0040606060134
:1022C00000808040201010030606060100E0202058
:1022D0002020E005030306000320508805010106C5
:1022E00000FEF80202020602048040040404060113
:1022F00000709090700406060601008080E09090C7
:10230000E0040404060100708080700406060601E3
:102310000010107090907004040406010060B0C0BA
:1023200070040606060100205040E0404004060606
:102330000601FE60909070106004060606010080A1
:1023400080E09090900306060601004000C04040E7
:10235000E00308080601FE200060202020A04004C1
:1023600006060601008080A0C0A0900306060601B4
:1023700000C040404040E0050404060000D0A8A88A
:1023800088040404060100E090909004040406010F
:1023900000609090600406060601FEE09090E080E8
:1023A000800406060601FE7090907010100404046C
:1023B000060100A0D0808004040406010070C03033
:1023C000E00406060601004040E0405020040404FA
:1023D0000601009090907004040406010090906043
:1023E0006005040406000088A8A85004040406013F
:1023F00000906060900406060601FE909090709038
:1024000060040404060100F02040F0030707060101
:1024100000204040804040200107070602FF8080E6
:1024200080808080800307070601008040402040B4
:10243000408004020206010350A0FFFFFFFFFFFFE0
:10244000FFFFFFFFFFFFFFFFFFFFFFFFFFFFFFFF9C
:10245000FFFFFFFFFFFFFFFFFFFFFF000000060081
:1024600007010606060200800080808080040606C0
:102470000601FF2070A0A070200507070600FF30AE
:102480004840F04040F8050505060000A850885077
:10249000A80506060600008850F820F82001070766
:1024A0000602FF808080008080800407070601FF0D
:1024B000708060906010E0030101060105A006072E
:1024C00007060000788494A4948478030505060127
:1024D0000160A06000E00505050600002850A0503E
:1024E00028040303060100F0101004010106010294
:1024F000F00607070600007884B4A4A484780401D9
:1025000001060105F004030306010260906005075F
:10251000070600FF2020F8202000F803050506012B
:102520000140A02040E0030505060101C020402035
:10253000C002020206020440800405050601FF9065
:1025400090B0D08005060606000078E8E8682828E4
:10255000010101060202800202020602FE4080031F
:10256000050506010140C04040E0030505060101E4
:1025700040A04000E0050505060000A0502850A03E
:102580000508080600FF40C040507030781005086C
:10259000080600FF40C040506808103805080806CB
:1025A00000FFC0204030F03078100407070601001B
:1025B0002000206080906005070706000040202072
:1025C000507088880507070600001020205070888A
:1025D00088050707060000205020507088880507EE
:1025E000070600002850205070888805070706005D
:1025F0000050002050708888050707060000205012
:10260000205070888805060606000078A0F0A0A07B
:10261000B80408080601FE609080809060204004A5
:1026200007070601004020F080E080F0040707065D
:1026300001002040F080E080F00407070601002040
:1026400050F080E080F00407070601005000F080A1
:10265000E080F00307070601008040E0404040E0D2
:102660000307070601002040E0404040E003070761
:1026700006010040A0E0404040E0030707060100DB
:10268000A000E0404040E00506060600007048E873
:1026900048487004070706010050A090D0B0909001
:1026A000040707060100402060909090600407072F
:1026B000060100204060909090600407070601002A
:1026C0002050609090906004070706010050A060C1
:1026D0009090906004070706010050006090909071
:1026E000600505050600008850205088040808068B
:1026F00001FF1070B0B0D0D0E080040707060100E1
:1027000040209090909060040707060100204090C0
:1027100090909060040707060100205090909090E0
:102720006004070706010050009090909060050734
:10273000070600001020885020202004060606010D
:102740000080E09090E0800406060601006090A002
:10275000A090A00407070601004020007090907030
:1027600004070706010020400070909070040707DE
:1027700006010020500070909070040707060100C9
:1027800050A0007090907004060606010050007082
:102790009090700407070601002050207090907000
:1027A00005040406000070A8B0780406060601FEC1
:1027B0007080807020400407070601004020006000
:1027C000B0C07004070706010020400060B0C07070
:1027D00004070706010020500060B0C07004060620
:1027E000060100500060B0C07003070706010080BA
:1027F0004000C04040E0030707060100204000C041
:102800004040E003070706010040A000C04040E050
:10281000030606060100A000C04040E004070706CA
:1028200001003060107090906004070706010050AE
:10283000A000E0909090040707060100402000608F
:1028400090906004070706010020400060909060AF
:1028500004070706010020500060909060040707FD
:1028600006010050A000609090600406060601007A
:102870005000609090600505050600002000F800FB
:102880002004040406010070B0D0E004070706012C
:10289000004020009090907004070706010020403F
:1028A000009090907004070706010020500090905F
:1028B0009070040606060100500090909070040984
:1028C000090601FE20400090909070906004080876
:1028D0000601FE8080E09090E080800408080601F8
:1028E000FE5000909090709060536E346B330049AE
:1028F0006E76616465727300427269636B6F7574A2
:10290000004D61696E005072696E742066726F6D61
:10291000205344005072696E742066726F6D2053AC
:102920004400022E2E004D61696E005072696E7473
:102930000043616E63656C00537461727420707241
:10294000696E7420003F00536D6F6F7468696E6725
:1029500000536D6F6F7468696E67005A005A0059B2
:1029600000590058005800436F7272656374696FB4
:102970006E00436F7272656374696F6E004D6169BA
:102980006E0046696C616D656E74004261636B6CCC
:102990006173680053746570732F6D6D004A6572C2
:1029A0006B00416363656C65726174696F6E00569C
:1029B000656C6F6369747900436F6E6669677572E1
:1029C0006174696F6E00453273746570732F6D6D3D
:1029D00000453273746570732F6D6D0045317374EB
:1029E0006570732F6D6D00453173746570732F6D55
:1029F0006D005A73746570732F6D6D005A73746532
:102A000070732F6D6D005973746570732F6D6D0049
:102A10005973746570732F6D6D005873746570739E
:102A20002F6D6D005873746570732F6D6D00416468
:102A300076616E6365642053657474696E677300B4
:102A400056652D6A65726B0056652D6A65726B005E
:102A5000567A2D6A65726B00567A2D6A65726B0024
:102A600056792D6A65726B0056792D6A65726B0016
:102A700056782D6A65726B0056782D6A65726B0008
:102A8000416476616E6365642053657474696E6732
:102A90007300416D617820486F74656E6420320068
:102AA000416D617820486F74656E64203200416D1D
:102AB000617820486F74656E64203100416D6178E3
:102AC00020486F74656E64203100416D6178205A32
:102AD00000416D6178205A00416D617820590041B4
:102AE0006D6178205900416D6178205800416D6119
:102AF00078205800412D74726176656C00412D7408
:102B0000726176656C00412D726574726163740048
:102B1000412D7265747261637400416363656C007A
:102B2000416363656C00416476616E636564205344
:102B3000657474696E6773005654726176206D69AE
:102B40006E005654726176206D696E00566D696E26
:102B500000566D696E00566D617820486F74656E21
:102B600064203200566D617820486F74656E642071
:102B70003200566D617820486F74656E64203100B4
:102B8000566D617820486F74656E64203100566D13
:102B90006178205A00566D6178205A00566D617830
:102BA000205900566D6178205900566D6178205883
:102BB00000566D6178205800416476616E636564EB
:102BC0002053657474696E6773004C6F6164206D87
:102BD0006D2032004C6F6164206D6D2032004C6FAF
:102BE0006164206D6D2031004C6F6164206D6D203B
:102BF00031004C6F6164206D6D004C6F6164206D1D
:102C00006D00556E6C6F6164206D6D203200556EE5
:102C10006C6F6164206D6D203200556E6C6F616465
:102C2000206D6D203100556E6C6F6164206D6D20DC
:102C30003100556E6C6F6164206D6D00556E6C6F68
:102C40006164206D6D00416476616E6365204B4860
:102C50006F74656E64203200416476616E63652036
:102C60004B486F74656E64203200416476616E6318
:102C700065204B486F74656E642031004164766155
:102C80006E6365204B486F74656E6420310041644B
:102C900076616E6365642053657474696E67730052
:102CA00044697361626C65207374657070657273DA
:102CB000004D3834004175746F20686F6D650047B2
:102CC0003238004C6576656C205820617869730055
:102CD000004D6F76652061786973004D61696E0003
:102CE0004578747275646572203200457874727527
:102CF00064657220310045787472756465722000D5
:102D00004D6F7665205A004D6F76652059004D6FE6
:102D100076652058004D6F76656D656E7400457858
:102D200074727564657220320045787472756465DA
:102D3000722031004D6F766520302E3032356D6D4A
:102D4000004D6F766520302E316D6D004D6F7665CC
:102D500020316D6D004D6F76652031306D6D004D09
:102D60006F7665206178697300486F74656E6420C2
:102D7000746F6F20636F6C6400457874727564655E
:102D80007220004D6F7665205A004D6F7665205990
:102D9000004D6F76652058004D6F7665205A004DC6
:102DA0006F76652059004D6F766520580057616930
:102DB0007420666F720066696C616D656E74207058
:102DC000757267650000506C656173652077616995
:102DD000742E00507265737320627574746F6E0088
:102DE000746F20726573756D65207072696E740002
:102DF0005761697420666F720066696C616D656EFB
:102E000074206C6F616400496E736572742066692A
:102E10006C616D656E7400616E64207072657373B1
:102E200020627574746F6E00746F20636F6E7469C6
:102E30006E756500507265737320627574746F6E81
:102E400000746F2068656174206E6F7A7A6C65001B
:102E50004E6F7A7A6C652068656174696E670050A0
:102E60006C6561736520776169742E2E2E00576141
:102E7000697420666F720066696C616D656E74209E
:102E8000756E6C6F6164005761697420666F7200C3
:102E900066696C616D656E74206368616E6765005C
:102EA000746F207374617274005061726B696E6725
:102EB0002E2E2E004368616E67696E672046696C2E
:102EC000616D656E7400554E4C4F41442046494C2F
:102ED000414D454E54004C4F41442046494C414DD4
:102EE000454E540020204E6F7A7A6C653A200020BF
:102EF00000456E642066696C616D656E7420636860
:102F0000616E6765005075726765206D6F72650050
:102F1000004D363030204230205431004D363030B4
:102F2000204230205430004368616E676520666936
:102F30006C616D656E7420486F74656E642032003C
:102F40004368616E67652066696C616D656E7420AB
:102F5000486F74656E642031004D61696E0043688E
:102F6000616E67652066696C616D656E7400556E93
:102F70006C6F61642066696C616D656E74004C6F86
:102F800061642066696C616D656E74004D36303029
:102F900020423020542564004D373032203B2564D8
:102FA000004D37303220542564004D3730312054E5
:102FB0002564005072656865617420437573746F91
:102FC0006D005072656865617420437573746F6D30
:102FD000005072656865617420414253005072650B
:102FE0006865617420504C41004261636B004E6F14
:102FF0002053442063617264005072696E742066CD
:10300000726F6D205344004368616E6765205344BE
:103010002063617264004D32310041626F7574202B
:103020005072696E746572004368616E67652066F0
:10303000696C616D656E7400436F6E666967757269
:103040006174696F6E0054656D706572617475723C
:1030500065004D6F76656D656E7400526573756DB4
:1030600065207072696E740054756E650053746FDC
:1030700070207072696E7400506175736520707293
:10308000696E7400496E666F2073637265656E00C9
:1030900053746F70004261636B0053746F702070E3
:1030A00072696E74003F0050726F6265205A204F43
:1030B0006666736574004261627973746570205945
:1030C000004261627973746570205800466C6F77B6
:1030D000203200466C6F77203200466C6F772031CB
:1030E00000466C6F7720310046616E207370656515
:1030F0006420310046616E20737065656420310084
:1031000042656400426564004E6F7A7A6C652032D5
:10311000004E6F7A7A6C652032004E6F7A7A6C6559
:103120002031004E6F7A7A6C6520310053706565EE
:1031300064005370656564004D61696E00426162B0
:103140007973746570205900426162797374657097
:1031500020580047616D6573004669726D77617232
:10316000652056657273696F6E004D61696E00432C
:103170006F6F6C646F776E0046616E20737065656B
:103180006420310046616E207370656564203100F3
:1031900042656400426564004E6F7A7A6C65203245
:1031A000004E6F7A7A6C652032004E6F7A7A6C65C9
:1031B0002031004E6F7A7A6C652031004D61696E66
:1031C000006F6F6F0000001FC07FF0DDD8FFF87F39
:1031D000F0444024800000318000002480444010EE
:1031E0007CFEFEFE04000E000E007FC0FFE0FFE04C
:1031F000FFE0FFE006000F001F8036C03FC009005F
:103200001680294006000F001F8036C03FC0168080
:1032100020401080104008801FC037607FF05FD0D2
:1032200050500D80104048905FD077707FF01FC0E5
:10323000104020200F007FE0FFF0E670FFF01980C3
:1032400036C0C0300F007FE0FFF0E670FFF019805D
:1032500036C0198047414D45204F564552005265B2
:1032600073746F7265206661696C73616665004C8A
:103270006F61642073657474696E67730053746F53
:1032800072652073657474696E677300546F6F6C38
:10329000204368616E676500546F6F6C204F6666EF
:1032A000736574730050726F6265205A204F6666B2
:1032B00073657400416476616E6365642053657460
:1032C00074696E6773004D61696E00473238005350
:1032D000746F72652073657474696E677300326E03
:1032E00064206E6F7A7A6C65205A00326E64206EAC
:1032F0006F7A7A6C65205A00326E64206E6F7A7A2B
:103300006C65205900326E64206E6F7A7A6C65208D
:103310005900326E64206E6F7A7A6C6520580032E4
:103320006E64206E6F7A7A6C65205800436F6E660B
:10333000696775726174696F6E005A2052616973B2
:1033400065005A20526169736500436F6E66696754
:1033500075726174696F6E0050726F6265205A20D9
:103360004F666673657400326E64206E6F7A7A6C95
:1033700065205A004D6F76696E672E2E2E004D32F5
:1033800034004D323520500A4D3234005072696E8F
:103390007420706175736564005061757365207089
:1033A00072696E74005072696E742061626F72741B
:1033B0006564004C756C7A426F742054415A203613
:1033C0002072656164792E005072696E74696E674F
:1033D0002E2E2E005072696E7420706175736564B4
:1033E00000436172642072656D6F766564004361AD
:1033F000726420696E736572746564004D31313793
:10340000004D33310043616E6E6F7420656E7465DC
:1034100072207375626469723A20002E0A006F7020
:10342000656E206661696C65642C2046696C653A3E
:1034300020006175746F25632E67006572726F726C
:103440002077726974696E6720746F2066696C6595
:103450000A004E6F74205344207072696E74696E56
:10346000670A005344207072696E74696E67206247
:1034700079746520002E0A0044656C6574696F6E6E
:10348000206661696C65642C2046696C653A200091
:1034900046696C652064656C657465643A005772B2
:1034A0006974696E6720746F2066696C653A2000E4
:1034B0002E0A006F70656E206661696C65642C2051
:1034C00046696C653A20002E0A006F70656E2066B2
:1034D00061696C65642C2046696C653A2000466918
:1034E0006C652073656C65637465640A00205369BC
:1034F0007A653A200046696C65206F70656E656478
:103500003A20002066696C653A200066726573682F
:1035100000646F696E67004E6F772000454E44204F
:10352000535542524F5554494E450A002220706F60
:1035300073002220706172656E743A220053554206
:10354000524F5554494E452043414C4C20746172B2
:103550006765743A2200747279696E6720746F200F
:1035600063616C6C207375622D67636F64652066A0
:10357000696C6573207769746820746F6F206D6162
:103580006E79206C6576656C732E204D4158206CE9
:103590006576656C2069733A310A004D3234004D0E
:1035A00032332025730053442063617264206F6BB3
:1035B0000A006F70656E526F6F74206661696C658A
:1035C000640A00766F6C756D652E696E697420668D
:1035D00061696C65640A00534420696E69742066F1
:1035E00061696C0A00286E6F2066696C652900436A
:1035F000616E6E6F74206F70656E207375626469A2
:103600007220007C3C3E5E2B3D3F2F5B5D3B2C2AB5
:10361000225C004F4646004F4E006563686F3A00DB
:103620004572726F723A004572726F7220777269DA
:1036300074696E6720746F20454550524F4D210AC2
:1036400000507265737320627574746F6E20286FFA
:1036500072204D3130382920746F206865617420E4
:103660006E6F7A7A6C650A005072657373206275AA
:1036700074746F6E20286F72204D31303829207499
:103680006F20726573756D650A00496E736572749B
:103690002066696C616D656E7420616E6420707265
:1036A00065737320627574746F6E20286F72204D7D
:1036B000313038290A004D3630303A20546F6F20AF
:1036C000636F6C6400486F74656E6420746F6F2064
:1036D000636F6C640A00486F74656E6420746F6F6A
:1036E00020636F6C640A00496E73657274206669AA
:1036F0006C616D656E7420616E64207072657373A9
:1037000020627574746F6E20286F72204D313038CE
:10371000290A0063616E63656C00726573756D657F
:103720006400726573756D65007061757365640022
:10373000706F7765726F6666002F2F616374696FB3
:103740006E3A0020573A0020573A00486F74656E71
:103750006420256320436F6F6C696E672E2E2E00E8
:10376000486F74656E642025632048656174696ED6
:10377000672E2E2E00202F002040002042403A00CD
:1037800020403A004D383420582059205A20450016
:10379000546865726D616C2052756E617761790055
:1037A000486F74656E64203120544845524D414C39
:1037B0002052554E4157415900486F74656E642040
:1037C0003220544845524D414C2052554E415741AC
:1037D000590042454420544845524D414C205255D1
:1037E0004E4157415900202D20496E76616C696425
:1037F000206578747275646572206E756D6265728D
:1038000020210A0048656174696E67206661696CF1
:103810006564004265642068656174696E6720664E
:1038200061696C656400546865726D616C205275E5
:103830006E617761790042454420544845524D41BC
:103840004C2052554E415741590048656174696E8C
:1038500067206661696C656400486F74656E6420FA
:10386000312048656174696E67206661696C6564C2
:1038700000486F74656E6420322048656174696E1B
:1038800067206661696C656400546865726D616C7F
:103890002052756E6177617900486F74656E64209F
:1038A0003120544845524D414C2052554E415741CC
:1038B0005900486F74656E64203220544845524D5B
:1038C000414C2052554E41574159004D494E5445A7
:1038D0004D502074726967676572656400486F7443
:1038E000656E642031204572723A204D494E544530
:1038F0004D5000486F74656E642032204572723AF4
:10390000204D494E54454D50004572723A204D4964
:103910004E54454D5020424544004D415854454D6C
:10392000502074726967676572656400486F7465DA
:103930006E642031204572723A204D415854454DF5
:103940005000486F74656E642032204572723A20D0
:103950004D415854454D50004572723A204D4158E2
:1039600054454D502042454400626564002C20734C
:10397000797374656D2073746F707065642120486D
:1039800065617465725F49443A2000236465666925
:103990006E652044454641554C545F004B64200001
:1039A0004B6920004B702000006265640050494460
:1039B000204175746F74756E652066696E697368F1
:1039C0006564212050757420746865206C6173747F
:1039D000204B702C204B6920616E64204B64206367
:1039E0006F6E7374616E74732066726F6D206265A2
:1039F0006C6F7720696E746F20436F6E66696775B0
:103A0000726174696F6E2E680A00504944204175D6
:103A1000746F74756E65206661696C6564212074CD
:103A2000696D656F75740A00546865726D616C200C
:103A300052756E6177617900486F74656E642031EC
:103A400020544845524D414C2052554E4157415902
:103A500000486F74656E64203220544845524D41D1
:103A60004C2052554E41574159004245442054483C
:103A700045524D414C2052554E41574159004865E1
:103A80006174696E67206661696C656400486F7473
:103A9000656E6420312048656174696E67206661D7
:103AA000696C656400486F74656E642032204865F7
:103AB0006174696E67206661696C65640042656463
:103AC0002068656174696E67206661696C65640071
:103AD000504944204175746F74756E652066616944
:103AE0006C6564212054656D7065726174757265D2
:103AF00020746F6F20686967680A00204B643A2061
:103B000000204B693A2000204B703A20000A2043E5
:103B10006C617373696320504944200A0020547516
:103B20003A2000204B753A2000206D61783A200041
:103B3000206D696E3A200020643A2000206269619D
:103B4000733A2000504944204175746F74756E6556
:103B50002073746172740A00504944204175746F77
:103B600074756E65206661696C6564212054656DAD
:103B7000706572617475726520746F6F2068696713
:103B8000680A001000AD0330016A0150022B017079
:103B9000030A019004F500B005E500D006D800F056
:103BA00007CE001009C500300ABE00500BB70070E8
:103BB0000CB100900DAB00B00EA600D00FA200F02B
:103BC000109D00101299003013950050149200704F
:103BD000158E0090168B00B0178700D0188400F067
:103BE000198100101B7E00301C7B00501D79007075
:103BF0001E7600901F7300B0207000D0216E00F080
:103C0000226B001024690030256600502663007086
:103C100027610090285E00B0295C00D02A5900F08E
:103C20002B5600102D5400302E5100502F4E007096
:103C3000304B0090314800B0324500D0334200F0A4
:103C4000343E0010363B00303737005038330070B8
:103C5000392E00903A2900B03B2300D03C1B00F0E5
:103C60003D1100103F0100F03F00001000C902109C
:103C7000012C014001220170011801B0010E01F078
:103C80000104015002FA00B002F0003003E600D057
:103C900003DC009004D2007005C800A006BE00003E
:103CA00008B400B009AA00D00BA000600E96006016
:103CB000118C000015820020197800C01D6E00A034
:103CC000226400B0275A00902C500000314600E0DA
:103CD000343C0010383200903A2800603C1E00A0AE
:103CE0003D1400803E0A00203F00006F70656E00AA
:103CF000545249474745524544003A20007A5F7084
:103D0000726F6265007A5F6D696E00795F6D6178D0
:103D100000795F6D696E00785F6D617800785F6D26
:103D2000696E005265706F7274696E6720656E64AB
:103D300073746F70207374617475730A00456E64D8
:103D400073746F70732025632025632025632025FD
:103D5000630020503A00205A3A0020593A00205877
:103D60003A00656E6473746F7073206869743A20EA
:103D700000486F6D696E67206661696C6564004913
:103D80006E76616C69642065787472756465720A18
:103D90000041637469766520457874727564657254
:103DA0003A200045313A200045303A20005A3A2066
:103DB00000593A20004D53312C4D53322C4D533382
:103DC0002050696E730A583A20004D6963726F7310
:103DD0007465707320756E617661696C61626C6583
:103DE0000A00205A3A0020593A0020436F756E7439
:103DF00020583A00C23100001C260000F4190000CF
:103E0000D80F0000EB080000C0040000750200009D
:103E10004001000024F4D43050C38E20C2A24017C9
:103E2000828B7011127A910D816CD90AA861E10818
:103E3000C7586607615143061E4B5D05C145A7047F
:103E40001A411104093D9803713931034036DB02F0
:103E500065339102D4305402802E1D02632CEE0192
:103E6000752AC501B028A001102781018F256401A2
:103E70002B244B01E0223401AC211F018D200D01C8
:103E8000801FFC00841EED00971DDF00B81CD200CF
:103E9000E61BC600201BBC00641AB200B219A800C1
:103EA0000A19A0006A189900D117910040178B00D9
:103EB000B516840031167E00B31579003A157300EB
:103EC000C7146F0058146A00EE136600881363006D
:103ED00025135E00C7125B006C12570015125400C8
:103EE000C111510070114F0021114B00D610490033
:103EF0008D1047004610440002104200C00F4000E1
:103F0000800F3E00420F3C00060F3B00CB0E3800F6
:103F1000930E37005C0E3500270E3400F30D32008F
:103F2000C10D3100900D3000600D2E00320D2D00BE
:103F3000050D2C00D90C2B00AE0C2900850C290096
:103F40005C0C2700350C27000E0C2600E80B240023
:103F5000C40B2400A00B23007D0B23005A0B21006F
:103F6000390B2100180B2000F80A1F00D90A1E0087
:103F7000BB0A1E009D0A1D00800A1D00630A1C006A
:103F8000470A1B002C0A1B00110A1A00F7091A0025
:103F9000DD091900C4091900AB09190092091700BD
:103FA0007B091800630917004C0916003609160032
:103FB000200916000A091500F5081500E00814008C
:103FC000CC081400B8081400A408140090081300CA
:103FD0007D0812006B0813005808120046081200F2
:103FE0003408110023081100120811000108110003
:103FF000F0071000E0071000D0071000C007100005
:10400000B0070F00A107100091070E0083070F00F3
:1040100074070F0065070E0057070E0049070E00D2
:104020003B070D002E070E0020070D0013070D00A3
:1040300006070D00F9060C00ED060D00E0060C0069
:10404000D4060C00C8060C00BC060C00B0060C0020
:10405000A4060B0099060C008D060B0082060B00CF
:1040600077060B006C060B0061060A0057060B0072
:104070004C060A0042060A0038060A002E060A000C
:1040800024060A001A060A001006090007060A009C
:10409000FD050900F4050900EB050900E20509002A
:1040A000D9050900D0050900C7050900BE050900AA
:1040B000B5050800AD050800A50509009C05080028
:1040C000940508008C050800840508007C0508009C
:1040D000740508006C050700650508005D0507000C
:1040E000560508004E050700470507004005080073
:1040F00038050700310507002A05070023050700DA
:104100001C050600160507000F0507000805060038
:1041100002050700FB040600F5040700EE04060094
:10412000E8040600E2040700DB040600D5040600EC
:10413000CF040600C9040600C3040600BD0406003F
:10414000B7040600B1040500AC040600A60406008E
:10415000A00405009B0406009504050090040600D9
:104160008A04050085040500800406007A04050021
:1041700075040500700405006B0405006604050065
:10418000610405005C0405005704050052040500A5
:104190004D04050048040500430405003E040400E6
:1041A0003A04050035040500300404002C04050021
:1041B00027040400230405001E0404001A0404005C
:1041C00016040500110404000D0404000904050090
:1041D0000404040000040400FC030400F8030400C9
:1041E000F4030400F0030400EC030400E8030400FB
:1041F000E4030400E0030400DC030400D80304002B
:10420000D4030400D0030400CC030400C80303005B
:10421000C503030024F404D9201BC40C5C0E9804CD
:10422000C4095F0265077101F405F900FB04B300DE
:1042300048048700C1036900580355000303450083
:10424000BE023A008402310053022A0029022500EE
:1042500004022000E4011C00C8011900AF0117008E
:104260009801140084011300710110006101100015
:1042700051010E0043010D0036010B002B010B0014
:1042800020010B00150109000C01090003010800C1
:10429000FB000800F3000800EB000700E400060044
:1042A000DE000600D8000600D2000600CC000500A3
:1042B000C7000500C2000500BD000400B9000400ED
:1042C000B5000400B1000400AD000400A900040022
:1042D000A5000300A20003009F0004009B00030050
:1042E0009800030095000200930003009000030073
:1042F0008D0002008B00030088000200860002008F
:1043000084000300810002007F0002007D000200A3
:104310007B000200790002007700010076000200B5
:104320007400020072000100710002006F000200C0
:104330006D0001006C0002006A00010069000200CB
:1043400067000100660001006500010064000200D2
:104350006200010061000100600001005F000200D6
:104360005D0001005C0001005B0001005A000100DB
:1043700059000100580001005700010056000100DB
:1043800055000100540001005300000053000100DB
:104390005200010051000100500001004F000100D7
:1043A0004E0000004E0001004D0001004C000100D5
:1043B0004B0000004B0001004A00010049000100D1
:1043C00048000000480001004700010046000000CE
:1043D00046000100450000004500010044000100C6
:1043E00043000000430001004200000042000100C1
:1043F0004100000041000100400001003F000000BA
:104400003F0001003E0000003E0001003D000000B2
:104410003D0001003C0000003C0000003C000100A9
:104420003B0000003B0001003A0000003A000100A0
:104430003900000039000100380000003800000099
:10444000380001003700000037000100360000008E
:104450003600000036000100350000003500000085
:104460003500010034000000340000003400010079
:104470003300000033000000330001003200000070
:104480003200000032000100310000003100000065
:104490003100010030000000300000003000010059
:1044A0002F0000002F0000002F0000002F0001004F
:1044B0002E0000002E0000002E0001002D00000044
:1044C0002D0000002D0000002D0001002C00000038
:1044D0002C0000002C0000002C0001002B0000002C
:1044E0002B0000002B0000002B0001002A00000020
:1044F0002A0000002A0000002A0001002900000014
:104500002900000029000000290000002900010006
:1045100028000000280000002800000028000000FB
:1045200028000100270000002700000027000000ED
:1045300027000000270001002600000026000000E0
:1045400026000000260000002600010025000000D3
:1045500025000000250000002500000025000000C7
:1045600025000100240000002400000024000000B9
:1045700024000000240001002300000023000000AC
:10458000230000002300000023000000230000009F
:104590002300010022000000220000002200000091
:1045A0002200000022000000220001002100000083
:1045B0002100000021000000210000002100000077
:1045C0002100000021000100200000002000000068
:1045D000200000002000000020000000200000005B
:1045E00020000000200001001F0000001F0000004C
:1045F0001F0000001F0000001F0000001F0000003F
:104600001F0001001E0000001E0000001E00000030
:104610001E00000020204D36303320003A0A0020D2
:10462000286D6D2900205300205A00205900205881
:104630000020204D3432352046004261636B6C61AE
:10464000736820636F6D70656E736174696F6E3A25
:104650000A00546F6F6C2D6368616E67696E673A0C
:104660000A002055005431204C00205500543020C1
:104670004C0046696C616D656E74206C6F61642FCF
:10468000756E6C6F6164206C656E677468733A0A4E
:1046900000204B0020204D3930302054004C696EF2
:1046A00065617220416476616E63653A0A0020207C
:1046B0004D383531205A005A2D50726F6265204FA7
:1046C00066667365740020440020490020204D3345
:1046D000303420500020440020490020204D333049
:1046E0003120500020440020490020500020204D5F
:1046F0003330312045005049442073657474696E2D
:1047000067733A0A0020460020420020480020201B
:104710004D3134352053004D6174657269616C20F0
:1047200068656174757020706172616D6574657221
:10473000733A0A0020204D34323020530041757402
:104740006F20426564204C6576656C696E673A0A35
:104750000020590020580020204D323138205400CC
:10476000486F74656E64206F6666736574733A0A89
:1047700000204500205A00205900205800205400F5
:1047800020530020204D32303520420020453C6D22
:1047900061785F655F6A65726B3E0020583C6D61B1
:1047A000785F785F6A65726B3E20593C6D61785F17
:1047B000795F6A65726B3E205A3C6D61785F7A5F03
:1047C0006A65726B3E00416476616E6365643A208F
:1047D000423C6D696E5F7365676D656E745F746989
:1047E0006D655F75733E20533C6D696E5F666565F0
:1047F00064726174653E20543C6D696E5F747261D1
:1048000076656C5F66656564726174653E00205410
:104810000020520020204D3230342050004163638C
:10482000656C65726174696F6E2028756E6974734A
:104830002F7332293A20503C7072696E745F616345
:1048400063656C3E20523C726574726163745F6193
:104850006363656C3E20543C74726176656C5F6185
:104860006363656C3E0A0020450020204D323031E4
:10487000205400205A0020590020204D3230312091
:1048800058004D6178696D756D20416363656C6595
:10489000726174696F6E2028756E6974732F73323C
:1048A000293A0A0020450020204D323033205400A0
:1048B000205A0020590020204D3230332058004D1E
:1048C0006178696D756D2066656564726174657384
:1048D0002028756E6974732F73293A0A0053746522
:1048E00070732070657220756E69743A0A0020201A
:1048F0004D3134392043203B20556E697473206953
:104900006E2043656C736975730A0020204732314D
:10491000202020203B20556E69747320696E206D25
:104920006D0048617264636F64656420446566610C
:10493000756C742053657474696E6773204C6F6175
:104940006465640A00282300002823000064000036
:104950000028230000282300000000964300009652
:1049600043000040400000C8410000C8410000C9A9
:10497000420000C9420000C84400804F4400804FFC
:1049800044454550524F4D20496E697469616C69C8
:104990007A65640A00290A002062797465733B20F5
:1049A00063726320002073746F7265642073657492
:1049B00074696E67732072657472696576656420C8
:1049C0002800202863616C63756C6174656429211B
:1049D0000A0020213D2000454550524F4D204352B2
:1049E00043206D69736D61746368202D2028737492
:1049F0006F7265642920002053697A653A20004966
:104A00006E6465783A2000204D61726C696E3D5687
:104A10003638290A00454550524F4D20766572734D
:104A2000696F6E206D69736D6174636820284545F8
:104A300050524F4D3D00290A002062797465733B46
:104A400020637263200053657474696E677320532A
:104A5000746F7265642028000A003B20454550525F
:104A60004F4D20496E6465783A200055706461743A
:104A7000696E67207A6F666673657420696E20457B
:104A80004550524F4D3A2000454550524F4D2064FD
:104A900061746173697A65206572726F722E0A00A3
:104AA0004175746F6C6576656C206661696C6564D0
:104AB0000A004175746F6C6576656C206661696C7F
:104AC0006564005761726E696E673A20486F6D6960
:104AD0006E672042756D702044697669736F72202D
:104AE0003C20310A00020204486F6D6520257325C1
:104AF000732573206669727374002066697273741B
:104B00000A00486F6D65200020746F6F206C6F6E17
:104B10006720657874727573696F6E207072657640
:104B2000656E7465640A0020636F6C642065787438
:104B3000727573696F6E2070726576656E746564E8
:104B40000A0020453A00205A3A0020593A00583AC3
:104B500000000048420000484200004040FF01FFC2
:104B60000000A0400000A0400000004000009B4367
:104B70000080A143000087430000B0C1008097433C
:104B8000000000000000904300809743000087432E
:104B90000000B0C10000A0C10000000020746F6FD1
:104BA000206C6F6E6720657874727573696F6E2004
:104BB00070726576656E7465640A0020636F6C645C
:104BC00020657874727573696F6E20707265766592
:104BD0006E7465640A00627573793A20706175734A
:104BE000656420666F7220696E7075740A00627564
:104BF00073793A2070617573656420666F722075F1
:104C00007365720A00627573793A2070726F63651A
:104C10007373696E670A004D3131372050726F62CD
:104C200065207375636365737366756C0A0020494C
:104C30006E76616C69642065787472756465722043
:104C400000205A3A200020593A200042656420583A
:104C50003A200050726F6265205A204F6666736575
:104C6000743A20003F5A206F7574206F662072617D
:104C70006E676520282D3220746F2035290A004D7B
:104C800031343520533C696E6465783E206F75740D
:104C9000206F662072616E67652028302D31290AE9
:104CA00000436C69636B20746F20726573756D656A
:104CB0002E2E2E00220A00556E6B6E6F776E2063CB
:104CC0006F6D6D616E643A202200454550524F4D24
:104CD000204F4B0A004E6F206D6F76652E004543C6
:104CE000484F00494E464F004552524F52530044E0
:104CF000525952554E00434F4D4D554E4943415424
:104D0000494F4E006F666600DE4CE34CE84CEF4CBA
:104D1000F64C44454255473A004C756C7A426F74E4
:104D20002054415A2036204F46462E00205A00205B
:104D30005900580020204D61783A2000205A002068
:104D40005900580020204D696E3A2000536F667458
:104D500020656E6473746F70733A20002569730068
:104D600025696D20256973002569682025696D20F6
:104D700025697300256964202569682025696D20EF
:104D800025697300256979202569642025696820D3
:104D900025696D20256973005072696E74207469ED
:104DA0006D653A20004D3131332053002F2F200004
:104DB0004361703A004348414D4245525F54454D6E
:104DC0005045524154555245004D4F54494F4E5F46
:104DD0004D4F44455300544845524D414C5F50524D
:104DE0004F54454354494F4E004155544F5245503E
:104DF0004F52545F53445F535441545553005052E3
:104E00004F4D50545F535550504F525400454D45EF
:104E10005247454E43595F5041525345520043411A
:104E200053455F4C494748545F4252494748544EA6
:104E300045535300544F47474C455F4C49474854EE
:104E40005300534F4654574152455F504F574552B8
:104E5000004255494C445F50455243454E54004C26
:104E60004556454C494E475F44415441005A5F50B6
:104E7000524F4245004155544F4C4556454C005009
:104E800052494E545F4A4F420050524F4752455389
:104E900053004155544F5245504F52545F54454D65
:104EA0005000564F4C554D455452494300454550CE
:104EB000524F4D0042494E4152595F46494C455F61
:104EC0005452414E534645520053455249414C5F5E
:104ED000584F4E5F584F4646004649524D57415233
:104EE000455F4E414D453A4D61726C696E202046DA
:104EF00049524D574152455F56455253494F4E3ADC
:104F0000322E302E302E31343720455854525544ED
:104F100045525F545950453A4475616C45787472F6
:104F20007564657220763220534F555243455F4376
:104F30004F44455F55524C3A68747470733A2F2F42
:104F4000636F64652E616C6570686F626A65637417
:104F5000732E636F6D2F646966667573696F6E2F4C
:104F60004D41524C494E2050524F544F434F4C5F8D
:104F700056455253494F4E3A312E30204D41434809
:104F8000494E455F545950453A4C756C7A426F749E
:104F90002054415A20362045585452554445525FBA
:104FA000434F554E543A3220555549443A383435DA
:104FB00066303033632D616562642D346535332D81
:104FC000613662392D37643039383466646536307D
:104FD000390A002020536D6F6F7468696E6720284E
:104FE0006D6D293A20202020202020202020202004
:104FF0002020202020530020204261636B6C6173CD
:10500000682044697374616E636520286D6D293A68
:10501000202020202020202000202846312E302053
:105020003D2066756C6C2C2046302E30203D206E65
:105030006F6E65290A002020436F72726563746980
:105040006F6E20416D6F756E742F466164652D6FB4
:1050500075743A20202020204600616374697665CB
:105060003A0A00696E004261636B6C6173682043A9
:105070006F7272656374696F6E2000486F6D652092
:1050800058592066697273740A00486F6D6520581C
:105090005920666972737400426564204C657665B8
:1050A0006C696E6720004661696C656420746F20CE
:1050B000656E61626C6520426564204C6576656C46
:1050C000696E670A00426564204C6576656C204312
:1050D0006F7272656374696F6E204D617472697866
:1050E0003A000A0A426564204C6576656C20436F7D
:1050F0007272656374696F6E204D61747269783A7B
:1051000000202B000A436F7272656374656420424D
:105110006564204865696768742076732E2042654F
:105120006420546F706F6C6F67793A0A00202B000F
:105130000A4265642048656967687420546F706F1F
:105140006772617068793A0A2020202B2D2D2D205E
:105150004241434B202D2D2B0A2020207C20202053
:1051600020202020202020207C0A204C207C202071
:105170002020282B29202020207C20520A20452076
:105180007C20202020202020202020207C20490A54
:105190002046207C20282D29204E20282B29207CC9
:1051A00020470A2054207C2020202020202020205E
:1051B00020207C20480A2020207C20202020282D10
:1051C00029202020207C20540A2020207C20202000
:1051D00020202020202020207C0A2020204F2D2D40
:1051E0002046524F4E54202D2D2B0A2028302C3093
:1051F000290A003474682070726F626520706F69CC
:105200006E742C2064697374616E63652066726FBE
:105210006D20706C616E653A20002028445259520E
:10522000554E2900473239204175746F204265641C
:10523000204C6576656C696E67003F20284C2C52C7
:105240002C462C4229206F7574206F6620626F7582
:105250006E64732E0A003F50726F626520706F6932
:105260006E74732028592920697320696D706C61F0
:10527000757369626C652028322D32292E0A003F31
:1052800050726F626520706F696E747320285829A0
:1052900020697320696D706C61757369626C65203B
:1052A00028322D32292E0A003F2856296572626F56
:1052B0007365206C6576656C20697320696D706C10
:1052C00061757369626C652028302D34292E0A00BF
:1052D00043757272656E742066696C653A2000458C
:1052E0006E642066696C65206C6973740A0042659F
:1052F00067696E2066696C65206C6973740A004189
:105300006476616E6365204B003F4B2076616C755F
:1053100065206F7574206F662072616E6765202846
:10532000302D3130292E0A003F542076616C75658E
:10533000206F7574206F662072616E67652E0A009B
:105340004D31313720486F7420456E6420486561C7
:1053500074696E672E2E2E0A4D313034205331374A
:10536000302054300A4D31303420533137302054FE
:10537000310A473238204F310A473120593235201F
:105380005A31302046353030300A4D3131372052D5
:1053900065776970696E67206E6F7A7A6C650A54FA
:1053A000300A473120582D313720593733204635C0
:1053B0003030300A4D3130392052313730205430BE
:1053C0000A4D31303920523137302054310A4731BB
:1053D000205A310A473120582D3137205937332090
:1053E00046343030300A473120582D313720593972
:1053F000352046343030300A473120582D3137209F
:105400005937332046343030300A473120582D3157
:1054100037205939352046343030300A473120584A
:105420002D3137205937332046343030300A473158
:1054300020582D3137205939352046343030300A44
:10544000473120582D3137205937332046343030FA
:10545000300A473120582D3137205939352046340C
:105460003030300A473120582D313720593733201A
:1054700046343030300A473120582D3137205939E1
:10548000352046343030300A473120582D3137200E
:105490005937332046343030300A473120582D31C7
:1054A00037205939352046343030300A4731205AB8
:1054B00031350A4D3130362053323535200A4730E8
:1054C0002058302059300A4D313039205231363091
:1054D0002054300A4D313039205231363020543189
:1054E0000A4D3130370A004732380020466C6F775A
:1054F0003A2000205A0020643A0020693A002070C7
:105500003A00204500204D3932205400205A002016
:105510005900204D3932205800486F74656E642060
:105520006F6666736574733A0043290A0061626CA2
:10553000656420286D696E2074656D702000646953
:105540007300656E00436F6C6420657874727564D7
:105550006573206172652000205400205200416371
:1055600063656C65726174696F6E3A205000496EB4
:1055700076616C69642065787472756465720A007E
:1055800020643A0020693A0020703A00536C656547
:10559000702E2E2E0047322F473320626164207018
:1055A0006172616D65746572730A00326E64206E9B
:1055B0006F7A7A6C65205A3A200050726F626520CB
:1055C0005A204F66667365743A2000446F6E6520FA
:1055D000736176696E672066696C652E0A005344B4
:1055E0002072656164206572726F720A00446F6E8A
:1055F00065207072696E74696E672066696C650AF1
:10560000004D32390053544F505045442E20005025
:1056100072696E7465722073746F70706564206453
:10562000756520746F206572726F72732E204669E3
:105630007820746865206572726F7220616E6420D4
:10564000757365204D39393920746F207265737414
:105650006172742E202854656D7065726174757264
:10566000652069732072657365742E2053657420FC
:1056700069742061667465722072657374617274F6
:10568000696E67290A004E6F20436865636B737506
:105690006D2077697468206C696E65206E756D6227
:1056A00065722C204C617374204C696E653A200041
:1056B0004E6F20436865636B73756D2077697468FE
:1056C000206C696E65206E756D6265722C204C6170
:1056D0007374204C696E653A2000636865636B7370
:1056E000756D206D69736D617463682C204C6173F6
:1056F00074204C696E653A20004C696E65204E75C9
:105700006D626572206973206E6F74204C617374D2
:10571000204C696E65204E756D6265722B312C20B0
:105720004C617374204C696E653A20004D31313004
:1057300000526573656E643A2000204200205000DC
:105740006F6B00220A00656E7175657565696E671D
:10575000202200504944204175746F74756E652095
:105760006661696C656421204261642065787472A9
:1057700075646572206E756D6265720A00426564BB
:1057800020636F6F6C696E672E2E2E004265642059
:1057900068656174696E672E2E2E006F6B00473945
:1057A000310A4730205A313520463630300A4739E1
:1057B000300A4730205831373020593239302046AE
:1057C000333030300A4D313137205072696E7420D9
:1057D00061626F727465642E002020506C616E6E81
:1057E000657242756666657242797465733A200027
:1057F0002046726565204D656D6F72793A200043D1
:105800006F6D70696C65643A204A756C2032362081
:10581000323031390A00207C20417574686F723A49
:105820002028416C657068204F626A65637473203C
:10583000496E632E2C204C756C7A426F7420476938
:1058400074205265706F7369746F7279290A000051
:10585000204C61737420557064617465643A200053
:10586000322E302E302E3134370A004D61726C6981
:105870006E0020536F6674776172652052657365A0
:10588000740A00205761746368646F6720526573FF
:1058900065740A002042726F776E206F7574205213
:1058A000657365740A002045787465726E616C20BA
:1058B00052657365740A00506F77657255700A00FF
:1058C00073746172740A004B494C4C45442E20009D
:1058D0005072696E7465722068616C7465642E2004
:1058E0006B696C6C28292063616C6C6564210A000B
:1058F0004B494C4C20636175736564206279207458
:105900006F6F206D75636820696E61637469766579
:105910002074696D65202D2063757272656E742028
:10592000636F6D6D616E643A20004730205A3130EC
:105930000A4731320A4D31303920523136300A4D62
:105940003131372050726F62696E67206265640082
:1059500070726F62655F726577697065004175741A
:105960006F6C6576656C206661696C6564004D31AD
:10597000313720426564206C6576656C696E6720FE
:105980006661696C65642E0A4730205A31300A47D7
:10599000302045300A4D33303020503235205338D6
:1059A00038300A4D333030205035302053300A4DD6
:1059B0003330302050323520533838300A4D3330B0
:1059C00030205035302053300A4D333030205032A3
:1059D0003520533838300A47342053310070726F05
:1059E00062655F6661696C65640050726F746563BF
:1059F0007465642050696E0A0025301D0C18282932
:105A000024311C0B174527232F1B0A444316222B36
:105A10001A4142212A193F40033809FF3607FF3750
:105A200003060802020001004C46998BBC955DAB51
:105A30007DC8EE00EA00F000E800EC00DC951124DF
:105A40001FBECFEFD1E2DEBFCDBF00E00CBF14E040
:105A5000A0E0B2E0ECECF3EC02E00BBF02C0079078
:105A60000D92AC33B107D9F728E1ACE3B4E001C043
:105A70001D92AF30B207E1F71DE2CEE1DDE200E0BA
:105A800006C021970109802FFE010F94A059C4314F
:105A9000D10780E00807A9F70E94C8390D94D461A6
:105AA0000C9400001F920F920FB60F9211242F93A7
:105AB0003F938F939F93AF93BF9380913D049091B9
:105AC0003E04A0913F04B091400430913C0423E097
:105AD000230F2D3720F40196A11DB11D05C026E826
:105AE000230F0296A11DB11D20933C0480933D0419
:105AF00090933E04A0933F04B093400480914104EE
:105B000090914204A0914304B09144040196A11DD8
:105B1000B11D8093410490934204A0934304B09339
:105B20004404BF91AF919F918F913F912F910F901E
:105B30000FBE0F901F9018952FB7F89460913D04F9
:105B400070913E0480913F04909140042FBF0895CE
:105B50003FB7F8948091410490914204A09143048E
:105B6000B091440426B5A89B05C02F3F19F00196BB
:105B7000A11DB11D3FBFBA2FA92F982F8827820FD3
:105B8000911DA11DB11DBC01CD0142E0660F771F23
:105B9000881F991F4A95D1F708958F929F92AF92CF
:105BA000BF92CF92DF92EF92FF926B017C01D0DF28
:105BB0004B015C01C114D104E104F104F1F09CD368
:105BC000C7DFDC01CB0188199909AA09BB09883E06
:105BD0009340A105B10570F321E0C21AD108E10894
:105BE000F10888EE880E83E0981EA11CB11CC11438
:105BF000D104E104F10421F7DDCFFF90EF90DF90B5
:105C0000CF90BF90AF909F908F9008958230910574
:105C100038F0880F991F880F991F05970197F1F7A2
:105C20000895789484B5826084BD84B5816084BD14
:105C300085B5826085BD85B5816085BDEEE6F0E005
:105C4000808181608083E1E8F0E010828081826061
:105C50008083808181608083E0E8F0E080818160E2
:105C60008083E1EBF0E0808184608083E0EBF0E012
:105C7000808181608083E1E9F0E0808182608083BF
:105C8000808181608083E0E9F0E0808181608083B1
:105C9000E1EAF0E08081826080838081816080839E
:105CA000E0EAF0E0808181608083E1E2F1E08081E0
:105CB00082608083808181608083E0E2F1E0808186
:105CC00081608083EAE7F0E0808184608083808166
:105CD000826080838081816080838081806880830E
:105CE0001092C10008951F93CF93DF93182FEB01FB
:105CF00061E016D1209711F460E004C0CF3FD105D8
:105D000031F461E0812FDF91CF911F9145C1E12FE7
:105D1000F0E0E15EFD4FE4914E2F50E0FA01319743
:105D2000E231F10508F09DC08827EE58FF4F8F4FF4
:105D30000D94A05984B5806884BDC7BD97C084B553
:105D4000806284BDC8BD92C08091800080688093CD
:105D50008000D0938900C093880088C08091800023
:105D6000806280938000D0938B00C0938A007EC0B5
:105D700080918000886080938000D0938D00C093D4
:105D80008C0074C08091B00080688093B000C09394
:105D9000B3006CC08091B00080628093B000C0936B
:105DA000B40064C080919000806880939000D0938C
:105DB0009900C09398005AC08091900080628093AF
:105DC0009000D0939B00C0939A0050C080919000A7
:105DD000886080939000D0939D00C0939C0046C043
:105DE0008091A00080688093A0008091A0008F7BAC
:105DF0008093A000D093A900C093A80037C08091E1
:105E0000A00080628093A000D093AB00C093AA0052
:105E10002DC08091A00088608093A000D093AD0039
:105E2000C093AC0023C08091200180688093200142
:105E3000D0932901C093280119C08091200180626C
:105E400080932001D0932B01C0932A010FC0809131
:105E50002001886080932001D0932D01C0932C01F4
:105E600005C0C038D1050CF04CCF46CFDF91CF91A3
:105E70001F91089590E0FC013197E231F10508F09F
:105E80004EC08827EC57FF4F8F4F0D94A05980913B
:105E900080008F7703C0809180008F7D8093800089
:105EA000089580918000877FF9CF84B58F7702C0F5
:105EB00084B58F7D84BD08958091B0008F7703C035
:105EC0008091B0008F7D8093B00008958091900004
:105ED0008F7707C0809190008F7D03C080919000E4
:105EE000877F8093900008958091A0008F7707C0EE
:105EF0008091A0008F7D03C08091A000877F809358
:105F0000A0000895809120018F7707C08091200123
:105F10008F7D03C080912001877F809320010895A9
:105F2000CF93DF9390E0FC01EB59FD4F2491FC01EE
:105F3000E555FD4F8491882361F190E0880F991F0A
:105F4000FC01EB5DFC4FC591D491FC01E55FFC4F7A
:105F5000A591B491611109C09FB7F89488812095EB
:105F600082238883EC912E230BC0623061F49FB7AB
:105F7000F8943881822F809583238883EC912E2B8F
:105F80002C939FBF06C08FB7F894E8812E2B2883EF
:105F90008FBFDF91CF9108951F93CF93DF93282F69
:105FA00030E0F901E15EFD4F8491F901EB59FD4FBD
:105FB000D491F901E555FD4FC491CC23C1F0162FC2
:105FC000811158DFEC2FF0E0EE0FFF1FE55FFC4F73
:105FD000A591B4918FB7F894111105C09C91ED2F44
:105FE000E095E92302C0EC91ED2BEC938FBFDF919C
:105FF000CF911F910895CF93DF93282F30E0F901BF
:10600000E15EFD4F8491F901EB59FD4FD491F90107
:10601000E555FD4FC491CC2389F081112BDFEC2F86
:10602000F0E0EE0FFF1FEF50FD4FA591B491EC9102
:10603000ED2381E090E021F480E002C080E090E078
:10604000DF91CF91089508951F920F920FB60F928E
:1060500011240BB60F922F933F934F935F936F933F
:106060007F938F939F93AF93BF93EF93FF93E091B1
:106070000802F09109021995FF91EF91BF91AF913C
:106080009F918F917F916F915F914F913F912F9150
:106090000F900BBE0F900FBE0F901F9018951F9280
:1060A0000F920FB60F9211240BB60F922F933F93BE
:1060B0004F935F936F937F938F939F93AF93BF9310
:1060C000EF93FF93E0910A02F0910B021995FF9173
:1060D000EF91BF91AF919F918F917F916F915F9160
:1060E0004F913F912F910F900BBE0F900FBE0F90CD
:1060F0001F9018951F920F920FB60F9211240BB696
:106100000F922F933F934F935F936F937F938F9350
:106110009F93AF93BF93EF93FF93E0910C02F091A5
:106120000D021995FF91EF91BF91AF919F918F91C2
:106130007F916F915F914F913F912F910F900BBE87
:106140000F900FBE0F901F9018951F920F920FB6D1
:106150000F9211240BB60F922F933F934F935F939F
:106160006F937F938F939F93AF93BF93EF93FF931F
:10617000E0910E02F0910F021995FF91EF91BF91FE
:10618000AF919F918F917F916F915F914F913F91CF
:106190002F910F900BBE0F900FBE0F901F90189570
:1061A0001F920F920FB60F9211240BB60F922F93DE
:1061B0003F934F935F936F937F938F939F93AF938F
:1061C000BF93EF93FF93E0910402F09105021995BC
:1061D000FF91EF91BF91AF919F918F917F916F91BF
:1061E0005F914F913F912F910F900BBE0F900FBE7B
:1061F0000F901F9018951F920F920FB60F921124B7
:106200000BB60F922F933F934F935F936F937F93B0
:106210008F939F93AF93BF93EF93FF93E091060209
:10622000F09107021995FF91EF91BF91AF919F9166
:106230008F917F916F915F914F913F912F910F902F
:106240000BBE0F900FBE0F901F9018951F920F92CC
:106250000FB60F9211240BB60F922F933F934F93CB
:106260005F936F937F938F939F93AF93BF93EF93BE
:10627000FF93E0911002F09111021995FF91EF91B7
:10628000BF91AF919F918F917F916F915F914F914E
:106290003F912F910F900BBE0F900FBE0F901F904C
:1062A00018951F920F920FB60F9211240BB60F92F2
:1062B0002F933F934F935F936F937F938F939F930E
:1062C000AF93BF93EF93FF93E0911202F09113020B
:1062D0001995FF91EF91BF91AF919F918F917F9110
:1062E0006F915F914F913F912F910F900BBE0F9047
:1062F0000FBE0F901F90189508951F93CF93DF93B3
:10630000EC011D821C821F821E82198681E0888713
:1063100082E28A871F861E86FE01B396CE01C19651
:106320002FEF2193E817F907E1F711E018A3CE0149
:1063300022D61F8B188E198E80E48A8F1B8E8CE8D4
:1063400095E39AAB89ABDF91CF911F910895DB0163
:10635000ED91FC911994EF92FF921F93CF93DF93ED
:106360001F921F92CDB7DEB77C01DC01D196ED9173
:10637000FC91D29782E069837A83199520E030E01E
:106380004AE069817A81C701E2DF182FD701D196EF
:10639000ED91FC91D29783E01995D701D196ED91BB
:1063A000FC91D29780E01995812F0F900F90DF918B
:1063B000CF911F91FF90EF9008950F931F93CF936C
:1063C000DF93EC018B01E9A9FAA982E01995E9A90B
:1063D000FAA981E0199520E030E044E1B801CE014E
:1063E000B6DF9E012D5C3F4F47E1B801CE01AFDF24
:1063F000E9A9FAA980E0DF91CF911F910F9119943B
:10640000EF92FF921F93CF93DF93EC017B01E9A9F9
:10641000FAA982E01995E9A9FAA981E0199520E085
:1064200030E045E1B701CE0192DF182F882339F023
:106430009E012D5C3F4F47E1B701CE0188DFE9A9FE
:10644000FAA980E01995812FDF91CF911F91FF90DC
:10645000EF900895FC01448F258F9C01245E3F4FEF
:1064600042E375CFCF93DF931F92CDB7DEB79E0186
:106470002F5F3F4F46E46BDF89810F90DF91CF9113
:106480000895CF93DF931F92CDB7DEB79E012F5FA4
:106490003F4F47E45CDF89810F90DF91CF910895F2
:1064A00020E030E048E453CFCF93DF93EC016A81E2
:1064B0007B81D8DF88836A817B81CE01E2DF89839B
:1064C0006A817B81CE01ECDF8B879E012D5C3F4F83
:1064D0006A817B8147E1CE01DF91CF9138CFCF93A5
:1064E000DF93EC016A817B8136DF882319F0CE01CE
:1064F000DBDF81E0DF91CF9108958F929F92AF9281
:10650000BF92CF92EF920F93CF93DF931F921F9280
:10651000CDB7DEB74C015B012A834983EEDEF4017F
:10652000B382A282498147A32A8120A705A3E4A2BE
:10653000C3A2C4010F900F90DF91CF910F91EF9004
:10654000CF90BF90AF909F908F90C9CFFC01628198
:10655000738133CFCF93DF93EC01EE85FF853097C6
:1065600009F019956A817B81CE01DF91CF9148CFE7
:10657000362F242FFC0162817381432F6BCF0F9341
:10658000FC0182819381648F458F278F068F9F0145
:10659000245E3F4F4BE3BC01CF010F91D8CEFC01ED
:1065A00060A30895BF92CF92DF92EF92FF920F9374
:1065B0001F93CF93DF936C01D62FB42EC22F780197
:1065C000CC2369F0F701049120E04B2D6D2FC6011B
:1065D000D6DFFFEFEF1AFF0AC150D85FF1CFDF918E
:1065E000CF911F910F91FF90EF90DF90CF90BF90D0
:1065F00008958F929F92AF92BF92CF92DF92EF92C7
:10660000FF920F931F93CF93DF935C01C62EC42F8D
:10661000D22ED02F220F220F220F1ED0882379F0E6
:10662000DC0F8D2C912CCD1751F087012D2D4C2F87
:106630006C2DC501B7DFE80CF91CCF5FF4CFDF91FB
:10664000CF911F910F91FF90EF90DF90CF90BF906F
:10665000AF909F908F9008950F93FC010150040F0D
:1066600084A996A9941718F0081728F402C00817EF
:1066700050F0041740F42150260F83A995A99617CE
:1066800020F4281720F480E007C0281720F481E0C8
:10669000261710F0F8CF81E00F91089581E008955A
:1066A0002EE93FE0009729F0F9013197F1F70197C2
:1066B000F9CF0895FC011282808181508383148276
:1066C0000895FC0180819281980F92832181921715
:1066D00060F494819F5F94839381890F821710F0F7
:1066E0008FEF820F838381E0089580E00895FC019D
:1066F00091E08381861708F490E031E0461708F0B6
:1067000030E0832F892B21E05281451708F420E0E7
:106710002823832F8923822B0895DC01FB0110821B
:1067200012968C911297818315968C9115978150B2
:10673000828313968C9183830895FB014181238189
:10674000213029F0233031F468EF640F04C0642F46
:10675000485F01C0642FCBCFDC0115962C911597B3
:106760001696ED91FC911797CF01820F911D820F24
:10677000911D1192E817F907E1F70895FC01A68130
:10678000B7818281481B8581483018F0A80FB11D60
:106790004770382F369536953695562F577080E8C6
:1067A00090E002C0959587955A95E2F7439F402D5A
:1067B0001124669566956695E62FF0E0E40FF11DCD
:1067C000EA0FFB1F3081222311F0832B02C080953A
:1067D000832380830895FB014181DC0112962C9173
:1067E0001297421760F013962C911397241738F0E4
:1067F000608115962C91621710F42481BFCF089503
:10680000CF92DF92FF920F931F93CF93DF936C0190
:10681000EB01FA809B81913051F030F0923049F0D9
:10682000933051F41FEF09C010E001E007C011E000
:1068300004C010E00FEF02C010E000E0F7FE03C05C
:10684000BE01C601C8DF9881900F98839981910F8E
:106850009983FF0C99F7DF91CF911F910F91FF90D2
:10686000DF90CF9008950F931F93CF93DF9389010B
:10687000FB01C281D3814233D9F058F44531E1F0B4
:10688000473109F1443141F5CE0166DFCE0112DF17
:1068900023C04634E1F04734E1F04B33E9F4B90169
:1068A000CE014BDF8823C1F0B801CE01A9DF14C0AF
:1068B000B901CE0190DF10C0CE0103DF882369F05B
:1068C000CE014ADF09C0B901CE0127DF05C08D81A5
:1068D00001C08981F801808381E0DF91CF911F9110
:1068E0000F910895CF92DF92EF92FF920F931F9333
:1068F000CF93DF937C01D62FD42EC22F122FC62E1A
:10690000C20E6C2D611B183038F00FEF20E04D2DBA
:10691000C70135DE1850F5CF6C2F687F6D0F2C2F17
:10692000277071F097E029272F5F27700FEF10E095
:1069300001C0000F2A95EAF720E04D2DC7011FDEA8
:10694000DF91CF911F910F91FF90EF90DF90CF904B
:106950000895CF92DF92EF92FF920F931F93CF9300
:10696000DF937C01D62ED42FC22F122FC42EC20E3D
:106970004C2D411B183038F00FEF21E06D2DC70171
:10698000FEDD1850F5CF4C2F487F4D0F2C2F277070
:1069900071F097E029272F5F27700FEF10E001C0FB
:1069A000000F2A95EAF721E06D2DC701E8DDDF91A0
:1069B000CF911F910F91FF90EF90DF90CF900895AE
:1069C000EF92FF920F931F93CF93DF93EC01162F5B
:1069D000F42EE22E01E040DE882359F02E2D4F2DBB
:1069E000612FCE01DF91CF911F910F91FF90EF901A
:1069F00079CFDF91CF911F910F91FF90EF90089584
:106A0000EF92FF920F931F93CF93DF93EC01162F1A
:106A1000F42EE22E022F21E01FDE882359F02E2DC6
:106A20004F2D612FCE01DF91CF911F910F91FF90DC
:106A3000EF908FCFDF91CF911F910F91FF90EF904B
:106A40000895DF92EF92FF920F931F93CF93DF93FE
:106A50007C01162FC42FD22ED02FFEDD8823F9F013
:106A60002D2D4C2F612FC7013DDF2D2F4C2F612F76
:106A7000C7016FDF6FEF6D0D610F2D2F4C2FC70119
:106A800068DF4FEF4D0F4C0F2D2D612FC701DF91A8
:106A9000CF911F910F91FF90EF90DF9023CFDF9167
:106AA000CF911F910F91FF90EF90DF900895EF929B
:106AB000FF920F931F93CF93DF937C01D62F122F5A
:106AC000C42F040F212F4C2F6D2FC7010BDFCF5F79
:106AD0000C13F8CFDF91CF911F910F91FF90EF90A2
:106AE0000895DF92EF92FF920F931F93CF93DF935E
:106AF000EC01162FF42EE22EAFDD882329F02E2D87
:106B00004F2D612FCE01D3DFDF91CF911F910F91D8
:106B1000FF90EF90DF9008950895FC01E60FF11DBE
:106B2000849190E0982F88273196E4918E0F911DE3
:106B30000895FC0184910895FCDF882321F08230C0
:106B400011F083E0089586E0089580E00895FC0147
:106B50008081089566E0E1CF68E0DFCF0A96FC010E
:106B6000849108950B96FC0184910895DC0114969C
:106B7000ED91FC911597319684910895BF92CF9233
:106B8000DF92EF92FF920F931F93CF93DF938C01CD
:106B9000E62EDC011496CD91DC911597CE01C9DF6C
:106BA000F82EF80184819581C7DFC82EF1E0FF122D
:106BB00003C02FE0B22E02C0BB24BA94D8011496B1
:106BC0008D919C911597CADFF82EF80184819581EB
:106BD000C9DFD82ED80114968D919C911597BCDFF2
:106BE000B0E6BE1538F4009729F0C80FD91F91E61A
:106BF000F92E0FC0F80184819581ACDFF0E4FE1519
:106C000038F4009729F0C80FD91F81E4F82E01C08D
:106C10006196DE1490F4D80150961C9250975396CA
:106C20001C92539754961C92549751961C925197CC
:106C300052961C9280E090E066C0DF1460F38C2DC9
:106C400090E0FE0124912F3F11F4219657C0FE10D1
:106C50004CC0D80114968D919C9115976ADF9E01C6
:106C60002F5F3F4FFE01882311F08230E1F48491C1
:106C7000D80153968C935397F901249154962C93F1
:106C80005497FE013396E4915096EC935097FE0191
:106C90003496E4915196EC935197FE013596E49128
:106CA0005296EC9320C08491982F9F709250D801F7
:106CB00052969C93529782958F7051968C935197D0
:106CC000F9012491822F8F7054968C9354972295BA
:106CD0002F7053962C935397FE013296E491E295D0
:106CE000EF705096EC93CE010EC0FE013296E49107
:106CF000EB219C012E0F311DC20FD31FFD1409F48F
:106D00008ACFF3949ECFDF91CF911F910F91FF9087
:106D1000EF90DF90CF90BF9008954F925F926F9267
:106D20007F929F92AF92BF92CF92DF92EF92FF92AB
:106D30000F931F93CF93DF931F92CDB7DEB72C0134
:106D4000C62E942E622F1ADF7C01892B09F43AC0DB
:106D5000F20184819581F0DEB82EF2011389048955
:106D60008189C80E8289981AD92CD01A212F4D2DCD
:106D70006C2DC20171DC882311F1EB0CF11C195F41
:106D8000169516951695612E712CD914C1F03C2DCF
:106D900057018A2D8E19811770F4F501049120E0B6
:106DA0004D2D632FC2013983EADBFFEFAF1ABF0A13
:106DB0003981385FEECFE60CF71CD394E6CFF201B1
:106DC000808901C080E00F90DF91CF911F910F91DA
:106DD000FF90EF90DF90CF90BF90AF909F907F900B
:106DE0006F905F904F9008950F931F93CF93DF9311
:106DF00000D0CDB7DEB78C01DC015596ED91FC914A
:106E000056972B834A83698319954A81480F2B81B2
:106E10006981C8010F900F900F90DF91CF911F9162
:106E20000F917BCFAF92BF92DF92EF92FF920F93C1
:106E30001F93CF93DF931F921F92CDB7DEB77C01D4
:106E4000D62E042FDC015596ED91FC91569729839F
:106E50003A831995080F2981A22E3A81B32E10E0AA
:106E6000F50121915F01222339F0402F6D2DC701DB
:106E700054DFD80E180FF4CF812F0F900F90DF91B1
:106E8000CF911F910F91FF90EF90DF90BF90AF9047
:106E90000895DF92EF92FF920F931F93CF93DF93AA
:106EA0007C01D62FD42E8901DC015596ED91FC9101
:106EB00056971995D80EC0E0F8012491222349F085
:106EC0004D2D6D2FC70129DFD80FC80F0F5F1F4F42
:106ED000F3CF8C2FDF91CF911F910F91FF90EF9007
:106EE000DF900895DC0114962D913C9115972115A2
:106EF000310509F43FC057968C915797F9018111DC
:106F000008C03596E4915896EC935897F9013C9651
:106F100011C0813041F43F96E4915896EC93589714
:106F2000F901709607C03D96E4915896EC935897F6
:106F3000F9013E96E4915996EC93599758968C91A5
:106F40005897082E000C990B59962C915997821B33
:106F5000910927FD93955A962C915A97203441F028
:106F6000829FC001112426E0969587952A95E1F726
:106F70005B968C93089525EA35E3FC01368B258BCF
:106F80000895CF92DF92EF92FF920F931F93CF93CA
:106F9000DF938C017B016A01CB01FA011995D82F8F
:106FA000882311F1682FC801E9DDF801C189C19575
:106FB000FFEFEF1AFF0AC701F6011995F8018823C0
:106FC00051F08089C80FC701F6011995D82F682F95
:106FD000C801D4DDEDCFD03221F091898389890FAA
:106FE00001C080898C0F01C080E0DF91CF911F919B
:106FF0000F91FF90EF90DF90CF90089547EA55E30F
:10700000C0CFCF93DF93FC0124813581261737074A
:1070100041F0EC017583648365DF85EA95E39E8B1F
:107020008D8BDF91CF910895CF93DF9300D01F9286
:10703000CDB7DEB7611571058105910579F09B012A
:10704000AC0169833A834B835C830F94105A298186
:107050003A814B815C810F94845903C060E070E0F9
:10706000CB010F900F900F900F90DF91CF9108956B
:10707000CF92DF92EF92FF920F931F9362177307E5
:10708000840795077CF489019A016B017C01C90191
:10709000B8016C197D098E099F09C6DF6C0D7D1D35
:1070A0008E1D9F1D1F910F91FF90EF90DF90CF904D
:1070B00008954F925F926F927F92AF92BF92CF925C
:1070C000DF92EF92FF920F931F93CF93DF93CDB791
:1070D000DEB729013A019B01AC01241935094609A3
:1070E00057098A899B89AC89BD89BC01CD016A1980
:1070F0007B098C099D090F942059A8019701241937
:107100003509460957090F948459CA01B9016A0D16
:107110007B1D8C1D9D1DDF91CF911F910F91FF90C5
:10712000EF90DF90CF90BF90AF907F906F905F9087
:107130004F90089580E090E008950895CF92DF92F7
:10714000EF92FF920F931F93CF93DF936C017A011D
:107150008B01C0E0D0E0CE15DF0589F0D8016D913C
:107160008D01D601ED91FC910190F081E02DC601D9
:107170001995892B11F47E0102C02196ECCFC7012D
:10718000DF91CF911F910F91FF90EF90DF90CF9003
:1071900008956115710579F0FB0101900020E9F770
:1071A0003197AF01461B570BDC01ED91FC9102803A
:1071B000F381E02D199480E090E00895DC01ED91D9
:1071C000FC910190F081E02D19944F925F926F92A3
:1071D0007F92EF92FF920F931F93CF93DF93CDB7E0
:1071E000DEB7A1970FB6F894DEBF0FBECDBF7C010E
:1071F000FA01CB0119A2223008F42AE08E010F5DBA
:107200001F4F422E512C612C712CBF01A301920102
:107210000F946259F901CA01015011096A3014F43E
:10722000605D01C0695CD8016C93232B242B252B56
:1072300061F7B801C701ADDFA1960FB6F894DEBFC4
:107240000FBECDBFDF91CF911F910F91FF90EF90B7
:107250007F906F905F904F900895CF92DF92EF9262
:10726000FF920F931F93CF93DF93EC016A017B0191
:107270002115310579F4E881F9810190F081E02D43
:10728000642FDF91CF911F910F91FF90EF90DF90CE
:10729000CF9019942A303105D9F477FF18C06DE2E8
:1072A0008DDF8C0144275527BA014C195D096E0901
:1072B0007F092AE0CE0189DF800F911FDF91CF91F6
:1072C0001F910F91FF90EF90DF90CF9008952AE0EB
:1072D000B701A601CE01DF91CF911F910F91FF90D1
:1072E000EF90DF90CF9071CF9A01AB01770F660BD3
:1072F000770BB3CFCF93CFB7F8948091450481112A
:1073000027C0E0EEF2E08491EAE9F2E09491E82F00
:10731000F0E0EE0FFF1FEB5DFC4FA591B491EC91F7
:10732000E92321F461E085E30E94CC2F61E085E34D
:107330000E94902F8CB580618CBD8CB580648CBD13
:1073400061E084E30E94902F61E083E30E94902F2C
:10735000809145048F5F80934504CFBFCF910895FE
:10736000CF92EF920F93FC0113AE14AE15AE0496BC
:10737000C4D80F91EF90CF9008958EBD00000DB44A
:1073800007FEFDCF8EB5089580E090E00895089542
:107390000E94112EFCDF0F948454C0E0D0E00F94C3
:1073A0000F552097E1F30E940000F9CFE7E6F4E0E3
:1073B00083AF64AF08954AE050E0BC0187E694E0F3
:1073C00093CFEF92FF920F931F93CF93DF937A01A6
:1073D0006F3F71058105910509F048F487E694E057
:1073E000EDDE8BE694E0C2DB282F30E014C0C091C4
:1073F000A204D091A3044D2F50E0EC2FF0E08B01BC
:107400009C01BF018BE694E0A0D6C80FC093A204F4
:10741000D093A3049C01C901DF91CF911F910F91DB
:10742000FF90EF900895EF92FF920F931F93CF93E9
:10743000DF938B01C7E6D4E0FBACECAC4E2D50E003
:107440006F2D70E09C018BE694E0D7D6F80EFBAE72
:10745000ECAEDF91CF911F910F91FF90EF900895C7
:10746000EF92FF920F931F93CF93DF938B01C7E6A9
:10747000D4E0FBACECAC4E2D50E06F2D70E09C01E5
:107480008BE694E006D7F80EFBAEECAEDF91CF9121
:107490001F910F91FF90EF9008956FEF7FEFC3CF93
:1074A0004FEF5FEF8ECF0F931F93CF93DF931F921A
:1074B000CDB7DEB7082F8CEF96E00E940D84182F11
:1074C000863168F48CEF96E0E8DF153109F43DC0B1
:1074D00060E270E080E090E0E3DF1F5FF6CFCE0176
:1074E00001960E94B58760E870E09DDF8981853153
:1074F00020F56EE270E080E090E0D2DF1981143177
:10750000E1F06EE270E080E090E0CADF1331A9F0B4
:1075100089812EEF3FEF281B310986E0829FB00161
:10752000839F700D112460587F4F8CEF96E07BDFB6
:1075300060E270E080E090E0B3DF80914604801765
:1075400021F0009346040E9497870F90DF91CF911E
:107550001F910F9108952F923F924F925F926F92D9
:107560007F928F929F92AF92BF92CF92DF92EF92D3
:10757000FF920F931F93CF93DF93CDB7DEB7629740
:107580000FB6F894DEBF0FBECDBF8091F206882300
:1075900009F4A1C060918C0D70918D0D072E000C27
:1075A000880B990B0F94BA5611E02091880D3091F9
:1075B000890D40918A0D50918B0D0F941B58181610
:1075C0000CF010E06091A30D7091A40D072E000C3B
:1075D000880B990B0F94BA5620919F0D3091A00DF6
:1075E0004091A10D5091A20D0F941B5818160CF448
:1075F000126060915B0D70915C0D072E000C880B82
:10760000990B0F94BA562091570D3091580D409117
:10761000590D50915A0D0F941B5818160CF4106800
:1076200010935904C0907302D0907402E0907502D8
:10763000F090760220E030E0A901C701B6010F9476
:10764000185687FD05C020E030E040E05FE304C04D
:1076500020E030E040E05FEBC701B6010F943F55FA
:107660000F948756CB010F940C4ABC0184E594E03B
:107670000F948B5EC0907702D0907802E0907902F0
:10768000F0907A0220E030E0A901C701B6010F9422
:10769000185687FD05C020E030E040E05FE304C0FD
:1076A00020E030E040E05FEBC701B6010F943F55AA
:1076B0000F948756CB010F940C4ABC018FE494E0E1
:1076C0000F948B5E8BE792E00F941D4FBC0187E413
:1076D00094E00F948B5E0E944C86182F81E09BD61D
:1076E0002091590427FD03C042E102E002C048E0B6
:1076F0000CE080919F0490E044977CF48091A10479
:10770000841758F027FD6EC28CE696E17C0123E0D9
:1077100060E58BE694E00E94F93280919F04843109
:10772000B8F48091A104823098F0112309F45DC26D
:107730008091820D882309F458C28CED95E17C017B
:1077400002E123E042E068E68BE694E00E94F93231
:1077500080919F048C3108F06EC154E8A52E5DE045
:10776000B52E6EE6862E6DE0962E2EE02E87C12C6D
:10777000D12C73E0272E312CFC2C8091590490E001
:10778000A0E0B0E00C2C04C0B695A795979587951E
:107790000A94D2F7082F0170F50144805580668065
:1077A000778060857185072E000C880B990B0F94EC
:1077B000BA566F87788B898B9A8B80919F0484311E
:1077C00008F58091A1048830E8F0C114D10409F4CF
:1077D00012C260E2F601E55CFC4F2081EF2DE17002
:1077E0000E2E000CFF0BEE0FFF1F002309F400C24A
:1077F000E852FA4EE590F4900CE048E08BE694E015
:107800000E94F93280919F048830A0F5F4018081B4
:10781000111102C081112EC020E030E040E05FE392
:107820006F85788989899A890F943F550F94875677
:10783000CB010F94D6497C01FC018081803209F094
:10784000DEC1F7018181803209F0D7C101E0902FBC
:10785000990F900F67E08E858F5F891BA7DDC101AF
:10786000801B91098E0D9F1D18DE69E070E080E09D
:1078700090E016DE80919F048C3180F58091A10408
:10788000853160F120E030E040E05FE3C301B20108
:107890000F943F550F948756CB010F94D6497C0126
:1078A000FC018081803209F0AEC1F7018181803214
:1078B00009F0A7C101E0902F990F900F6CE18E8520
:1078C0008F5F891B73DDC101801B91098E0D9F1D88
:1078D000E4DD69E070E080E090E0E2DDFFEFCF1AE8
:1078E000DF0A2E85285E2E8747E1A40EB11C55E0E5
:1078F000850E911C2E3309F03FCF8090570D90904C
:10790000580DA090590DB0905A0D80915B0D90913B
:107910005C0D20919F042830B8F520914A0D11117B
:1079200002C0211131C0BC01990F880B990B0F9433
:10793000BA5620E030E040E05FE30F943F550F94EB
:107940008756CB010F94D6497C01FC01808180329F
:1079500009F05DC1F7018181803209F056C101E073
:10796000902F990F900F892F819567E0845A1EDD23
:1079700083E090E0801B91098E0D9F1D8EDD69E0F4
:1079800070E080E090E08CDD80919F048C3188F580
:107990008091A104853168F120E030E040E05FE3B0
:1079A000C501B4010F943F550F948756CB010F9436
:1079B000D6497C01FC018081803209F02CC1F7019D
:1079C0008181803209F025C101E0902F990F900F3D
:1079D000892F81956CE1845AE9DC83E090E0801B7B
:1079E00091098E0D9F1D59DD69E070E080E090E007
:1079F00057DD80919F048C31F0F48091A104853192
:107A0000D0F00091820D0023B1F06CE187E6CEDC6E
:107A1000F4E60F9FC001112481589F4F6FEF70E073
:107A20000F944F59CB010F94D64937DD65E270E0D2
:107A300080E090E035DD8091D60983FF28C08091F9
:107A40000608882321F180919F04843300F58091FA
:107A5000A1048A32E0F007E028E04AE26AE28BE61D
:107A600094E03FD805E022E04CE262E38BE694E04C
:107A700038D804E02AE041E36AE28BE694E00E9411
:107A800021354BE262E38BE694E00E94B8328091AC
:107A90009F04853328F48091A104813308F0BDC090
:107AA0000E94678B823048F090919F04943328F4B1
:107AB0009091A104923308F0B9C080919F048F3255
:107AC00008F05EC08091A104883208F459C00F9478
:107AD000D2502B013C018CE3C82ED12CE12CF12C8F
:107AE000C301B201A70196010F946259CA01B901FD
:107AF000A70196010F946259CA01062FD72E59018A
:107B0000AE014F5F5F4F7A0150E8451651E55506CB
:107B100051E06506710408F4A4C0B90128E130E021
:107B200040E050E00F94625929013A01DF920F932F
:107B3000C50168E170E00F943B599F938F935F926A
:107B40004F9286EC95E19F938F93FF92EF920F9463
:107B5000BA5E0FB6F894DEBF0FBECDBF5AE0451631
:107B600051046104710408F0A6C098E0892F880FC1
:107B7000980F892F81956FE2855A18DCC7018DDC3B
:107B800080919F048632A8F48091A1048E3188F000
:107B900008E020E84EE160E08BE694E00E94713559
:107BA00080919F04863228F48091A1048F3108F0DF
:107BB00084C080919F04823328F48091A1048B3289
:107BC00008F02BC180919F04813408F042C180915C
:107BD000A104873308F43DC16EE380E0E7DB812F29
:107BE00062DC37C188E496E191CD82E196E1A7CDD0
:107BF000EC52FA4EFFCD68E0EDCD02E028CE03E076
:107C000026CE02E058CE03E056CE02E0A9CE03E035
:107C1000A7CE02E0DACE03E0D8CE04E02AE441E3C6
:107C200066E38BE694E00E9421353ACFF8E48F9F1B
:107C3000B0011124072E000C880B990B0F94BA5633
:107C40002AE037ED43E25CE30F9456580F948C56CC
:107C5000262F02E042E367E38BE694E00E94713551
:107C60002CCF84E6A816B10498F4DF920F933F93CB
:107C70002F938CEB95E19F938F93FF92EF920F944C
:107C8000BA5E0FB6F894DEBF0FBECDBF95E06ECFE3
:107C9000DF920F933F932F9384EB95E19F938F9304
:107CA000FF92EF920F94BA5E0FB6F894DEBF0FBE4C
:107CB000CDBF96E05BCF99E059CF60E08BE694E0D2
:107CC0000E94CF3265E283E071DB68E570E080E01E
:107CD00090E0E6DB65E28BE069DB112321F084E5CF
:107CE00094E0DBDB24C08091760E80FD17C034E584
:107CF000E32E34E0F32EF70161917F016623B9F0A2
:107D00006F3234F4062E000C770B880B990B04C0ED
:107D10006FE370E080E090E0C3DBEDCF8091750E03
:107D200080FDDDCF6FEF7FEF87EA95E199DB65E2BC
:107D300088E23CDB69E570E080E090E0B1DB65E281
:107D400080E334DB112321F08FE494E0A6DB26C02E
:107D50008091760E869580FD17C02FE4E22E24E0F8
:107D6000F22EF70161917F016623C1F06F3234F486
:107D7000062E000C770B880B990B04C06FE370E0A4
:107D800080E090E08DDBEDCF8091750E869580FDD3
:107D9000DBCF6FEF7FEF87EA95E162DB65E28DE491
:107DA00005DB6AE570E080E090E07ADB65E285E57E
:107DB000FDDA112321F087E494E06FDB28C0809185
:107DC000760E8695869580FD17C097E4E92E94E09F
:107DD000F92EF70161917F016623C9F06F3234F407
:107DE000062E000C770B880B990B04C06FE370E034
:107DF00080E090E055DBEDCF8091750E86958695FD
:107E000080FDD9CF6FEF7FEF8CEA95E129DB61E050
:107E10008BE694E00E94CF32CCCE83E0FCD262E3CA
:107E200083E0C4DA66E070E080E090E039DB81E076
:107E3000F2D262E38CE0BADA80916D0290916E0228
:107E40000F94D6492ADB65E270E080E090E028DB01
:107E5000B9CE62960FB6F894DEBF0FBECDBFDF91EC
:107E6000CF911F910F91FF90EF90DF90CF90BF9037
:107E7000AF909F908F907F906F905F904F903F90CA
:107E80002F9008950F931F93CF93DF93CDB7DEB755
:107E900028970FB6F894DEBF0FBECDBF8A0123E04E
:107EA000660F771F2A95E1F7680F791F48E050E0C9
:107EB000CE0101960F94EE5D29813A81F80180810F
:107EC00091812817390790F08217930760F09C8101
:107ED0008281981758F081E090E03B81238123173D
:107EE00038F080E005C081E090E002C08FEF9FEFA6
:107EF00028960FB6F894DEBF0FBECDBFDF91CF91AD
:107F00001F910F910895EF92FF920F931F93CF93BC
:107F1000DF93EC018B017A018A859B858617970791
:107F200029F0888199816DD81B870A878885998572
:107F3000019681F00E811F81B701888199815ED8F9
:107F4000080F111D888599858017910718F481E025
:107F500090E011C06E818A81680F97014C81888101
:107F600099810E9412372E813F81280F311D3F8356
:107F70002E8380E090E0DF91CF911F910F91FF90D1
:107F8000EF9008954F925F926F927F928F929F929F
:107F9000AF92BF92CF92DF92EF92FF920F931F9317
:107FA000CF93DF93CDB7DEB72D970FB6F894DEBF32
:107FB0000FBECDBF6C012A013B01490158011B8650
:107FC0001C86CE0101967C0188E0F70111928A950A
:107FD000E9F7DB01CA0127E0B695A7959795879544
:107FE0002A95D1F79A838983F42FFF77FD878F2F06
:107FF00080588B838C831A8619864F3F5105610503
:10800000710509F018F460E070E026C060915C042E
:1080100070915D048E01075F1F4F970142E45FE39B
:1080200080915A0490915B040E945E8297FDEBCF91
:1080300069857A8583E0660F771F8A95E1F78091DD
:108040005A0490915B04680F791F48E050E0C70123
:108050000F94EE5D6F8178856115710519F44B867B
:10806000B60106C0C616D70619F08D8580688B87C5
:10807000AE01455F5F4FC401F50119952D960FB60E
:10808000F894DEBF0FBECDBFDF91CF911F910F914E
:10809000FF90EF90DF90CF90BF90AF909F908F9028
:1080A0007F906F905F904F9008956F927F928F9224
:1080B0009F92AF92BF92CF92DF92EF92FF920F9377
:1080C0001F93CF93DF9300D01F92CDB7DEB76C0123
:1080D0007B013A015901480119821A821B821C82D4
:1080E000AE014F5F5F4FB301C7010E94BE827C01AA
:1080F00049815A816B817C8141155105610571056A
:1081000029F084019501C6013DDFE6CF0F900F9065
:108110000F900F90DF91CF911F910F91FF90EF90F3
:10812000DF90CF90BF90AF909F908F907F906F9097
:10813000089521E020935E04EAE5F4E091838083D2
:108140007383628380E090E008957F92AF92BF9244
:10815000CF92DF92EF92FF920F931F93CF93DF9313
:10816000CDB7DEB72C970FB6F894DEBF0FBECDBFEC
:108170006C01762EF72F842FE52FB901A801D601C7
:108180001496AD90BC90159790915E0491110AC021
:1081900022E137E1482F672DC6010E94493780E070
:1081A00090E019C0DA82C9827B82FC838D83EE83E2
:1081B00018861F82FA86E9861C861B8603E81FE361
:1081C0009E012F5F3F4FC501DDDEB501C6010E9454
:1081D00001388F8198852C960FB6F894DEBF0FBEBC
:1081E000CDBFDF91CF911F910F91FF90EF90DF9066
:1081F000CF90BF90AF907F900895CF92DF92EF9293
:10820000FF920F931F93CF93DF93CDB7DEB72C97D9
:108210000FB6F894DEBF0FBECDBF7C01C901F701D8
:10822000C480D58020915E04211108C022EF36E180
:10823000C7010E94493780E090E01CC0FA82E982C1
:108240006B837C834D835E8318861F821A87098720
:108250001C861B8603E81FE39E012F5F3F4F48E506
:1082600052E8BC01C60121DFB601C7010E940138F6
:108270008F8198852C960FB6F894DEBF0FBECDBFC8
:10828000DF91CF911F910F91FF90EF90DF90CF90F2
:108290000895CF92DF92EF92FF920F931F93CF93A7
:1082A000DF93CDB7DEB72C970FB6F894DEBF0FBEC5
:1082B000CDBF7C01C901F701C480D58020915E0447
:1082C000211108C022ED36E1C7010E94493780E044
:1082D00090E01CC0FA82E9826B837C834D835E83CD
:1082E00018861F821A8709871C861B8603E81FE3EE
:1082F0009E012F5F3F4F4BE552E8BC01C601D5DE22
:10830000B601C7010E9401388F8198852C960FB65F
:10831000F894DEBF0FBECDBFDF91CF911F910F91BB
:10832000FF90EF90DF90CF900895CF93DF93EC0113
:10833000262F4CAD6BAD04960E94F4362BAD082E63
:10834000000C990B820F911D8BAF81E090E0DF91C3
:10835000CF9108950F939CE0899F802D112421E0F7
:10836000280F20936604845F8093650490E0029652
:1083700040919F0450E08417950714F480E034C0C6
:10838000822F90E02091A10430E082179307B4F788
:108390006623A9F061E08BE694E00E94CF32409121
:1083A00066044E5F0BE020E860E08BE694E00E94FC
:1083B000713560E08BE694E00E94CF3205C061E049
:1083C0008BE694E00E94CF326091650480919F0417
:1083D0006817A0F2909166048091A104891770F249
:1083E00080E00E94D63981E00F910895CF93DF930A
:1083F000FC0185ADEF012496811105C081E085AFB8
:10840000CE010E946F32CE01DF91CF910C94A63243
:108410006FEF7FEF25C8482F50E020916404022EB3
:10842000000C330B4217530781F0809364048130B2
:1084300031F46DEE7FE18BE694E00C9401386DEF42
:1084400077E18BE694E00C9401380895EF92FF9267
:108450000F938FEAE82E8DE1F82E00E428E040E04B
:1084600060E08BE694E00E94F9326FE373E08BE604
:1084700094E00E9401382DE333E041E169E38BE6AB
:1084800094E00E9412376FEA7BE08BE694E00E9452
:10849000013823E433E04CE16AE38BE694E00E9488
:1084A00012376AE07FE08BE694E00E94013823E512
:1084B00033E049E26BE38BE694E00E9412376AE016
:1084C0007FE08BE694E00E9401382FE533E04EE335
:1084D0006DE38BE694E00E94123721E633E04EE331
:1084E00062E48BE694E00E9412376DEF77E18BE651
:1084F00094E00F91FF90EF900C94013887E694E0A0
:1085000075DF61E080E0A2DF8BE694E00E94AA3292
:108510008111F7CF64EC79E080E090E00C9493A3B4
:10852000EF92FF920F938AE2E82E8DE1F82E03E19D
:1085300027E047E064E28BE694E00E94F93283E0B2
:108540006ADF21E633E04BE265E28BE694E00E94CD
:1085500012372BE633E047E367E08BE694E00F91B8
:10856000FF90EF900C94123787E694E03FDFD8DF5E
:108570008BE694E00E94AA328111F9CF64EC79E095
:1085800080E090E00C9493A3B9DFEECF60E070E060
:108590008DEE9FE1CECD1F93CF93DF93C0916C04FE
:1085A000C695C69587E694E021DFDC2FDD0F1D2FF1
:1085B0001C0F83E030DF6C2F80E00E94D6398CEFF7
:1085C00096E00E944D3A6D2F80E00E94D6398FE3ED
:1085D00097E11EDF612F80E00E94D63982E397E1A8
:1085E00017DF8BE694E00E94AA328111E2CFDF917F
:1085F000CF911F91089508950F931F93CF93E62F66
:108600006CE0869F602D112481E0860F80936604C4
:10861000645F60936504462F50E04E5F5F4F20918A
:108620009F0430E0421753070CF45AC090E02091A9
:10863000A10430E0821793070CF052C0CE2F8EE3D6
:108640000E94D63965E470E080E090E00E94503AE4
:1086500061E36C0F062E000C770B880B990B0E94C0
:10866000503A60E270E080E090E00E94503A0C2FB7
:1086700010E087E1C89FF0011124EC57F24F6481AC
:108680007581868197810F948756CB010F94D649C7
:108690000E944D3A6FE270E080E090E00E94503A14
:1086A0000E944C8681110BC085E0809FF001819F64
:1086B000F00D1124E659F24F8481811111C087E138
:1086C000809FF001819FF00D1124EC57F24F8085BF
:1086D00091850F94D649CF911F910F910C944D3AEB
:1086E000CF911F910F910895CF92DF92EF92FF9259
:1086F0000F931F93CF93DF931F921F92CDB7DEB7D7
:108700007B01622F498326DE4981882309F444C016
:10871000442311F101151105F9F4C7010E942E84BB
:1087200025E130E0281B310937FF02C02F5F3F4FA2
:108730003595279530E82158822F830F87FD0DC08E
:1087400060E270E080E090E02A8339830E94503A32
:10875000398131502A81F0CF30E8C32ED12CB601B7
:10876000C7010E94303A7601E81AF90A011511058D
:1087700011F41E2D07C0FF24B701C8010E94133A4F
:108780001E2D181B173040F060E270E080E090E092
:108790000E94503A181BF6CF0F900F90DF91CF91A7
:1087A0001F910F91FF90EF90DF90CF9008950F935E
:1087B000CF93DF93982F862FEA01692FCBDD882393
:1087C00031F162E770E0CE010E94303AC2E7C81B87
:1087D000C73040F060E270E080E090E00E94503AE4
:1087E000C81BF6CF609165048AE70E94D639602FD6
:1087F000000F770B880B990B0E94503A60E270E0F3
:1088000080E090E0DF91CF910F910C94503ADF918E
:10881000CF910F910895CF92DF92EF92FF920F9335
:108820001F93CF93DF93982F862F6A017901692FC9
:1088300091DD882309F447C0C701002321F00E947D
:108840002E84182F03C00E940D84182FC3E1D0E09E
:10885000C11BD1098C2F880FC80FCC0FD0E0BE01EF
:10886000C6010E94303AC81B6AE370E080E090E0E5
:108870000E94503AC73040F060E270E080E090E043
:108880000E94503AC81BF6CF8AEF189F802D112402
:108890006091650480580E94D639C701002349F0D1
:1088A000DF91CF911F910F91FF90EF90DF90CF90CC
:1088B000AFCDDF91CF911F910F91FF90EF90DF909F
:1088C000CF900C944D3ADF91CF911F910F91FF9073
:1088D000EF90DF90CF900895BF92CF92DF92EF920A
:1088E000FF920F931F93CF93DF936C017B010E9444
:1088F0002E84C82FC7010E940D8403E110E0081BDD
:1089000011098C2F90E0BB24B394081719071CF0B1
:10891000B12CC5E201C0CFE12C2F30E0A9014E5FA0
:108920005F4F80919F0490E04817590744F0295009
:1089300031098091A10490E082179307BCF5D0E043
:10894000E114F104D9F16AE370E080E090E00E9464
:10895000503ABB2081F0C45F80919F04C81770F12A
:108960002C2F30E0295031098091A10490E082172A
:1089700093071CF423C0DD2309F1802F880F800F9B
:108980006C2F880F0E94D63960E270E080E090E0A2
:108990000E94503AC701DF91CF911F910F91FF9034
:1089A000EF90DF90CF90BF900C944D3A6C2F80E009
:1089B0000E94D639C6012CDDD1E0C2CFDF91CF9124
:1089C0001F910F91FF90EF90DF90CF90BF9008958F
:1089D000CF92DF92EF92FF920F931F93CF93DF938B
:1089E0001F92CDB7DEB7182F7A01D22ECA01698344
:1089F0000E942E84082F812F880F810FC82ECC0C47
:108A00001CE06981169F100D1124DD20C1F061E08A
:108A10008BE694E00E94CF32202F220F200F220FEE
:108A20002E5F0BE047EF410F6FEF6C0D8BE694E08C
:108A30000E94713560E08BE694E00E94CF32612F96
:108A40008C2D0E94D639C701E3DCDD2071F061E096
:108A50008BE694E00F90DF91CF911F910F91FF90E3
:108A6000EF90DF90CF900C94CF320F90DF91CF91A9
:108A70001F910F91FF90EF90DF90CF900895AF92EC
:108A8000BF92DF92EF92FF920F931F93CF93DF93EA
:108A9000EC015B01D42EC901B801A7010E94DD855C
:108AA00091E02D2D2927A50164E081E091DFCE0121
:108AB0000E942E842D2DAE0164E094E1981B892F35
:108AC000DF91CF911F910F91FF90EF90DF90BF90BA
:108AD000AF907ECFEF92FF920F93CF93DF93D82F7B
:108AE000C62F7901682F8C2F35DC8823F1F0002305
:108AF00031F062E070E080E090E00E94503A2D2F6B
:108B00004C2F64E1C7010E94B98468E770E00E94BD
:108B1000133AC8E7C81BC73040F060E270E080E05D
:108B200090E00E94503AC81BF6CFDF91CF910F9191
:108B3000FF90EF9008958F929F92AF92BF92CF9245
:108B4000DF92EF92FF920F936B017C0180906004A3
:108B500090906104A0906204B0906304A501940118
:108B60000F941856882301F120E030E0A901C701D5
:108B7000B6010F941856882351F0A5019401C7013E
:108B8000B6010F94185687FD04C081E003C080E051
:108B900001C08FEF80935F04C0926004D0926104A3
:108BA000E0926204F092630480919F04813128F482
:108BB0008091A104833008F048C080919F048531E2
:108BC00028F48091A104843108F04FC080919F0463
:108BD0008F3308F057C08091A1048F3208F452C03F
:108BE00080915F0440E3481B83E8E82E87E1F82E7C
:108BF0000DE022E06AE58BE694E00E94F932809174
:108C00005F0441E3481B99E6E92E97E1F92E22E043
:108C100065E08BE694E00E94F9322DE9E22E27E12F
:108C2000F22E00E123E04FE262E18BE694E00E9445
:108C3000F9323DECE32E37E1F32E23E04FE267E615
:108C40008BE694E00E94F9321DC080915F0444E0FD
:108C5000481B5EE4E52E57E1F52E0CE022E062E4CD
:108C60008BE694E00E94F932A8CF46E6E42E47E175
:108C7000F42E01E023E044E16CE38BE694E00E94F3
:108C8000F932A4CF0F91FF90EF90DF90CF90BF907B
:108C9000AF909F908F900895CF92EF920F93CF93C4
:108CA000DF93C7E6D4E01B821A8283E893E09983BE
:108CB0008883CC24CA94EE24EA9406E427E448E4AA
:108CC00064E172E0CE010E94B0398FE893E09983AD
:108CD0008883DF91CF910F91EF90CF90089590917D
:108CE000050194709093030187FD76C0A39890913D
:108CF00005019095947090930301909105019470F3
:108D000090930301982F990F86FD72C0A3988091CC
:108D10000501809584708093030180910501847022
:108D200080930301292F220F96FD60C0A3988091A4
:108D30000501809584708093030180910501847002
:108D400080930301922F990F26FD4EC0A398809126
:108D500005018095847080930301809105018470E2
:108D600080930301292F220F96FD3CC0A398809188
:108D700005018095847080930301809105018470C2
:108D800080930301922F990F26FD2AC0A39880910A
:108D900005018095847080930301809105018470A2
:108DA00080930301292F220F96FD18C0A39880916C
:108DB0000501809584708093030180910501847082
:108DC0008093030126FD16C0A3988091050180952C
:108DD0008470809303010895A39A89CFA39AE7CF63
:108DE000A39AD5CFA39AC3CFA39AB1CFA39A9FCF6B
:108DF000A39A8DCFA39A809105018095847080936A
:108E0000030108952F923F925F927F929F92AF92BB
:108E1000BF92CF92DF92EF92FF920F931F93CF9367
:108E2000DF937C011B01942E69018AE0481709F445
:108E30007BC0A5E14A134EC0DB011296ED91FC9177
:108E400013971281C681D781A49A88E28A9500007F
:108E5000E9F700EE010F80E1582E510E98E2792ECD
:108E600088EF3DDF872D8A950000E9F7103208F082
:108E700046C0812F8077806832DF812F8295807F86
:108E80002EDF872D8A950000E9F780E828DF80E053
:108E900026DF872D8A950000E9F78AEF20DF872DEE
:108EA0008A950000E9F75E01B0E1AB0EB11C888144
:108EB000807F15DF89918295807F11DFCA15DB05E0
:108EC000B1F7872D8A950000E9F71F5F0F5F151135
:108ED000C7CFA4989601492DB101C701DF91CF9169
:108EE0001F910F91FF90EF90DF90CF90BF90AF90C8
:108EF0009F907F905F903F902F900C943334802F01
:108F000080778068ECDE802F8295807FE8DE872D79
:108F10008A950000E9F780E8E2DE80E8E0DE872D50
:108F20008A950000E9F7B9CF9C9AA4989B9AA398D8
:108F300080910401846080930401809105018095F3
:108F4000847080930301A49AC8E28C2F8A95000054
:108F5000E9F788E790E00E94503388EFC0DE8C2F5D
:108F60008A950000E9F780E2BADE80E0B8DE8C2F57
:108F70008A950000E9F780E0B2DE80E8B0DE8C2F51
:108F80008A950000E9F780E0AADE80E1A8DE8C2F58
:108F90008A950000E9F78FE090E00E94503380E26C
:108FA0009EDE80E49CDE8C2F8A950000E9F780E24B
:108FB00096DE80E694DECA950000E9F710E0D8E27C
:108FC00008E2812F807780688ADE812F8295807FFA
:108FD00086DE8D2F8A950000E9F780E880DE80E04C
:108FE0007EDE8D2F8A950000E9F78AEF78DE8D2FDF
:108FF0008A950000E9F7C0E280E071DE80E06FDE74
:109000009D2F9A950000E9F7C150B1F788EF67DE10
:10901000802F8A950000E9F71F5F103209F0D1CF49
:1090200080E05DDE80EC5BDE88E28A950000E9F797
:10903000A49850CFCF93DF931F921F92CDB7DEB786
:1090400089839A830E94F87E20E040E060E070E02F
:1090500089819A810F900F90DF91CF910C949D7F21
:109060000F93CF93DF9361E081E00E94A680D091BF
:10907000C906C0E0D11117C08091C806811104C093
:109080000E940385811165C080912202882309F422
:1090900057C081E09091C806911180E004E024E07F
:1090A00041E059E24BC0D130C1F48091C806813013
:1090B00021F40E940385811154C0809122028823EB
:1090C00009F43EC081E09091C806913009F080E03B
:1090D00003E02EE348EF58E231C0D230B9F480917A
:1090E000C806823021F40E940385811143C080911B
:1090F0002202882329F181E09091C806923009F07C
:1091000080E003E02EE34FEE58E218C0D330C1F404
:109110008091C806833021F40E940385811133C0F9
:1091200080912202882361F081E09091C8069330FB
:1091300009F080E003E02EE349EE58E26C2F37DBC4
:10914000CF5FDF5FC53009F095CF84E08093C7061D
:1091500021C00E94D07F80919506882309F494CF86
:1091600019C089E892E766DF80919506882309F4A3
:10917000A4CF10C088E997E75DDF8091950688232A
:1091800009F4B5CF07C08AE59BE754DF80919506C7
:10919000882331F2DF91CF910F910895CF92DF9222
:1091A000EF92FF920F931F9380918709811103C063
:1091B00089EC99E002C087E899E025E4C22E29E213
:1091C000D22E7C0108E319E220ED3FE745EF58E499
:1091D00061E379E28BE299E20E94FE811F910F9197
:1091E000FF90EF90DF90CF90089589EC99E00E9476
:1091F000D58F0E94C97F0C940C8B0E94719421E042
:1092000030E0811102C020E030E03093F10620937D
:10921000F0061092C90681E08093950683E0809362
:1092200022020895CF92DF92EF92FF920F931F9345
:10923000CF93DF930E9475956C0161E081E00E94FD
:10924000A680C091C906D0E081E0C81AD108C1113A
:1092500017C08091C806811104C00E940385811146
:1092600095C080912202882359F081E09091C80630
:10927000911180E004E024E046E259E26D2F97DA94
:1092800069EC79E080E599E00E946E9B8091C909C4
:109290008F3201F18091D60983FF1CC0C130C1F427
:1092A0008091C806813021F40E940385811176C027
:1092B00080912202882361F081E09091C80691306C
:1092C00009F080E000E22EE342E259E26D2F6FDA0E
:1092D00092E001C091E080912202882309F44EC0FF
:1092E000760111E01C0F8FEFE816F80609F446C06E
:1092F000C9133FC060E070E0C7010E944A9190919D
:10930000D6098091C80694FF1CC08C134EC00E94E1
:109310000385882309F449C089EC99E00E941B94D5
:109320001092C90682E090E09093F1068093F006D7
:1093300081E0809395061092F30683E080932202E9
:1093400052C08C1304C00E94038581113DC08091DE
:109350002202882361F081E09091C8069C1380E08E
:1093600000E028E038E146E059E26D2FB3DB912FB1
:1093700001C09F5F81E0E81AF108B5CFDF5FCF5FE2
:10938000D53009F064CF9093C7062DC00E94D07FDE
:1093900080919506882309F464CF25C02EDF809143
:1093A0009506882309F484CF1EC080912202882369
:1093B000F1F281E09091C8069C1380E001E028E082
:1093C00038E144E159E2D1CF0E94F87E20E040E04C
:1093D00060E070E08EEC98E40E949D7F809195069D
:1093E000882309F4B4CFDF91CF911F910F91FF90A3
:1093F000EF90DF90CF900895CF93DF93EC01CB01F6
:10940000BA010F94BA560F948C566883DF91CF91AE
:109410000895CF93DF93EC01CB01BA010F94BA56B4
:109420002FE632E143E85AE30F9456586883798374
:109430008A839B83DF91CF9108956CEF79E489E271
:109440009AE40C94E57F69E07AE486E49AE40C946B
:10945000E57F0F94BA560F948C56862F0D942B49A6
:10946000CF93DF9300D01F92CDB7DEB769837A83A5
:109470008B839C8360E2CE0101960F944F4C0F903A
:109480000F900F900F90DF91CF9108950F94BA56DF
:109490002FE632E143E85AE30F945658E1CF2F927A
:1094A0003F924F925F926F927F928F929F92AF9274
:1094B000BF92CF92DF92EF92FF920F931F93CF93C1
:1094C000DF93CDB7DEB729970FB6F894DEBF0FBE96
:1094D000CDBF1C0179876887CA01B901E982FA8288
:1094E0000B831C83DE82CD82AF8220E030E04AE72E
:1094F00054E40F9456586B017C0120E030E040E0CA
:1095000057EC0F941B5818162CF0C12CD12CE12CC1
:1095100027ECF22EC701B6010F9487562B013C01B0
:1095200020E030E04AE754E469817A818B819C81B4
:109530000F9456584B015C0120E03EEF4FEF56E48C
:109540000F94185687FD07C0812C9EEF992EAA24F0
:10955000AA9496E4B92E20E030E04AE754E4E88586
:10956000F98560817181828193810F9456586B01D6
:109570007C01C301B2010F94BA569B01AC01C70133
:10958000B6010F943E550F948C5669837A838B8372
:109590009C83C501B4010F9487567B018C01E418AC
:1095A000F50806091709FF81FF938D809E8083E2ED
:1095B000A82E8AE4B82EC980DA80A30192016885BA
:1095C0007985C1010E941F7F0F9029960FB6F894EC
:1095D000DEBF0FBECDBFDF91CF911F910F91FF90E6
:1095E000EF90DF90CF90BF90AF909F908F907F9043
:1095F0006F905F904F903F902F9008958F929F9221
:10960000AF92BF92CF92DF92EF92FF920F931F9390
:10961000CF93DF9361E081E00E94A680D091C906DC
:10962000C0E0D11119C08091C806811104C00E9408
:1096300003858111C4C080912202882309F4B6C039
:1096400081E09091C806911180E004E024E04DE7AC
:1096500059E26C2FACD8AAC0D130E1F48091C80691
:10966000813021F40E9403858111B1C080912202D2
:10967000882309F49BC011E08091C806813009F06D
:1096800010E08091D30C0F942B4900E09C0147E639
:1096900059E289C0D23009F58091C806823021F4A0
:1096A0000E9403858111B4C080912202882309F4AD
:1096B0007DC011E08091C806823009F010E0609111
:1096C000D40C7091D50C8091D60C9091D70CC8DE3B
:1096D00000E09C0143E659E266C0D33009F5809171
:1096E000C806833021F40E9403858111AAC08091AD
:1096F0002202882309F45AC011E08091C806833001
:1097000009F010E06091D80C7091D90C8091DA0CBE
:109710009091DB0CA5DE00E09C014FE559E243C0CF
:10972000D43001F58091C806843021F40E9403856D
:109730008111A0C0809122028823C1F111E08091A3
:10974000C806843009F010E06091DC0C7091DD0CEB
:109750008091DE0C9091DF0C83DE00E09C014BE5F4
:1097600059E221C0D53011F58091C806853021F429
:109770000E940385811197C0809122028823B1F055
:1097800011E08091C806853009F010E06091260252
:1097900070912702809128029091290261DE00E0F9
:1097A0009C0147E459E26C2F812F35D8CF5FDF5FF2
:1097B000C53009F036CF86E08093C7068CC00E9482
:1097C000D07F80919506882309F435CF84C081E04D
:1097D0000E94F884C090D30CD12C1F92812C912C24
:1097E0004DE1A42E4AE4B42EE12CF12C8701EA9439
:1097F00020E030E0A90163ED7CE082E799E20E947D
:109800001F7F0F9080919506882309F42FCF63C0A6
:1098100081E00E94F884A12CC12CD12C16E6E12E07
:10982000FE2C0EE111E420E030E0A90164ED7CE0C3
:1098300085E699E234DE80919506882309F434CFD9
:109840004AC081E00E94F884A12CC12CD12C16E6DC
:10985000E12EFE2C0EE111E420E030E0A90168EDDC
:109860007CE081E699E21BDE80919506882309F46D
:109870003ECF31C081E00E94F884A12CC12CD12CB4
:1098800016E6E12EFE2C0EE111E420E030E0A90105
:109890006CED7CE08DE599E202DE809195068823EF
:1098A00009F448CF18C081E00E94F884A12CC12C93
:1098B000D12C16E6E12EFE2C0EE111E420E030E082
:1098C000A90166E272E081E599E2E9DD8091950601
:1098D000882309F451CFDF91CF911F910F91FF9011
:1098E000EF90DF90CF90BF90AF909F908F900895B2
:1098F000CF93DF93EC01CB01BA010F94BA562AE063
:1099000037ED43E25CE30F945658688379838A838A
:109910009B83DF91CF910895CF93DF93EC01CB012F
:10992000BA010F94BA56688379838A839B83DF9147
:10993000CF910895CF93DF93EC01CB01BA010F943F
:10994000BA5620E030E048EC51E40F945658688352
:1099500079838A839B83DF91CF910895CF93DF939F
:10996000EC01CB01BA010F94BA5620E030E048EC8C
:1099700052E40F945658688379838A839B83DF91DE
:10998000CF910895CF93DF93EC01CB01BA010F94EF
:10999000BA5620E030E048EC51E40F9456580F944A
:1099A0008C56688379838A839B83DF91CF91089556
:1099B000CF93DF93EC01CB01BA010F94BA5620E0AC
:1099C00030E048EC52E40F9456580F948C5668835C
:1099D00079838A839B83DF91CF910895CF93DF931F
:1099E000EC01CB01BA010F94BA562AE037ED43E2FD
:1099F0005CE30F945658688379838A839B83DF9155
:109A0000CF910895CF93DF93EC01CB01BA010F946E
:109A1000BA562DEC3CEC4CEC5DE30F945658688341
:109A200079838A839B83DF91CF91089568E77CE4F3
:109A300087E69DE40C94E57F6CE87CE48EEF9DE482
:109A40000C94E57F6EEA7CE481EA9DE40C94E57F6A
:109A50006AE97CE484E89DE40C94E57F62EC7CE4B4
:109A60008EEB91E50C94E57F68ED7CE48AE19EE461
:109A70000C94E57F6EEE7CE48EEB9DE40C94E57F28
:109A800062E07DE48AE49DE40C94E57F0D946C0A29
:109A90000D94C30ACF93DF9300D01F92CDB7DEB7EA
:109AA0000F94BA562DEC3CEC4CEC5DE30F945658F9
:109AB00069837A838B839C83CE0101960F946D4ECC
:109AC0000F900F900F900F90DF91CF910895CF934B
:109AD000DF9300D01F92CDB7DEB70F94BA562AE0BD
:109AE00037ED43E25CE30F94565869837A838B83A6
:109AF0009C83CE0101960F94114B0F900F900F9005
:109B00000F90DF91CF910895CF93DF9300D01F92F4
:109B1000CDB7DEB70F94BA5620E030E048EC51E400
:109B20000F94565869837A838B839C83CE01019668
:109B30000F94984D0F900F900F900F90DF91CF9151
:109B40000895CF93DF9300D01F92CDB7DEB70F9467
:109B5000BA5620E030E048EC52E40F94565869833E
:109B60007A838B839C83CE0101960F94984D0F903E
:109B70000F900F900F90DF91CF910895CF93DF93C7
:109B800000D01F92CDB7DEB70F94BA562AE037ED5A
:109B900043E25CE30F94565869837A838B839C83FA
:109BA000CE0101960F94CD4D0F900F900F900F9016
:109BB000DF91CF910895CF92DF92EF92FF926B01E8
:109BC0007C0120E030E0A9010F94185687FD05C004
:109BD00020E030E040E05FE304C020E030E040E01F
:109BE0005FEBC701B6010F943F550F948756CB0129
:109BF000FF90EF90DF90CF900D94D6490F94BA5616
:109C0000DACFCF93DF9300D01F92CDB7DEB70F949A
:109C10008C560F94B85669837A838B839C83CE01CC
:109C200001960F94984D0F900F900F900F90DF9129
:109C3000CF9108950F94BA5620E030E048EC52E4FA
:109C40000F945658DECFCF93DF9300D01F92CDB73D
:109C5000DEB70F948C560F94B85669837A838B8342
:109C60009C83CE0101960F94984D0F900F900F900A
:109C70000F90DF91CF9108956F927F928F929F9274
:109C8000AF92BF92CF92DF92EF92FF920F931F930A
:109C9000CF93DF9300D01F92CDB7DEB761E081E0B4
:109CA0000E94A6806090C906712C61101AC0809134
:109CB000C806811104C00E940385811178C180917A
:109CC0002202882309F46AC181E09091C8069111AB
:109CD00080E004E024E046E25BE2672D0E94D74387
:109CE0005DC181E068122CC08091C806813021F4EA
:109CF0000E940385811163C180912202882309F4A7
:109D00004DC111E08091C806813009F010E08091CA
:109D1000730F9091740FA091750FB091760F898396
:109D20009A83AB83BC83CE0101960F94984D00E0DB
:109D30009C014AE15BE2672D812F0E940B442EC1FA
:109D400082E068122CC08091C806823021F40E9403
:109D5000038581116CC180912202882309F41EC100
:109D600011E08091C806823009F010E08091770FF1
:109D70009091780FA091790FB0917A0F89839A838F
:109D8000AB83BC83CE0101960F94984D00E09C01FB
:109D900046E05BE2672D812F0E940B44FFC083E009
:109DA00068122CC08091C806833021F40E9403857C
:109DB000811175C180912202882309F4EFC011E05E
:109DC0008091C806833009F010E080917B0F90915C
:109DD0007C0FA0917D0FB0917E0F89839A83AB8316
:109DE000BC83CE0101960F94984D00E09C0144EF96
:109DF0005AE2672D812F0E940B44D0C084E0681284
:109E000027C08091C806843021F40E940385811107
:109E10007EC180912202882309F4C0C011E08091A4
:109E2000C806843009F010E06091330F7091340F50
:109E30008091350F9091360F0F94B85604DF00E0F3
:109E40009C0146EE5AE2672D812F0E940B44A6C06A
:109E500085E0681227C08091C806853021F40E94F1
:109E60000385811190C180912202882309F496C054
:109E700011E08091C806853009F010E06091370F3D
:109E80007091380F8091390F90913A0F0F94B85616
:109E9000DADE00E09C0148ED5AE2672D812F0E9436
:109EA0000B447CC086E0681227C08091C8068630CB
:109EB00021F40E9403858111A2C18091220288238E
:109EC00009F46CC011E08091C806863009F010E0FA
:109ED00060913B0F70913C0F80913D0F90913E0F30
:109EE0000F94B856B0DE00E09C014AEC5AE2672DB0
:109EF000812F0E940B4452C087E0681227C08091D6
:109F0000C806873021F40E9403858111ADC180917C
:109F10002202882309F442C011E08091C8068730EC
:109F200009F010E060913F0F7091400F8091410F58
:109F30009091420F0F94B85664DE00E09C014EEA07
:109F40005AE2672D812F0E940B4428C088E06812D6
:109F500025C08091C806883021F40E9403858111B4
:109F6000BFC1809122028823C9F011E08091C80608
:109F7000883009F010E06091430F7091440F809198
:109F8000450F9091460F0F94B8563BDE00E09C01C0
:109F900042E95AE2672D812F0E940B447394639427
:109FA00085E0781282CE89E08093C706D4C10E94F2
:109FB000D07F80919506882309F481CECCC181E0C1
:109FC0000E94F8842AE037ED43E25DE36091730F6D
:109FD0007091740F8091750F9091760F0F94565871
:109FE00020E030E040E85FE30F943E550F948C563C
:109FF0001F92812C912CA8E2AA2EADE4BA2E6B01FF
:10A0000017E7E12E1FE0F12E00E010E021E030E044
:10A0100040E050E063E77FE080E29BE20E941F7F28
:10A020000F9080919506882309F466CE94C181E053
:10A030000E94F8842AE037ED43E25CE36091770FF9
:10A040007091780F8091790F90917A0F0F945658F4
:10A0500020E030E040E85FE30F943E550F948C56CB
:10A060001F92812C912CE2E2AE2EEDE4BE2E6B010C
:10A070001DEDE12E13E0F12E00E010E021E030E0D4
:10A0800040E050E067E77FE080E19BE20E941F7FB5
:10A090000F9080919506882309F45DCE5CC181E024
:10A0A0000E94F8842AE037ED43E25DE360917B0F84
:10A0B00070917C0F80917D0F90917E0F0F94565878
:10A0C00020E030E040E85FE30F943E550F948C565B
:10A0D0001F92812C912C48E2A42E4DE4B42E6B01EA
:10A0E00017E7E12E1FE0F12E00E010E021E030E064
:10A0F00040E050E06BE77FE08DEF9AE20E941F7F27
:10A100000F9080919506882309F454CE24C181E0F4
:10A110000E94F8846091330F7091340F8091350F55
:10A120009091360F0F94B8562AE037ED43E25DE385
:10A130000F94565820E030E040E850E40F943E552C
:10A140000F948C561F9296E4892E9DE4992E2EE250
:10A15000A22E2DE4B22E6B0114E7E12E1FE0F12EAA
:10A1600000E010E024E030E040E050E063E37FE016
:10A170008DEE9AE20E941F7F0F90809195068823B2
:10A1800009F447CEE8C081E00E94F8846091370F5F
:10A190007091380F8091390F90913A0F0F94B85603
:10A1A0002AE037ED43E25DE30F94565820E030E0BB
:10A1B00040E850E40F943E550F948C561F92B6E43D
:10A1C0008B2EBDE49B2E1EE2A12E1DE4B12E6B0151
:10A1D00014E7E12E1FE0F12E00E010E024E030E073
:10A1E00040E050E067E37FE08FED9AE20E941F7F3E
:10A1F0000F9080919506882309F435CEACC081E09C
:10A200000E94F88460913B0F70913C0F80913D0F4C
:10A2100090913E0F0F94B8562AE037ED43E25DE38C
:10A220000F9456580F948C561F92E6E48E2EEDE450
:10A230009E2EFEE2AF2EFDE4BF2E6B0118E7E12E4D
:10A240001FE0F12E00E010E020E030E0A9016BE318
:10A250007FE081ED9AE20E941F7F0F90809195062A
:10A26000882309F42ACE77C081E00E94F8846091A7
:10A270003F0F7091400F8091410F9091420F0F94CA
:10A28000B8562AE037ED43E25CE30F94565820E0DD
:10A2900030E040E85FE30F943E550F948C561F92D8
:10A2A0003EEC832E31E5932E44E3A42E4DE4B42EF0
:10A2B0006B011DEDE12E13E0F12E00E010E021E036
:10A2C00030E040E050E06FE37FE08CEB9AE20E94E8
:10A2D0001F7F0F9080919506882309F418CE3BC00C
:10A2E00081E00E94F8846091430F7091440F809147
:10A2F000450F9091460F0F94B8562AE037ED43E290
:10A300005CE30F94565820E030E040E85FE30F94A0
:10A310003E550F948C561F9280ED882E81E5982E25
:10A3200094E3A92E9DE4B92E6B011DEDE12E13E0FF
:10A33000F12E00E010E021E030E040E050E063E486
:10A340007FE080EA9AE20E941F7F0F90809195063D
:10A35000882309F406CE0F900F900F900F90DF9195
:10A36000CF911F910F91FF90EF90DF90CF90BF9012
:10A37000AF909F908F907F906F9008950F94BA56F2
:10A3800020E030E048EC51E40F9456585CCC9091BA
:10A39000630E891302C00D946C0A089580E0F7CF14
:10A3A00081E0F5CFCF93DF939091630E891304C0C2
:10A3B000DF91CF910D94C30A8D5F90E0EC01CC0F3B
:10A3C000DD1FCC0FDD1FC55FD04F880F991F880F91
:10A3D000991FFC01E55BF04F20813181428153815F
:10A3E00060E070E080E89FE30F941F5668837983F4
:10A3F0008A839B83DF91CF91089580E0D3CF81E062
:10A40000D1CF0F931F93CF93DF9361E081E00E9440
:10A41000A680C091C906D0E0C1111AC08091C806BB
:10A42000811104C00E9403858111CCC08091220259
:10A43000882309F461C081E09091C806911180E001
:10A4400004E024E048EB59E26D2F0E94D74354C04A
:10A45000C130D9F48091C806813021F40E9403856F
:10A460008111B8C080912202882309F445C081E09F
:10A470009091C806913009F080E003E02EE34FEAA6
:10A4800059E26D2F0E94D74337C0C230D1F480917A
:10A49000C806823021F40E9403858111A5C08091F5
:10A4A0002202882349F181E09091C806923009F098
:10A4B00080E003E02EE342EA59E26D2F0E94D74389
:10A4C0001BC0C330C9F48091C806833021F40E94B8
:10A4D0000385811193C080912202882369F081E075
:10A4E0009091C806933009F080E003E02EE34DE937
:10A4F00059E26D2F0E94D7430E94867F81111DC0B3
:10A50000C430E9F48091C806843021F40E940385A8
:10A5100081117EC080912202882309F483C081E0EA
:10A520009091C806943009F080E003E02EE344E9FE
:10A5300059E26D2F0E94D74375C014E001C015E0A9
:10A54000C1131BC08091C8068C1304C00E940385F0
:10A5500081116AC080912202882371F081E090917C
:10A56000C8069C1380E003E02EE34BE859E26D2F10
:10A570000E94D7431C2F01C01C2F81E0810FC813FC
:10A5800018C08091C8068C1304C00E9403858111F5
:10A5900055C080912202882361F081E09091C80625
:10A5A0009C1380E003E02EE342E859E26D2F0E9405
:10A5B000D743DF5FCF5FD53009F02ECF1E5F1093FA
:10A5C000C70645C00E94D07F80919506882309F474
:10A5D0002DCF3DC08BE596E50E941A4880919506E7
:10A5E000882309F43FCF33C08CE39EE40E941A48CD
:10A5F00080919506882309F452CF29C08BE698E50F
:10A600000E941A4880919506882309F464CF1FC0E0
:10A610008FE99AE50E941A4880919506882309F4EB
:10A6200079CF15C015E0A9CF8EEF9AE40E941A48A1
:10A6300080919506882309F48DCF09C087EB93E5B7
:10A640000E941A4880919506882309F4A2CFDF91D1
:10A65000CF911F910F9108952F923F924F925F9249
:10A660006F927F928F929F92AF92BF92CF92DF9222
:10A67000EF92FF920F931F93CF93DF9300D000D000
:10A68000CDB7DEB71C017E836D8329013A014601F7
:10A6900020E030E040E057ECB201C3010F941B58BA
:10A6A00018162CF0412C512C612C27EC01C0272DC1
:10A6B000B201862D922F0F9487562B013C0120E08A
:10A6C0003EEF4FEF56E4B701C8010F94185687FDCF
:10A6D00006C0B12C9EEFF92E0FEF16E401C0BE2C80
:10A6E000C301B2010F94BA569B01AC01ED81FE810A
:10A6F00060817181828193810F943E550F948C56B5
:10A7000069837A838B839C836B2D7F2DC8010F9483
:10A7100087567B018C01E418F50806091709AF92EA
:10A720008CE1A82E8DE4B82EC980DA80A3019201B5
:10A730006D817E81C1010E941F7F0F9026960FB60A
:10A74000F894DEBF0FBECDBFDF91CF911F910F9167
:10A75000FF90EF90DF90CF90BF90AF909F908F9041
:10A760007F906F905F904F903F902F9008956F92E1
:10A770007F928F929F92AF92BF92CF92DF92EF9291
:10A78000FF920F931F93CF93DF9300D01F92CDB70B
:10A79000DEB761E081E00E94A6806090C906712C5E
:10A7A00061101AC08091C806811104C00E940385FF
:10A7B00081116FC180912202882309F461C181E077
:10A7C0009091C806911180E004E024E04EE85CE23C
:10A7D000672D0E94D74354C181E068122CC080913C
:10A7E000C806813021F40E94038581115AC18091ED
:10A7F0002202882309F444C111E08091C806813007
:10A8000009F010E08091970E9091980EA091990E0A
:10A81000B0919A0E89839A83AB83BC83CE01019653
:10A820000F94114B00E09C014AE65CE2672D812FFA
:10A830000E940B4425C182E068122CC08091C8069A
:10A84000823021F40E940385811159C18091220236
:10A85000882309F415C111E08091C806823009F0FF
:10A8600010E080919B0E90919C0EA0919D0EB09156
:10A870009E0E89839A83AB83BC83CE0101960F948D
:10A88000114B00E09C0146E45CE2672D812F0E94A1
:10A890000B44F6C083E0681229C08091C80683305B
:10A8A00021F40E940385811158C1809122028823DE
:10A8B00009F4E6C011E08091C806833009F010E089
:10A8C000E091630E88E0E89FF0011124EC55F34F0E
:10A8D00060817181828193816ED900E09C0142E3A5
:10A8E0005CE2672D812F0E940B44CAC084E068128D
:10A8F00025C08091C806843021F40E94038581110F
:10A900004AC180912202882309F4BAC011E08091E3
:10A91000C806843009F010E06091A40C7091A50C79
:10A920008091A60C9091A70C46D900E09C014AE1C9
:10A930005CE2672D812F0E940B44A2C085E0681263
:10A9400025C08091C806853021F40E9403858111BD
:10A950003AC180912202882309F492C011E08091CB
:10A96000C806853009F010E06091AC0C7091AD0C18
:10A970008091AE0C9091AF0C1ED900E09C0142E09A
:10A980005CE2672D812F0E940B447AC086E068123A
:10A9900029C08091C806863021F40E940385811168
:10A9A0002AC180912202882309F46AC011E08091B3
:10A9B000C806863009F010E0E091630E88E0E89F59
:10A9C000F0011124EC55F34F6481758186819781E4
:10A9D000F2D800E09C0142EF5BE2672D812F0E94DC
:10A9E0000B444EC087E0681225C08091C8068730AE
:10A9F00021F40E94038581111CC1809122028823C9
:10AA000009F43EC011E08091C806873009F010E0DB
:10AA10006091A80C7091A90C8091AA0C9091AB0C3C
:10AA2000CAD800E09C014EED5BE2672D812F0E94A9
:10AA30000B4426C088E0681223C08091C806883085
:10AA400021F40E94038581110CC180912202882388
:10AA5000B9F011E08091C806883009F010E06091EB
:10AA6000B00C7091B10C8091B20C9091B30CA3D842
:10AA700000E09C014AEC5BE2672D812F0E940B44B1
:10AA80007394639485E078128BCE89E08093C70637
:10AA9000FFC00E94D07F80919506882309F48ACE5A
:10AAA000F7C020E030E048EC52E46091970E7091DE
:10AAB000980E8091990E90919A0E0F9456580F947B
:10AAC0008C561F92812C912CA6E1AA2EADE4BA2EB1
:10AAD0006B01EE24EA941FE7F12E00E010E020E085
:10AAE00030E0A90167E97EE08CE79CE20E941F7FCD
:10AAF0000F9080919506882309F479CEC9C020E093
:10AB000030E048EC52E460919B0E70919C0E809175
:10AB10009D0E90919E0E0F9456580F948C561F9236
:10AB2000812C912CE6E1AE2EEDE4BE2E6B01EE24DD
:10AB3000EA941FE7F12E00E010E020E030E0A901E8
:10AB40006BE97EE088E59CE20E941F7F0F90809178
:10AB50009506882309F47ACE9BC081E00E94F88490
:10AB60006091630E88E0689FB00111246C55734FAB
:10AB7000A12CC12CD12CE12CF12C08E413E420E011
:10AB800030E0A9018CE39CE267DD80919506882383
:10AB900009F48BCE7DC081E00E94F884A12CC12CE9
:10ABA000D12CE12CF12C08E413E420E030E0A901E1
:10ABB00064EA7CE086E29CE24FDD80919506882382
:10ABC00009F49FCE65C081E00E94F884A12CC12CBD
:10ABD000D12CE12CF12C08E413E420E030E0A901B1
:10ABE0006CEA7CE08EE09CE237DD8091950688235C
:10ABF00009F4AFCE4DC081E00E94F8846091630EED
:10AC000088E0689FB00111246855734FA12CC12CB6
:10AC1000D12CE12CF12C08E413E420E030E0A90170
:10AC20008AEF9BE219DD80919506882309F4B9CE5D
:10AC30002FC081E00E94F884A12CC12CD12CE12CE2
:10AC4000F12C08E413E420E030E0A90168EA7CE09C
:10AC500088EE9BE201DD80919506882309F4CDCE34
:10AC600017C081E00E94F884A12CC12CD12CE12CCA
:10AC7000F12C08E413E420E030E0A90160EB7CE073
:10AC800084ED9BE2E9DC80919506882309F4DDCE12
:10AC90000F900F900F900F90DF91CF911F910F9118
:10ACA000FF90EF90DF90CF90BF90AF909F908F90EC
:10ACB0007F906F900895AF92CF92DF92EF92FF92C4
:10ACC0000F931F93CF93DF9361E081E00E94A680F2
:10ACD000D091C906C0E0D1111AC08091C806811177
:10ACE00004C00E940385811131C180912202882312
:10ACF00009F423C181E09091C806911180E004E03D
:10AD000024E048EB5BE26C2F0E94D74316C1D130A0
:10AD100031F58091C806813021F40E9403858111AC
:10AD20001DC180912202882309F407C111E080919E
:10AD3000C806813009F010E060915F0F7091600FDC
:10AD40008091610F9091620F0E94DB4D00E09C01A9
:10AD50004AEA5BE26C2F812F0E940B44EEC0D23096
:10AD600031F58091C806823021F40E94038581115B
:10AD70000FC180912202882309F4DFC011E0809185
:10AD8000C806823009F010E06091630F7091640F83
:10AD90008091650F9091660F0E94DB4D00E09C0151
:10ADA0004CE95BE26C2F812F0E940B44C6C0D3306C
:10ADB00031F58091C806833021F40E94038581110A
:10ADC00001C180912202882309F4B7C011E080916B
:10ADD000C806833009F010E06091670F7091680F2A
:10ADE0008091690F90916A0F0E94DB4D00E09C01F9
:10ADF0004EE85BE26C2F812F0E940B449EC0D43042
:10AE000031F58091C806843021F40E9403858111B8
:10AE1000F3C080912202882309F48FC011E0809151
:10AE2000C806843009F010E060916B0F70916C0FD0
:10AE300080916D0F90916E0F0E94DB4D00E09C01A0
:10AE400042E75BE26C2F812F0E940B4476C0D53025
:10AE500031F58091C806853021F40E940385811167
:10AE6000E5C080912202882309F467C011E0809137
:10AE7000C806853009F010E060916F0F7091700F77
:10AE80008091710F9091720F0E94DB4D00E09C0148
:10AE900046E55BE26C2F812F0E940B444EC0D630FA
:10AEA00031F58091C806863021F40E940385811116
:10AEB000D7C080912202882309F43FC011E080911D
:10AEC000C806863009F010E060917F0F7091800F06
:10AED0008091810F9091820F0E94DB4D00E09C01D8
:10AEE0004CE45BE26C2F812F0E940B4426C0D730CC
:10AEF00021F58091C806873021F40E9403858111D5
:10AF0000C8C0809122028823C1F011E08091C80658
:10AF1000873009F010E06091830F7091840F809169
:10AF2000850F9091860F0E94DB4D00E09C0148E365
:10AF30005BE26C2F812F0E940B44CF5FDF5FC53037
:10AF400009F0C9CE88E08093C706BBC00E94D07FBD
:10AF500080919506882309F4C8CEB3C081E00E9491
:10AF6000F884A12CC12CD12CE12C10ECF12E09E796
:10AF700014E420E030E040E85FE36FE57FE081EB40
:10AF80009BE26ADB80919506882309F4CACE99C0BA
:10AF900081E00E94F884A12CC12CD12CE12C10EC72
:10AFA000F12E09E714E420E030E040E85FE363E6D7
:10AFB0007FE083EA9BE250DB80919506882309F4C9
:10AFC000D8CE7FC081E00E94F884A12CC12CD12C66
:10AFD000E12C10ECF12E09E714E420E030E040E829
:10AFE0005FE367E67FE085E99BE236DB80919506CB
:10AFF000882309F4E6CE65C081E00E94F884A12C84
:10B00000C12CD12CE12C10ECF12E09E714E420E046
:10B0100030E040E85FE36BE67FE080E89BE21CDB2A
:10B0200080919506882309F4F4CE4BC081E00E94FC
:10B03000F884A12CC12CD12CE12C10ECF12E09E7C5
:10B0400014E420E030E040E85FE36FE67FE084E670
:10B050009BE202DB80919506882309F402CF31C080
:10B0600081E00E94F884A12CC12CD12CE12C10ECA1
:10B07000F12E09E714E420E030E0A9016FE77FE05A
:10B0800081E59BE2E9DA80919506882309F411CFE6
:10B0900018C081E00E94F884A12CC12CD12CE12C95
:10B0A00010ECF12E09E714E420E030E0A90163E898
:10B0B0007FE082E49BE2D0DA80919506882309F450
:10B0C00020CFDF91CF911F910F91FF90EF90DF90F4
:10B0D000CF90AF9008956F927F928F929F92AF9290
:10B0E000BF92CF92DF92EF92FF920F931F93CF9375
:10B0F000DF9300D01F92CDB7DEB761E081E00E9400
:10B10000A6806090C906712C61101AC08091C80693
:10B11000811104C00E9403858111C2C08091220266
:10B12000882309F4B5C081E09091C806911180E0B0
:10B1300004E024E040E85AE2672D0E94D743A8C00B
:10B1400081E0681226C08091C806813021F40E94F7
:10B1500003858111ADC080912202882309F498C033
:10B1600011E08091C806813009F010E06091FB0E7B
:10B170007091FC0E8091FD0E9091FE0E0E94DB4DB1
:10B1800000E09C0140E75AE2672D812F0E940B44AA
:10B190007FC082E0681226C08091C806823021F408
:10B1A0000E94038581119EC080912202882309F4A8
:10B1B0006FC011E08091C806823009F010E0609104
:10B1C000FF0E7091000F8091010F9091020F0E946D
:10B1D000DB4D00E09C0140E65AE2672D812F0E9482
:10B1E0000B4456C083E068122CC08091C80683309F
:10B1F00021F40E94038581118FC08091220288234F
:10B2000009F446C011E08091C806833009F010E0CF
:10B210008091030F9091040FA091050FB091060F3C
:10B2200089839A83AB83BC83CE0101960F94CD4D65
:10B2300000E09C0140E55AE2672D812F0E940B44FB
:10B2400027C084E0681224C08091C806843021F4AD
:10B250000E940385811198C0809122028823C1F049
:10B2600011E08091C806843009F010E06091070F6A
:10B270007091080F8091090F90910A0F0E94DB4D89
:10B2800000E09C0140E45AE2672D812F0E940B44AC
:10B290007394639485E0781237CF7092C7068DC09F
:10B2A0000E94D07F80919506882309F437CF85C00E
:10B2B00081E00E94F884A12CC12CD12CE12C10E853
:10B2C000F12E07E714E420E030E040E85FE36BEFA5
:10B2D0007EE088E79AE2C0D980919506882309F438
:10B2E0003ACF6BC081E00E94F884A12CC12CD12CF4
:10B2F000E12C10E8F12E07E714E420E030E040E80C
:10B300005FE36FEF7EE088E69AE2A6D9809195062A
:10B31000882309F449CF51C081E00E94F88420E0DD
:10B3200030E048EC52E46091030F7091040F80917B
:10B33000050F9091060F0F94565820E030E040E240
:10B3400051E40F943E550F948C561F92812C912CF2
:10B350009AE3A92E9DE4B92E6B0115EFE12E1FE7AC
:10B36000F12E00E010E02AE030E040E050E063E041
:10B370007FE088E59AE20E941F7F0F9080919506FA
:10B38000882309F43ACF19C081E00E94F884A12CE7
:10B39000C12CD12CE12C10E8F12E07E714E420E0B9
:10B3A00030E040E85FE367E07FE088E49AE254D968
:10B3B00080919506882309F44FCF0F900F900F903E
:10B3C0000F90DF91CF911F910F91FF90EF90DF9041
:10B3D000CF90BF90AF909F908F907F906F90089587
:10B3E0002F923F924F925F926F927F928F929F9295
:10B3F000AF92BF92CF92DF92EF92FF920F931F9383
:10B40000CF93DF93CDB7DEB729970FB6F894DEBFA1
:10B410000FBECDBF1C0179876887CA01B901E982D7
:10B42000FA820B831C83DE82CD82AF8220E030E083
:10B4300040E251E40F9456586B017C0120E030E06B
:10B4400040E057EC0F941B5818162CF0C12CD12C4F
:10B45000E12C27ECF22EC701B6010F9487562B0181
:10B460003C0120E030E040E251E469817A818B8147
:10B470009C810F9456584B015C0120E03EEF4FEF4A
:10B4800056E40F94185687FD07C0812C9EEF992E25
:10B49000AA24AA9496E4B92E20E030E040E251E4D8
:10B4A000E885F98560817181828193810F94565876
:10B4B0006B017C01C301B2010F94BA569B01AC0130
:10B4C000C701B6010F943E550F948C5669837A8359
:10B4D0008B839C83C501B4010F9487567B018C013B
:10B4E000E418F50806091709FF81FF938D809E80F7
:10B4F00080E4A82E8DE4B82EC980DA80A3019201E1
:10B5000068857985C1010E941F7F0F9029960FB62B
:10B51000F894DEBF0FBECDBFDF91CF911F910F9189
:10B52000FF90EF90DF90CF90BF90AF909F908F9063
:10B530007F906F905F904F903F902F9008959F92D3
:10B54000AF92BF92CF92DF92EF92FF920F931F9331
:10B55000CF93DF9300D01F92CDB7DEB761E081E0DB
:10B560000E94A6809090C906B12C91101AC08091BB
:10B57000C806811104C00E940385811104C1809115
:10B580002202882309F4F6C081E09091C806911147
:10B5900080E004E024E04EE25AE26B2D0E94D743A3
:10B5A000E9C081E098122CC08091C806813021F456
:10B5B0000E9403858111EFC080912202882309F443
:10B5C000D9C011E08091C806813009F010E0809167
:10B5D0004B0F90914C0FA0914D0FB0914E0F89835E
:10B5E0009A83AB83BC83CE0101960F946D4E00E02D
:10B5F0009C014AE15AE26B2D812F0E940B44BAC094
:10B6000082E098122CC08091C806823021F40E94FA
:10B6100003858111DCC080912202882309F4AAC02D
:10B6200011E08091C806823009F010E080914F0F40
:10B630009091500FA091510FB091520F89839A832E
:10B64000AB83BC83CE0101960F946D4E00E09C014C
:10B6500046E05AE26B2D812F0E940B448BC083E0A1
:10B6600098122CC08091C806833021F40E94038573
:10B670008111C9C080912202882309F47BC011E0A6
:10B680008091C806833009F010E08091530F9091AB
:10B69000540FA091550FB091560F89839A83AB83B5
:10B6A000BC83CE0101960F946D4E00E09C0142EFE9
:10B6B00059E26B2D812F0E940B445CC084E09812EC
:10B6C0002CC08091C806843021F40E94038581112A
:10B6D000B6C080912202882309F44CC011E0809109
:10B6E000C806843009F010E08091570F9091580FF0
:10B6F000A091590FB0915A0F89839A83AB83BC8371
:10B70000CE0101960F946D4E00E09C014CED59E284
:10B710006B2D812F0E940B442DC085E098122AC00A
:10B720008091C806853021F40E9403858111A3C051
:10B73000809122028823F1F011E08091C8068530C3
:10B7400009F010E080915B0F90915C0FA0915D0F6C
:10B75000B0915E0F89839A83AB83BC83CE0101963F
:10B760000F946D4E00E09C0146EC59E26B2D812F49
:10B770000E940B44B394939485E0B812F6CE86E011
:10B780008093C70693C00E94D07F8091950688233E
:10B7900009F4F5CE8BC081E00E94F884A12CE8E486
:10B7A000CE2EEDE4DE2EE12C1CE3F12E0CE116E4AE
:10B7B00020E030E040EA50E46BE47FE084E29AE28B
:10B7C0000FDE80919506882309F4F6CE6FC081E0E4
:10B7D0000E94F884A12C68E4C62E6DE4D62EE12CDC
:10B7E0001CE3F12E0CE116E420E030E040EA50E4E6
:10B7F0006FE47FE080E19AE2F3DD80919506882393
:10B8000009F409CF53C081E00E94F884A12C48E4D8
:10B81000C42E4DE4D42EE12C1CE3F12E0CE116E4F1
:10B8200020E030E040EA50E463E57FE08CEF99E20D
:10B83000D7DD80919506882309F41CCF37C081E0BD
:10B840000E94F884A12C2DEFC22E21E5D22EE12CEE
:10B850001CE3F12E0CE116E420E030E040EA50E475
:10B8600067E57FE087EE99E2BBDD8091950688234E
:10B8700009F42FCF1BC081E00E94F884A12C8FEF28
:10B88000C82E81E5D82EE12C1CE3F12E0CE116E444
:10B8900020E030E040EA50E46BE57FE081ED99E2A2
:10B8A0009FDD80919506882309F442CF0F900F9079
:10B8B0000F900F90DF91CF911F910F91FF90EF901C
:10B8C000DF90CF90BF90AF909F9008950F93CF934C
:10B8D000DF9361E081E00E94A680D091C906C0E0BC
:10B8E000D1111AC08091C806811104C00E9403853D
:10B8F0008111C6C080912202882309F4B8C081E07A
:10B900009091C806911180E004E024E045E15DE2F9
:10B910006C2F0E94D743ABC0D130D9F48091C806B8
:10B92000813021F40E9403858111B2C080912202EE
:10B93000882309F49CC081E09091C806913009F0F9
:10B9400080E003E02EE34EE05DE26C2F0E94D743DF
:10B950008EC0D230D9F48091C806823021F40E9482
:10B96000038581119FC080912202882309F47FC042
:10B9700081E09091C806923009F080E003E02EE368
:10B9800047E05DE26C2F0E94D74371C0D330D9F4F9
:10B990008091C806833021F40E94038581118CC0F8
:10B9A00080912202882309F462C081E09091C80648
:10B9B000933009F080E003E02EE340E05DE26C2F7D
:10B9C0000E94D74354C0D430D9F48091C806843043
:10B9D00021F40E940385811179C08091220288237D
:10B9E00009F445C081E09091C806943009F080E0E8
:10B9F00003E02EE346EF5CE26C2F0E94D74337C092
:10BA0000D530D1F48091C806853021F40E94038599
:10BA1000811166C080912202882349F181E09091D2
:10BA2000C806953009F080E003E02EE34BEE5CE2BF
:10BA30006C2F0E94D7431BC0D630C9F48091C80632
:10BA4000863021F40E940385811154C08091220226
:10BA5000882369F081E09091C806963009F080E073
:10BA600003E02EE340EE5CE26C2F0E94D743CF5FF1
:10BA7000DF5FC53009F034CF87E08093C70643C04D
:10BA80000E94D07F80919506882309F433CF3BC074
:10BA900088E691E60E941A4880919506882309F469
:10BAA00045CF31C08DE691E60E941A4880919506F7
:10BAB000882309F458CF27C082E791E60E941A48EC
:10BAC00080919506882309F46BCF1DC087E791E626
:10BAD0000E941A4880919506882309F47ECF13C0EE
:10BAE0008CE791E60E941A4880919506882309F414
:10BAF00091CF09C081E891E60E941A48809195068D
:10BB0000882309F4A3CFDF91CF910F910895CF92AD
:10BB1000DF92EF92FF92CF93C82F833029F467FD15
:10BB20006091630E6093DC060E949C2D6B017C018A
:10BB300024EA30E74DE75FE36091E1067091E206A9
:10BB40008091E3069091E4060F94185687FD05C096
:10BB50008AEF90E0A0E0B0E003C080E090E0DC017C
:10BB6000C80ED91EEA1EFB1EC092DD06D092DE066C
:10BB7000E092DF06F092E006C0932302CF91FF909F
:10BB8000EF90DF90CF9008952F923F924F925F9267
:10BB90006F927F928F929F92AF92BF92CF92DF92DD
:10BBA000EF92FF921F93CF93DF93CDB7DEB7289725
:10BBB0000FB6F894DEBF0FBECDBF1C01162F0E943A
:10BBC0000385882329F01092F8060E94D07FDBC0FD
:10BBD0002091F0063091F1063E832D83232B09F44A
:10BBE0009EC0E4E01E9FC001112498878F83FC0152
:10BBF000ED58FD4F80809180A280B38020E030E03E
:10BC00004AE754E4C501B4010F943E552B013C01B1
:10BC100020E030E04AE754E4C501B4010F943F55F9
:10BC20006B017C01809168028823B9F1113029F100
:10BC300098F0123091F5409060025090610260904F
:10BC4000620270906302C0906402D0906502E0903E
:10BC50006602F090670221C040905002509051025D
:10BC60006090520270905302C0905402D0905502DE
:10BC7000E0905602F090570210C040905802509049
:10BC8000590260905A0270905B02C0905C02D090A2
:10BC90005D02E0905E02F0905F022D813E81B9016D
:10BCA000330F880B990B0F94BA562091E10630910F
:10BCB000E2064091E3065091E4060F9456589B012A
:10BCC000AC01C501B4010F943F55EF81F885ED58E3
:10BCD000FD4F5F0160837183828393832D813E8159
:10BCE00037FF0CC0A30192010F94185687FF11C0B3
:10BCF000F50140825182628273820BC0A7019601D6
:10BD00000F941B5818162CF4F501C082D182E282E0
:10BD1000F3826FEF812FFBDE81E08093220210928D
:10BD2000F1061092F00680912202882361F124E04E
:10BD3000129FF0011124ED58FD4F80819181A28165
:10BD4000B38189839A83AB83BC832DEC3CEC4CECB0
:10BD50005DE36091E1067091E2068091E3069091C7
:10BD6000E4060F941B5887FD05C0CE0101960F9481
:10BD7000D74B05C060E2CE0101960F944F4CBC0139
:10BD8000C1010E946C4428960FB6F894DEBF0FBE26
:10BD9000CDBFDF91CF911F91FF90EF90DF90CF90BB
:10BDA000BF90AF909F908F907F906F905F904F90DB
:10BDB0003F902F90089560E086EA9DE2E5CE61E035
:10BDC0008FE99DE2E1CE62E088E99DE2DDCE0F934E
:10BDD0001F93CF93DF9300D01F92CDB7DEB7182FFC
:10BDE0000E940385882329F01092F8060E94D07FD4
:10BDF0005EC06091F0067091F1066115710571F1F8
:10BE0000072E000C880B990B0F94BA562091E1066F
:10BE10003091E2064091E3065091E4060F945658A3
:10BE20009B01AC0160917F02709180028091810240
:10BE3000909182020F943F5560937F02709380022D
:10BE40008093810290938202612F83E060DE81E023
:10BE5000809322021092F1061092F0068091220245
:10BE6000882329F1113019F40EE11DE202C009E224
:10BE70001DE22091A7053091A8054091A905509198
:10BE8000AA0560917F027091800280918102909159
:10BE900082020F943E5569837A838B839C83CE0103
:10BEA00001960F94D74BBC01C8010E946C440F90BF
:10BEB0000F900F900F90DF91CF911F910F910895E8
:10BEC0008FEF85CF80E083CF81E081CF21E0209389
:10BED000F8066093E1067093E2068093E306909380
:10BEE000E40620E040E060E070E08091A5059091DC
:10BEF000A6050C949D7F60E070E080E291E4E6CFBF
:10BF000060E070E080E89FE3E1CF6DEC7CEC8CECCE
:10BF10009DE3DCCF6DEC7CEC8CEC9CE3D7CFDF9227
:10BF2000EF92FF920F931F93CF93DF93F82EE42E9F
:10BF30007093A6056093A50561E081E00E94A6804C
:10BF4000D091C906C0E091E087E1D82E81E0F816D3
:10BF500059F1F81628F082E0F81609F449C06CC0CF
:10BF6000D111D8C0992389F08091C80618166CF0B9
:10BF70002091F0063091F1062F5F3F4F3093F1068C
:10BF80002093F0068F5F8093C80680912202882359
:10BF900009F435C100E010E021E041E061E97DE213
:10BFA0008C2F0E9474432BC1D111B4C0992389F006
:10BFB0008091C80618166CF02091F0063091F106B9
:10BFC0002F5F3F4F3093F1062093F0068F5F8093F1
:10BFD000C80680912202882309F431C100E010E0F4
:10BFE00021E041E06AE87DE28C2F0E94744327C182
:10BFF000D11190C0992389F08091C80618166CF071
:10C000002091F0063091F1062F5F3F4F3093F106FB
:10C010002093F0068F5F8093C806809122028823C8
:10C0200009F40BC100E010E021E041E063E87DE2AB
:10C030008C2F0E94744301C140917F025091800275
:10C0400060918102709182024093A7055093A805E8
:10C050006093A9057093AA05D11120C0992389F096
:10C060008091C80618166CF02091F0063091F10608
:10C070002F5F3F4F3093F1062093F0068F5F809340
:10C08000C80680912202882349F000E010E021E0F8
:10C0900041E069E77DE28C2F0E94744383E0F8124F
:10C0A00039C0E7FC02C0EE2D02C0E091630EDE9EB7
:10C0B000F0011124EC57F24F6481758186819781DC
:10C0C0002091450D211126C00F94875620913D02E5
:10C0D00030913E0262177307ECF4D130C9F48091BD
:10C0E000C806813021F40E9403858111B2C080917D
:10C0F0002202882369F081E09091C806913009F00E
:10C1000080E004E024E049E65DE26C2F0E94D74322
:10C1100082E096C0D130D9F48091C806813021F4F4
:10C120000E94038581119DC080912202882309F419
:10C1300066C081E09091C806913009F080E004E08B
:10C1400024E04FE55DE26C2F0E94D74358C0D23007
:10C15000D9F48091C806823021F40E9403858111B0
:10C1600088C080912202882309F449C081E090911F
:10C17000C806923009F080E003E02EE345E55DE279
:10C180006C2F0E94D7433BC0D330D1F48091C806B6
:10C19000833021F40E940385811175C080912202B1
:10C1A000882369F181E09091C806933009F080E01E
:10C1B00003E02EE34CE45DE26C2F0E94D7431FC0E6
:10C1C000D430E9F48091C806843021F40E940385BC
:10C1D000811163C080912202882389F081E09091CF
:10C1E000C806943009F080E003E02EE341E45DE20C
:10C1F0006C2F0E94D74382E0F81221C01EC082E05B
:10C20000F8121DC0D530C9F48091C806853021F4DC
:10C210000E94038581114BC080912202882369F01E
:10C2200081E09091C806953009F080E003E02EE3AC
:10C2300044E35DE26C2F0E94D74386E001C085E0B5
:10C24000CF5FDF5F90E0C53009F080CE8093C706F6
:10C2500037C00E94D07F80919506882309F447CF8C
:10C260002FC00E94D07F80919506882309F45CCF6F
:10C2700027C08BE79FE50E941A4880919506882386
:10C2800009F46FCF1DC080E89FE50E941A48809195
:10C290009506882309F482CF13C085E89FE50E94A4
:10C2A0001A4880919506882309F494CF09C08AE83A
:10C2B0009FE50E941A4880919506882309F4ACCF27
:10C2C000DF91CF911F910F91FF90EF90DF90089534
:10C2D0004FEF6BED7EE580E022CE4FEF6FED7EE518
:10C2E00081E01DCE4FEF63EE7EE582E018CE4FEF8A
:10C2F00060E67FE583E013CE40E062E67FE583E021
:10C300000ECE41E064E67FE583E009CE0F93CF9344
:10C31000DF9361E081E00E94A680D091C906C0E071
:10C32000D1111AC08091C806811104C00E940385F2
:10C3300081118BC080912202882309F47EC081E0A4
:10C340009091C806911180E004E024E04BED5CE29E
:10C350006C2F0E94D74371C0D130D9F48091C806A8
:10C36000813021F40E940385811177C080912202DF
:10C37000882309F462C081E09091C806913009F0E9
:10C3800080E003E02EE341ED5CE26C2F0E94D74396
:10C3900054C0D230D9F48091C806823021F40E9472
:10C3A0000385811164C080912202882309F445C06D
:10C3B00081E09091C806923009F080E000E22EE31F
:10C3C00043EC5CE26C2F0E94D74337C0D330D1F4EA
:10C3D0008091C806833021F40E940385811151C0E9
:10C3E00080912202882349F181E09091C806933020
:10C3F00009F080E000E22EE345EB5CE26C2F0E9446
:10C40000D7431BC0D430C9F48091C806843021F4CE
:10C410000E94038581113FC080912202882369F028
:10C4200081E09091C806943009F080E000E22EE3AC
:10C4300040EA5CE26C2F0E94D743CF5FDF5FC530DC
:10C4400009F06ECFC093C7062FC00E94D07F8091A5
:10C450009506882309F46ECF27C086E69CE50E94E6
:10C460001A4880919506882309F480CF1DC080ED7D
:10C470009CE20E941D7F80919506882309F493CF4A
:10C4800013C08FEB9CE20E941D7F8091950688234C
:10C4900009F4A6CF09C081EB9CE20E941D7F809128
:10C4A0009506882309F4B8CFDF91CF910F910895B5
:10C4B000CF93DF93EC01CB01BA010F94BA560F94DE
:10C4C000875679836883DF91CF91089568E572E696
:10C4D0008FEE92E60C94E57F0F931F93CF93DF933B
:10C4E00061E081E00E94A680C091C906D0E081E0B1
:10C4F000C11122C0882389F08091C80618166CF0FB
:10C500002091F0063091F1062F5F3F4F3093F106F6
:10C510002093F0068F5F8093C806809122028823C3
:10C5200009F441C000E010E020E041E060E17FE27A
:10C530008D2F0E94744337C0C130D1F48091C8065A
:10C54000813021F40E940385811137C0809122023D
:10C55000882349F181E09091C806913009F080E08C
:10C5600000E22EE345E05FE26D2F0E94D7431BC03F
:10C57000C230C9F48091C806823021F40E9403853C
:10C58000811122C080912202882369F081E090917C
:10C59000C806923009F080E000E22EE341EF5EE24F
:10C5A0006D2F0E94D743DF5FCF5F80E0D53009F069
:10C5B0009FCF83E08093C7060DC0C093B40C8091D9
:10C5C0009506882319F206C0C093B40C8091950695
:10C5D0008823C1F2DF91CF911F910F9108950F949D
:10C5E000BA560F948756CB010D94D649EF92FF921D
:10C5F0000F931F93CF93DF93CDB7DEB72B970FB673
:10C60000F894DEBF0FBECDBF7C014091AC05642F16
:10C61000042E000C770B8091AD05823051F08330F1
:10C6200019F02CE83FE20AC047FF06C028E93FE2C4
:10C6300005C02AEA3FE202C021EA3FE27F934F931E
:10C640003F932F938E010F5F1F4F1F930F930F94F4
:10C65000BA5E8091AC0597E1899FF0011124EC57F7
:10C66000F24F98E0899FD0011124A35DBD4F16962B
:10C670004D915C9117974F50510997010F900F9072
:10C680000F900F900F900F904E155F050CF49A01CC
:10C69000318720870E94C6B8C8010E94DB812B9693
:10C6A0000FB6F894DEBF0FBECDBFDF91CF911F91C3
:10C6B0000F91FF90EF900895E091AC0587E1E802BB
:10C6C000F0011124EC57F24F808591858FCF7F9236
:10C6D0008F929F92AF92BF92CF92DF92EF92FF9292
:10C6E0000F931F93CF93DF93782E8093AD056093C4
:10C6F000AC0561E081E00E94A680D091C906C0E04F
:10C7000081E0D1112EC0882389F08091C8061816C7
:10C710006CF02091F0063091F1062F5F3F4F30937F
:10C72000F1062093F0068F5F8093C8068091220265
:10C73000882309F494C022E0721649F033E07312A2
:10C7400003C06EE67FE205C06EE57FE202C06EE7E1
:10C750007FE200E010E021E041E08C2F0E94744372
:10C760007EC0D130D9F48091C806813021F40E9476
:10C77000038581117DC080912202882309F46FC056
:10C7800081E09091C806913009F080E004E024E057
:10C7900049EE5FE26C2F0E94D74361C0D230D9F4DA
:10C7A0008091C806823021F40E940385811168C0FF
:10C7B00080912202882309F452C081E09091C8063A
:10C7C000923009F080E000E22EE34DED5FE26C2F45
:10C7D0000E94D74344C0D330D1F48091C80683303F
:10C7E00021F40E940385811156C080912202882382
:10C7F000B1F181E09091C806933009F080E000E249
:10C800002EE341ED5FE26C2F0E94D74328C0D43065
:10C8100031F58091C806843021F40E94038581118E
:10C8200045C0809122028823D1F011E08091C80692
:10C83000843009F010E02091AC0537E12303F001CA
:10C840001124EC57F24F808591850F94D64900E072
:10C850009C0143EB5FE26C2F812F0E940B44CF5F62
:10C86000DF5F80E0C53009F04CCFC093C7065BC0E6
:10C870000E94D07F80919506882309F47CCF53C015
:10C880008091B4059091B505B1DE8091950688231D
:10C8900009F48ECF48C08091B6059091B705A6DE09
:10C8A00080919506882309F4A0CF3DC081E00E94C5
:10C8B000F8840091AC0527E1020380011124F801FE
:10C8C000EC57F24F60857185072E000C880B990B91
:10C8D0000F94BA5620E030E040EF52E40F943E55FA
:10C8E0000F948C56F801E457F24F1F928CE5882E76
:10C8F00083E6982E96E6A92E92E6B92E6B011AEAE7
:10C90000E12EF12C00E010E028E730E040E050E0BC
:10C91000BF0182EC9FE20E941F7F0F9080919506DD
:10C92000882309F47ECFDF91CF911F910F91FF9063
:10C93000EF90DF90CF90BF90AF909F908F907F90BF
:10C94000089560E081E0C3CE61E081E0C0CE0F9346
:10C95000CF93DF9361E081E00E94A680C091C90679
:10C96000D0E0C11118C08091C806811104C00E9496
:10C970000385811198C080912202882361F081E0B3
:10C980009091C806911180E004E024E049E55FE25F
:10C990006D2F0E94D74320918C0D30918D0D809189
:10C9A000450D81115AC080913D0290913E02281799
:10C9B0003907E4F4C13031F58091C806813021F4A3
:10C9C0000E940385811177C0809122028823D1F0D3
:10C9D00081E09091C806913009F080E003E02EE3F9
:10C9E00040E45FE26D2F0E94D7430CC0C13009F0D4
:10C9F0009CC08091C806813009F47AC080912202DF
:10CA000081117BC08091A30D9091A40D2091450DC3
:10CA1000211125C020913D0230913E0282179307DB
:10CA2000F4F4C230B9F58091C806823021F40E9436
:10CA3000038581114AC080912202882359F181E047
:10CA40009091C806923009F080E003E02EE347E2BF
:10CA50005FE26D2F0E94D7431DC0C13051F2C2303A
:10CA6000C9F48091C806823021F40E9403858111A7
:10CA700036C080912202882369F081E09091C80637
:10CA8000923009F080E000E22EE347E25FE26D2F92
:10CA90000E94D743DF5FCF5FD53009F062CF83E0DC
:10CAA0008093C70647C00E94D07F80919506882357
:10CAB00009F461CF3FC081EA94E60E941A48809150
:10CAC0009506882309F480CF35C084EA94E60E9455
:10CAD0001A4880919506882309F4ADCF2BC081E1D7
:10CAE0009FE20E941D7F80919506882311F222C04B
:10CAF0000E94038581110FC081CF81E09091C8060B
:10CB0000913009F080E000E22EE340E45FE26D2F17
:10CB10000E94D74377CF8CE19FE20E941D7F8091D6
:10CB20009506882309F46ACF05C08091A30D9091E2
:10CB3000A40D70CFDF91CF910F9108958F929F92A6
:10CB4000AF92BF92CF92DF92EF92FF920F931F931B
:10CB5000CF93DF934C015B016A0160E085E00E94A6
:10CB6000A680D091C906F12C82E0E82ED1111AC01E
:10CB700080912202882321F180912502823041F0A8
:10CB8000833019F466EC7EE205C064EB7EE202C0FD
:10CB900066ED7EE200E010E021E041E08F2D0E9492
:10CBA00074430EC0D13061F480912202882341F099
:10CBB00000E010E020E041E0B4018F2D0E947443BA
:10CBC000A114B10481F0D23081F480912202882333
:10CBD00009F46EC000E010E020E041E0B5018F2DC7
:10CBE0000E94744365C0C2E001C0C3E0C114D10417
:10CBF00091F0DC130FC080912202882351F000E0F5
:10CC000010E020E041E0B6018F2D0E947443CD2F4B
:10CC100001C0CD2FCF5F21E030E0A114B10411F4A9
:10CC200020E030E081E090E0C114D10411F480E014
:10CC300090E0820F931F029781F0DC130DC080916A
:10CC40002202882349F000E010E020E041E06FEE8E
:10CC50007EE28F2D0E947443CF5FDC1314C080915D
:10CC60002202882371F000E010E021E040E064EE51
:10CC70007EE28F2D0E9474436091AB058F2D0E9440
:10CC8000FC42E0922202F394DF5F85E0F8126ECF5F
:10CC9000CF5FC093C706DF91CF911F910F91FF9097
:10CCA000EF90DF90CF90BF90AF909F908F900895BE
:10CCB000C3E0C114D10409F0ADCFADCF40E050E0E6
:10CCC00060E070E089EA9EE239CF40EA5EE260E926
:10CCD0007EE287E89EE232CF40E050E067E77EE206
:10CCE0008EE69EE22BCF40E050E06FE57EE280E5ED
:10CCF0009EE224CF40E050E061E47EE284E39EE2E5
:10CD00001DCF48E25EE267E17EE287E09EE216CF59
:10CD100040E050E069EF7DE280EF9DE20FCF40E020
:10CD200050E060EE7DE283ED9DE208CF40E050E010
:10CD300066EC7DE285EC9DE201CF40E050E066EBE1
:10CD40007DE28DEA9DE2FACE611160932502409367
:10CD5000AB05082E000C990BAA0BBB0B8C30910570
:10CD6000A0F5FC018827EA56FF4F8F4F0D94A0597C
:10CD700085E696E61FC08CE696E61CC08FE896E630
:10CD800019C081E896E616C088E896E613C08DE9DA
:10CD900096E610C086E996E60DC08AE796E60AC0D8
:10CDA00083E796E607C01092B40C8CE692E602C0C8
:10CDB0008EE596E6009749F021E02093F80620E002
:10CDC00040E060E070E00C949D7F0C94C97FCF92AE
:10CDD000DF92EF92FF920F931F9385EAC82E80E3B4
:10CDE000D82EE12CF12C0AE910E320ED3FE74CE2CC
:10CDF0005BE865E970E380E990E30E94FE811F91A2
:10CE00000F91FF90EF90DF90CF9008959091D60909
:10CE100093FB882780F993FF06C081E09091060874
:10CE2000911101C080E00895EF92FF920F931F933C
:10CE3000CF93DF9361E081E00E94A680C091C90694
:10CE400010E0C11118C08091C806811104C00E9471
:10CE5000038581119FC180912202882361F081E0C6
:10CE60009091C806911180E004E024E044E850E38A
:10CE7000612F0E94D7438091D60982FB002700F9D9
:10CE800082FD07C0D1E09091FC17913019F0D0E0FD
:10CE900001C0D02F83FBEE24E0F883FF03C0B6DF90
:10CEA000F82E01C0F12CDD2309F458C0C130D9F4AB
:10CEB0008091C806813021F40E940385811172C1DE
:10CEC00080912202882309F47FC181E09091C806F5
:10CED000913009F080E000E22EE348E750E3612F53
:10CEE0000E94D74371C1C230D9F48091C806823004
:10CEF00021F40E94038581115DC180912202882363
:10CF000009F462C181E09091C806923009F080E096
:10CF100003E02EE34DE650E3612F0E94D74354C156
:10CF2000C33009F063C08091C806833021F40E94A9
:10CF3000038581114BC180912202882309F444C1E9
:10CF400081E09091C806933009F080E003E02EE381
:10CF500048E650E3612F0E94D74336C18091FC1709
:10CF6000823029F053DF8823F9F001111DC0C13050
:10CF7000E9F48091C806813021F40E940385811173
:10CF80002FC180912202882309F432C181E090915F
:10CF9000C806913009F080E000E22EE34BE550E353
:10CFA000612F0E94D74324C1D1E001C0D2E0CD134C
:10CFB0001BC08091C8068C1304C00E940385811198
:10CFC00019C180912202882371F081E09091C806F6
:10CFD0009C1380E003E02EE342E550E3612F0E94C2
:10CFE000D743DC2F01C0DC2FDF5F01C0D4E0CD13BD
:10CFF0001BC08091C8068C1304C00E940385811158
:10D0000003C180912202882371F081E09091C806CB
:10D010009C1380E003E02EE346E450E3612F0E947E
:10D02000D743DC2F01C0DC2F81E08D0FC81318C05F
:10D030008091C8068C1304C00E9403858111EEC044
:10D0400080912202882361F081E09091C8069C13B0
:10D0500080E003E02EE348E350E3612F0E94D743D2
:10D0600082E08D0FC81318C08091C8068C1304C0CD
:10D070000E9403858111DCC080912202882361F027
:10D0800081E09091C8069C1380E003E02EE348E223
:10D0900050E3612F0E94D74383E08D0FC81318C05F
:10D0A0008091C8068C1304C00E9403858111CAC0F8
:10D0B00080912202882361F081E09091C8069C1340
:10D0C00080E003E02EE34AE150E3612F0E94D74362
:10D0D00094E09D0FEE2009F43BC0F11053C0C9133A
:10D0E00018C08091C8068C1304C00E94038581116A
:10D0F000B3C080912202882361F081E09091C8063C
:10D100009C1380E000E22EE347E050E3612F0E9491
:10D11000D74385E08D0FC81318C08091C8068C13C3
:10D1200004C00E9403858111A1C08091220288233E
:10D1300061F081E09091C8069C1380E003E02EE34B
:10D1400049EF5FE2612F0E94D74396E09D0F1AC01E
:10D15000C91316C08091C8068C1302C00E940385B3
:10D1600080912202882361F081E09091C8069C138F
:10D1700080E000E22EE34EEE5FE2612F0E94D74393
:10D1800095E09D0F1F5FCF5F153009F05ACE909349
:10D19000C70675C00E94D07F80919506882309F448
:10D1A0005ACE6DC00E943F8B80919506882309F46A
:10D1B00087CE65C087EE96E60E941A488091950654
:10D1C000882309F49ACE5BC0D4E02ECF8EEB9AE68A
:10D1D0000E941A4880919506882309F4ACCE4FC06E
:10D1E0000E94518B80919506882309F4CACE47C0CE
:10D1F000D2E0FACE86E891E60E941A488091950620
:10D20000882309F4DECE3BC08DEE9DE60E941A48CD
:10D2100080919506882309F4F4CE31C08BEB9DE70D
:10D220000E941A4880919506882309F409CF27C0E7
:10D2300087EA94E60E941A4880919506882309F4AB
:10D240001BCF1DC086E49DE60E941A48809195067A
:10D25000882309F42DCF13C086E190E30E941D7F3F
:10D2600080919506882309F444CF09C082E199E4AE
:10D270000E941A4880919506882309F456CFDF91C1
:10D28000CF911F910F91FF90EF9008956091800DC5
:10D2900070E080E00C9407B460918B0270918C0276
:10D2A000072E000C880B990B0F94BA562AE037ED25
:10D2B00043E25CE30F9456586093830270938402B8
:10D2C0008093850290938602089560918D027091FB
:10D2D0008E02072E000C880B990B0F94BA562AE089
:10D2E00037ED43E25CE30F945658609387027093E6
:10D2F00088028093890290938A020895CF93DF93E6
:10D30000EC01CB01BA010F94BA560F948C56688386
:10D31000DF91CF91089581E00C94C6B880E00C9421
:10D32000C6B86EE779E687E999E60C94E57F0F9435
:10D33000BA560F948C56862F0D945A490F948756DF
:10D34000CB010D94D649EF92FF920F931F93CF9389
:10D35000DF9300D01F92CDB7DEB7082F7B010E946C
:10D360000385882329F01092F8060E94D07F3BC0E5
:10D370006091F0067091F1066115710551F01092FF
:10D38000F1061092F00681E080932202802F0E9425
:10D390008DAB80912202882331F184E0089F8001C7
:10D3A0001124055F104F6091960C7091970C072E19
:10D3B000000C880B990B0F94BA569B01AC01F80135
:10D3C00060817181828193810F94565869837A8339
:10D3D0008B839C8360E2CE0101960F94E74CBC01E5
:10D3E000C7010E946C440F900F900F900F90DF9137
:10D3F000CF911F910F91FF90EF90089568E471E332
:10D4000080E0A1CF6DE371E381E09DCF20E040E0BB
:10D4100060E070E00E949D7F81E08093F8061092AA
:10D42000970C1092960C08958EEF99E6EFCF82E05C
:10D430009AE6ECCF2F923F924F925F926F927F923B
:10D440008F929F92AF92BF92CF92DF92EF92FF9214
:10D450000F931F93CF93DF93CDB7DEB729970FB606
:10D46000F894DEBF0FBECDBF1C01798768876901C4
:10D470001A830983EB82BA01550F880B990B0F941D
:10D48000BA564B015C0120E030E040E057EC0F94CD
:10D490001B5818162CF0812C912CA12C27ECB22EA5
:10D4A000C501B4010F9487562B013C01B601DD0C78
:10D4B000880B990B0F94BA564B015C0120E03EEFAC
:10D4C0004FEF56E40F94185687FD07C0812C9EEF4E
:10D4D000992EAA24AA9496E4B92EE885F98560814C
:10D4E0007181072E000C880B990B0F94BA566B01B3
:10D4F0007C01C301B2010F94BA569B01AC01C70174
:10D50000B6010F943E550F948C566C837D838E83A9
:10D510009F83C501B4010F9487567B018C01E418E9
:10D52000F50806091709FB81FF9389809A8086E632
:10D53000A82E82E6B82ECC80DD80A30192016885FA
:10D540007985C1010E941F7F0F9029960FB6F8942C
:10D55000DEBF0FBECDBFDF91CF911F910F91FF9026
:10D56000EF90DF90CF90BF90AF909F908F907F9083
:10D570006F905F904F903F902F9008958F929F9261
:10D58000AF92BF92CF92DF92EF92FF920F931F93D1
:10D59000CF93DF9361E081E00E94A680D091C9061D
:10D5A000C0E0D1111AC08091C806811104C00E9448
:10D5B0000385811187C180912202882309F479C1F2
:10D5C00081E09091C806911180E004E024E048E3F6
:10D5D00051E36C2F0E94D7436CC1D13039F5809153
:10D5E000C806813021F40E940385811173C18091A6
:10D5F0002202882309F45DC111E08091C8068130C0
:10D6000009F010E060916D0270916E02072E000C1F
:10D61000880B990B0F94BA5691DE00E09C014CE206
:10D6200051E36C2F812F0E940B4443C1D23039F556
:10D630008091C806823021F40E94038581115CC16B
:10D6400080912202882309F434C111E08091C80638
:10D65000823009F010E060918C0D70918D0D072ED5
:10D66000000C880B990B0F94BA5668DE00E09C0101
:10D670004AE151E36C2F812F0E940B441AC1D33031
:10D6800039F58091C806833021F40E940385811109
:10D6900048C180912202882309F40BC111E08091D6
:10D6A000C806833009F010E06091A30D7091A40DBD
:10D6B000072E000C880B990B0F94BA563FDE00E042
:10D6C0009C0148E051E36C2F812F0E940B44F1C074
:10D6D000D43039F58091C806843021F40E94038546
:10D6E000811134C180912202882309F4E2C011E043
:10D6F0008091C806843009F010E060915B0D709154
:10D700005C0D072E000C880B990B0F94BA5616DE91
:10D7100000E09C0140E051E36C2F812F0E940B44FC
:10D72000C8C0D53001F58091C806853021F40E942B
:10D730000385811120C180912202882309F4B9C098
:10D7400011E08091C806853009F010E08091800DCD
:10D750000F945A4900E09C0148EE50E36C2F812F52
:10D760000E940B44A6C0D63039F58091C806863099
:10D7700021F40E940385811121C180912202882316
:10D7800009F497C011E08091C806863009F010E0D6
:10D7900060918B0270918C02072E000C880B990B04
:10D7A0000F94BA56CBDD00E09C014AED50E36C2F9C
:10D7B000812F0E940B447DC0D73039F58091C80677
:10D7C000873021F40E94038581110AC180912202D1
:10D7D000882309F46EC011E08091C806873009F0F3
:10D7E00010E060918D0270918E02072E000C880B64
:10D7F000990B0F94BA56A2DD00E09C014CEC50E36B
:10D800006C2F812F0E940B4454C0D830D9F48091E2
:10D81000C806883021F40E9403858111F3C08091ED
:10D820002202882309F445C081E09091C80698300F
:10D8300009F080E003E02EE341EC50E36C2F0E94FE
:10D84000D74337C0D930D1F48091C806893021F44C
:10D850000E9403858111E0C080912202882349F152
:10D8600081E09091C806993009F080E003E02EE352
:10D8700046EB50E36C2F0E94D7431BC0DA30C9F44B
:10D880008091C8068A3021F40E9403858111CEC0A0
:10D8900080912202882369F081E09091C8069A3035
:10D8A00009F080E003E02EE347EA50E36C2F0E948A
:10D8B000D743CF5FDF5FC53009F073CE8BE0809335
:10D8C000C706BDC00E94D07F80919506882309F4C9
:10D8D00072CEB5C0E12C00E010E027EE33E04AE064
:10D8E00050E06DE672E082E391E3A4DD809195065D
:10D8F000882309F47CCEA3C081E00E94F884E12C47
:10D900000EE819E622E231E040E050E06CE87DE00C
:10D9100083E291E38FDD80919506882309F490CE10
:10D920008EC081E00E94F884E12C0BE819E622E227
:10D9300031E040E050E063EA7DE081E191E37ADDAF
:10D9400080919506882309F4A4CE79C081E00E94D5
:10D95000F884E12C00E219EB2CE830E040E050E0E4
:10D960006BE57DE084E091E365DD80919506882399
:10D9700009F4B8CE64C081E00E94F884C090800DA4
:10D98000D12C1F9286E4882E89E6982E91E9A92E43
:10D9900099E6B92EE12CF12C8701EA9420E030E0E1
:10D9A000A90160E87DE084EF90E30E941F7F0F9063
:10D9B00080919506882309F4BECE41C0E12C0CE489
:10D9C00019E627EE33E04AE050E06BE872E081EEC2
:10D9D00090E330DD80919506882309F4CECE2FC0E8
:10D9E000E12C05E619E627EE33E04AE050E06DE869
:10D9F00072E083ED90E31EDD80919506882309F4A3
:10DA0000E5CE1DC084E19AE60E941A4880919506F1
:10DA1000882309F404CF13C087E19AE60E941A48CC
:10DA200080919506882309F417CF09C08CE091E80E
:10DA30000E941A4880919506882309F429CFDF9126
:10DA4000CF911F910F91FF90EF90DF90CF90BF90FB
:10DA5000AF909F908F9008950E940385882321F0B6
:10DA60001092F8060E94D07F0C9490420E94038589
:10DA7000882341F020E040E060E070E08CE29DE629
:10DA80000E949D7F61E080E00C9426420F93CF932B
:10DA9000DF9361E081E00E94A680D091C906C0E0DA
:10DAA000D11117C08091C806811104C00E9403855E
:10DAB00081114CC080912202882309F43EC081E08C
:10DAC0009091C806911180E004E024E04AE651E319
:10DAD00031C0D130B9F48091C806813021F40E9460
:10DAE000038581113BC080912202882331F181E0BE
:10DAF0009091C806913009F080E003E02EE349E5FB
:10DB000051E318C0D530C9F48091C806853021F49E
:10DB10000E94038581112CC080912202882369F024
:10DB200081E09091C806953009F080E003E02EE393
:10DB300043E551E36C2F0E94D743CF5FDF5FC530D1
:10DB400009F0AECF86E08093C7061AC00E94D07F4E
:10DB500080919506882309F4ADCF12C086E39DE637
:10DB60000E941A4880919506882309F4BCCF08C00A
:10DB700080E398E40E941A4880919506882361F218
:10DB8000DF91CF910F91089527E1629FF001112459
:10DB9000EC57F24F28E0629FD0011124A35DBD4FE6
:10DBA00016962D913C9117972F5031092817390758
:10DBB0000CF4C90191878087862F0C94C6B860E069
:10DBC00070E080E00E9407B460E070E081E00E94B5
:10DBD00007B40E946DB90C94C97F8F929F92AF9247
:10DBE000BF92CF92DF92EF92FF920F931F93CF934A
:10DBF000DF9361E081E00E94A680D091C906C0E079
:10DC0000D1111AC08091C806811104C00E940385F9
:10DC10008111DBC080912202882309F498C081E041
:10DC20009091C806911180E004E024E04CEB51E3B0
:10DC30006C2F0E94D7438BC0D13011F58091C8065C
:10DC4000813021F40E9403858111C7C08091220296
:10DC5000882309F47CC011E08091C806813009F066
:10DC600010E080918C0D90918D0D0F94D64900E0BD
:10DC70009C014AEA51E36C2F812F0E940B4467C03C
:10DC8000D23011F58091C806823021F40E940385BC
:10DC90008111C9C080912202882309F458C011E083
:10DCA0008091C806823009F010E08091A30D909118
:10DCB000A40D0F94D64900E09C0148E951E36C2F74
:10DCC000812F0E940B4443C0D33009F58091C806D0
:10DCD000833021F40E9403858111CBC08091220200
:10DCE0008823A9F111E08091C806833009F010E083
:10DCF00080915B0D90915C0D0F94D64900E09C01E2
:10DD000040E951E36C2F812F0E940B4420C0D43096
:10DD1000F1F48091C806843021F40E9403858111BA
:10DD2000CDC080912202882391F011E08091C80635
:10DD3000843009F010E08091800D0F942B4900E0B1
:10DD40009C0148E751E36C2F812F0E940B44809186
:10DD50008C0D90918D0D892B49F481E02091A30DBC
:10DD60003091A40D232B19F480E001C081E02091B3
:10DD70005B0D30915C0D232B11F48823E9F0D53035
:10DD8000C9F48091C806853021F40E940385811171
:10DD9000B8C080912202882369F081E09091C80682
:10DDA000953009F080E000E22EE34FE651E36C2F5E
:10DDB0000E94D74386E001C085E0CF5FDF5FC530BA
:10DDC00009F01ECF8093C706A2C00E94D07F809129
:10DDD0009506882309F41ECF9AC081E00E94F8843A
:10DDE000C0908C0DD0908D0D1F92FEE88F2EF9E61D
:10DDF0009F2EA6E6AA2EA2E6BA2E12E2E12EFF245C
:10DE0000F39400E010E020E030E0A9016CE87DE050
:10DE100083EB91E30E941F7F0F90809195068823EA
:10DE200009F414CF74C081E00E94F884C090A30D5F
:10DE3000D090A40D1F926BE8862E69E6962E76E6AA
:10DE4000A72E72E6B72E12E2E12EFF24F39400E033
:10DE500010E020E030E0A90163EA7DE081EA91E38F
:10DE60000E941F7F0F9080919506882309F412CF9E
:10DE70004EC081E00E94F884C0905B0DD0905C0D94
:10DE80001F9230E2832E39EB932E46E6A42E42E613
:10DE9000B42E1CE8E12EF12C00E010E020E030E090
:10DEA000A9016BE57DE084E991E30E941F7F0F905B
:10DEB00080919506882309F411CF29C081E00E9442
:10DEC000F884C090800DD12C1F9286E4882E89E6BC
:10DED000982E9DE1A92E9AE4B92EE12CF12C870110
:10DEE000EA9420E030E0A90160E87DE084E891E375
:10DEF0000E941F7F0F9080919506882309F411CF0F
:10DF000006C05DDE80919506882309F442CFDF913B
:10DF1000CF911F910F91FF90EF90DF90CF90BF9026
:10DF2000AF909F908F90089580E095E29093BD050B
:10DF30008093BC058CE491E09093B9058093B8057B
:10DF400080EC9EEF9093BB058093BA059091C1053C
:10DF500080E2890F863740F080EF890F20E431E0BE
:10DF60003093BB052093BA051092BE058093BF0580
:10DF70008FEF8093C00508958F929F92BF92CF92AA
:10DF8000DF92EF92FF920F931F93CF93DF931F9235
:10DF9000CDB7DEB7E1D7882309F4D6C18091F0066A
:10DFA000863214F085E202C087FD80E0282F082E1B
:10DFB000000C330B3093F1062093F006982F990F45
:10DFC000890F8093C10580911106882309F4BCC193
:10DFD0002091BA053091BB050091BE051091BF0597
:10DFE000020F131FE090BC05F090BD058091B805AD
:10DFF0009091B905E80EF91E01304FE7140768F05B
:10E000003195219531093093BB052093BA056CED0C
:10E0100070E085E090E00F944E50F7FE15C08091BF
:10E02000B8059091B9059195819591099093B9059D
:10E030008093B80568E171E085E090E00F944E5060
:10E0400081E08093C00517C081E0E81680E4F806FF
:10E0500094F06BE470E084EF91E00F944E50809167
:10E06000CB0581508093CB05882311F05DDF6CC117
:10E070001092110669C12091B8053091B905C70108
:10E080009A508130934108F098C08F2D992787FDD1
:10E090009A950A9765E070E00F944F59812F17FF0A
:10E0A00002C087E0810F482F45954595459581E051
:10E0B00090E0A0E0B0E004C0880F991FAA1FBB1F2A
:10E0C0004A95D2F7FB01EE0FFF1FEE53FA4F408146
:10E0D00051818A0108231923012B09F419C1809564
:10E0E0009095842395239183808384E090E0861B20
:10E0F000970B4091120650911306840F951F909331
:10E100001306809312068091CA0581508093CA0538
:10E11000811103C082E080931106932F9095991F7F
:10E120009927991F8091C005881F8827881F9817F5
:10E13000F1F03195219531093093B9052093B80557
:10E1400020E130E040E050E060EF7FEF8FEF9FEFA5
:10E150000E9438382091BA053091BB05620F731FB9
:10E160007093BB056093BA0560E773E021C08091AE
:10E17000BA059091BB059195819591099093BB0546
:10E180008093BA0520E130E040E050E060EF7FEF9F
:10E190008FEF9FEF0E9438382091B8053091B90574
:10E1A000620F731F7093B9056093B80560E872E061
:10E1B00085E090E00F944E50ABC0121613060CF0A1
:10E1C000A7C0FDE3FF1A41E0E41642E0F40608F0C0
:10E1D0009FC08091C105181B103108F099C031957E
:10E1E000219531093093B9052093B80560E773E0B4
:10E1F00083E090E00F944E508FEF8093C00521E0B4
:10E2000012300CF020E08EEF810F8C30A0F0809166
:10E21000BA059091BB0541E050E01816190614F0BC
:10E2200040E050E030E04217530709F055C09195A7
:10E230008195910927C0143050F520E030E0A90104
:10E2400060EC7FEF8FEF9FEF0E9438382091BA0586
:10E250003091BB05620F731F7093BB056093BA05C5
:10E2600061157E4F34F480E09EEF9093BB05809360
:10E27000BA058091BA059091BB058130924064F156
:10E2800080E092E09093BB058093BA0525C01C30D6
:10E290001CF120E430E040E050E060E070E0CB01B1
:10E2A0000E9438382091BA053091BB05620F731F68
:10E2B0007093BB056093BA0561157E4F34F480E01E
:10E2C0009EEF9093BB058093BA058091BA0590911B
:10E2D000BB0581309240A4F6809111068230C1F4D2
:10E2E00080E48093CA058FEF9FEF9093C3058093DE
:10E2F000C2059093C5058093C4059093C70580938C
:10E30000C6059093C9058093C80581E080931106E6
:10E310002091BE053091BF058091BA059091BB0553
:10E32000820F931F9093BF058093BE052091BC057B
:10E330003091BD058091B8059091B905820F931F6A
:10E340009093BD058093BC0561E08BE694E00E944C
:10E35000CF3280919F048E3130F080919F048E33B4
:10E3600008F456C05AC08091A1048A30B0F382EC00
:10E37000E82E85E0F82E9AE0892E912CB82C809119
:10E380009F0490E094012C5F3F4F281739075CF4FD
:10E3900042E0E40EF11C85E0880E911CEEE18E1641
:10E3A000910461F7DACF8091A104881588F330E0F9
:10E3B000C12CD12CF70180819181A0E0B0E00C2C20
:10E3C00004C0B695A795979587950A94D2F780FDD6
:10E3D00007C0FFEFCF1ADF0A385F303859F7D8CFC0
:10E3E00000E010E0A801480D591D80919F0490E0C5
:10E3F000481759073CF08091A10490E084179507D5
:10E400000CF055C00F5F1F4F0430110559F7E1CFD5
:10E410008091A1048C3308F055C0809111068823A7
:10E42000B1F08091BD05482F582F550F550B9A011B
:10E4300033272F5F3F4F80919F0490E028173907C3
:10E440003CF08091A104841708F04DC001C09DD517
:10E4500080919F048B30D0F469E080E00E94D6392F
:10E4600080911206909113060E94DB3969E08EE6D6
:10E470000E94D6392091CB0583E090E0821B910960
:10E480006FEF7FEF8F539E4C0E94303A0E940385BE
:10E49000882391F10F90DF91CF911F910F91FF9001
:10E4A000EF90DF90CF90BF909F908F90ABC527E00B
:10E4B0004B2D400F632F8BE694E039830E94E034AC
:10E4C0003981A0CF20E14DE36091C1058BE694E056
:10E4D0000E94E03420E14CE36091C1058BE694E0BA
:10E4E0000E94E0349ACF6091BF0502E022E08BE603
:10E4F00094E00E942135ACCF0F90DF91CF911F9116
:10E500000F91FF90EF90DF90CF90BF909F908F90F2
:10E5100008956CEB7FE682E064D588E38093C105C3
:10E5200083E08093CB0580E48093CA05E2ECF5E0BC
:10E53000118210821382128215821482178216822F
:10E54000F3DC82E190E09093F1068093F006089569
:10E550008F929F92AF92BF92CF92DF92EF92FF92F3
:10E56000CF937091E405AFEDB5E020E030E090E0AE
:10E5700080E0622FCD902F5F3F4FC110722F8C290A
:10E580006295607F40E050E0D12CE12CF12C4601F7
:10E590005701042E04C0B694A794979487940A94C4
:10E5A000D2F780FE08C0E92FF0E0E053FA4FC62F03
:10E5B000C42BC0839F5F4F5F5F4F4530510539F7D4
:10E5C00023303105B1F67093E40540E050E020E0DF
:10E5D00090E0A0E0B0E06C017D01042E04C0F69450
:10E5E000E794D794C7940A94D2F7C0FE05C020934D
:10E5F000E6052AE335E007C02E504F5F5F4F4530F8
:10E60000510549F7F4CF422F3150A0F0225F6C0141
:10E610007D01032E04C0F694E794D794C7940A941E
:10E62000D2F7C0FEF0CF4093E5058091E30582303C
:10E6300069F403C02093E505F8CF8091E70518162B
:10E6400014F08CEF01C084E08093E705CF91FF9038
:10E65000EF90DF90CF90BF90AF909F908F900895F4
:10E6600080E090E0FC01E651FA4F128203968E3171
:10E670009105C1F708951092E9058AE08093E805B5
:10E6800083E08093E7058FE08093E305EFEDF5E00D
:10E690008FE18083818382835BDFE2CF1F93CF93FF
:10E6A000DF93EC01162FDCDF80910E0680930B06C2
:10E6B00087E380930C0686E080930D066AE070E0A5
:10E6C00088EE93E00F944E5090910F0691509093E6
:10E6D0000F06992351F010920A06188310920E0625
:10E6E0001092F1061092F00601C01882DF91CF91CE
:10E6F0001F9108955F926F927F928F929F92AF9237
:10E70000BF92CF92DF92EF92FF920F931F93CF931E
:10E71000DF9384E0809322028091F206882309F43B
:10E7200067C28091F0069091F1068E31910514F048
:10E730008DE190E097FF02C080E090E09093F106B9
:10E740008093F006880F991F880F991F20910E065D
:10E75000422F022E000C550B4817590774F42D5FF9
:10E76000AC01421B510927FD5395423051051CF065
:10E7700020930E0602C080930E0620910E06422FB3
:10E78000022E000C550B841795077CF42350422F62
:10E79000022E000C550B481B590B423051051CF042
:10E7A00020930E0602C080930E06809111068823E6
:10E7B00009F41EC22091CE05222349F09091CF0585
:10E7C000920F9093CF05933F14F41092CE058230B0
:10E7D00070F0815080931106823011F44CDF08C232
:10E7E000843609F005C281E08093110601C2809150
:10E7F000CD058F5F8093CD054091E30590E0242FF8
:10E8000030E035952795281739070CF0ACC090916A
:10E81000CC0581E089278093CC051092CD05442357
:10E8200009F4A1C09091E7058091E905890F209135
:10E83000E605821724F02091E5052817D4F4919578
:10E840009093E7052091E8052B5F2093E8058093DE
:10E85000E9058091E4053AE08302C0011124820FAA
:10E86000911D27FD9A95C99724F064E181E196E016
:10E8700015DF9091E9058091E705890F8093E905FF
:10E880008091E305882309F46EC024E130E040E084
:10E8900050E060E070E0CB010E943838672B682BB5
:10E8A000692B09F060C0ECEEF5E0C0E0D0E08081BB
:10E8B000811153C0CE01880F991FC80FD91FC651AF
:10E8C000DA4F209709F44FC02091E30530E02F5F25
:10E8D0003F4F032E000C440B550B60E070E0CB0162
:10E8E0000E943838FB01E053FA4F4081242F30E07A
:10E8F000B4E035952795BA95E1F7F901E356FC4F59
:10E90000808190E04F705091E9056EE0469F500D78
:10E910001124452FFC01E656FC4F5081450FFC01A8
:10E92000E956FC4F90819695842F890F88838091BA
:10E93000E80582502F5F3F4F9AE0299F800D1124F8
:10E94000898322E030E040E050E060E070E0CB01FD
:10E950000E9438386E5F6A8306C021963396CA30AB
:10E96000D10509F0A4CF90910A06992341F0809136
:10E970000906890F8093090687FD10920A06809187
:10E980000A06882309F4A2C020910906E091E8054F
:10E990002E170CF49BC0022E000C330B0E2E000C15
:10E9A000FF0BCF014D96821793070CF48FC0E090B8
:10E9B0000806CE2D0E2C000CDD0B1091E905CE01C2
:10E9C000811B910917FD93956EE070E00F944F59EC
:10E9D000F62E653008F07AC02E1B3F0BC901029657
:10E9E0006AE070E00F944F59062F633008F06EC054
:10E9F000812C912C540183940F2C04C0880C991CF9
:10EA0000AA1CBB1C0A94D2F7A62F660FBB0BBD0134
:10EA100061527A4FFB019081892F882109F456C0F9
:10EA2000FD01E356FC4FE0814E2F50E0812FFEE0C8
:10EA3000FF9E800D11249A0126563C4FF901F0806B
:10EA4000F80EEF140CF442C0FA01E956FC4F1081A5
:10EA5000412F50E04F0D511DF7FC5A95C417D507B3
:10EA6000ACF510920A06282D20952923FB0120835E
:10EA700023E030E02A1B3B0B809112069091130695
:10EA8000280F391F30931306209312066AE070E0B6
:10EA900088E290E00F944E502091E805FAE00F9F35
:10EAA000200D1124912F96958F2D890F85508093DD
:10EAB0000B0620930C0684E080930D068091E305FD
:10EAC00081508093E305882321F042DDCCEED5E030
:10EAD00011C084E180931106C3DDF8CFFE0182915D
:10EAE000890F8083803454F01882239626E0CA3040
:10EAF000D207E1F098819923C1F3F0CF8733ACF3CB
:10EB0000FE013297208180910E06281774F3022EA1
:10EB1000000C330B082E000C990B0A9682179307F2
:10EB200024F368E781E196E0B9DDDFCF8091CE057F
:10EB3000811124C024EF31E040E050E060E070E05B
:10EB4000CB010E943838672B682B692BB9F422E07F
:10EB500030E040E050E060E070E0CB010E943838E7
:10EB6000672B682B692B09F091C18FEF8093CE053D
:10EB7000813009F48DC18FE78093CF0580910A061B
:10EB80008823B1F18091CE05882391F18091090607
:10EB9000873074F5209108068091CF05281744F13D
:10EBA000022E000C330B082E000C990B0C968217CA
:10EBB0009307F4F01092CE0510920A068091120687
:10EBC000909113060A9690931306809312066AE0BA
:10EBD00070E088E290E00F944E508091CF058F5FF7
:10EBE00080930B0681E080930C0684E080930D06F1
:10EBF0008091FA0682FF04C08091E205815001C035
:10EC00008AE08093E2050E9403858823C1F0809109
:10EC10001106811103C01092E20511C0813079F410
:10EC200080910A0681110BC080910E068B5F809344
:10EC3000080684E3809309068CEF80930A0680918E
:10EC4000E205811101C0DED161E08BE694E00E9413
:10EC5000CF32C091E8054C2F0C2E000C550B809143
:10EC6000E4059A016AE08602200D311D112422502C
:10EC7000310980919F0490E0821793072CF08091D6
:10EC8000CE05811165C069C08091A10490E0841710
:10EC90009507ACF37DE9672E73E0772EEFED8E2EAE
:10ECA000E5E09E2EFEE15F2E5C0EF301C1903F0178
:10ECB0002C2F0C2E000C330BA901495F5F4F809164
:10ECC0009F0490E0481759073CF4C65FFFEF8F1A86
:10ECD0009F0AC511EACFD3CF8091A10490E082179B
:10ECE00093079CF3D091E90516E41D0FA12CB12CDC
:10ECF000D12CCC0CDD1CF401808190E0A0E0B0E0D0
:10ED00000A2C04C0B695A795979587950A94D2F7D3
:10ED100080FF17C08091CC057601E80EF11CC70179
:10ED200064E0880F991F6A95E1F79C012C503E4CD6
:10ED3000790108E022E04C2F6D2F8BE694E00E94D1
:10ED4000F932D25F3FEFA31AB30AD113D4CFBDCFAC
:10ED500080919F04883008F49DC08091110688231B
:10ED600069F090919F049F3348F49091A1049733E8
:10ED700028F0823008F49CC081FD9AC080910A0678
:10ED80008823B1F040910906242F042E000C330B88
:10ED9000B9016D5F7F4F80919F0490E068177907FC
:10EDA0003CF08091A10490E0821793070CF08EC094
:10EDB000C0E0D0E0FE01E651FA4F8281882399F04D
:10EDC0004181842F042E000C990B20919F0430E088
:10EDD0008217930744F002972091A10430E028178E
:10EDE00039070CF07BC02396CE31D10519F78091FD
:10EDF0000D068823B1F040910C06242F042E000C40
:10EE0000330BB9016A5F7F4F80919F0490E06817D0
:10EE100079073CF08091A10490E0821793070CF0F1
:10EE200065C080911106811101C0AFD080919F040F
:10EE30008A3008F06DC069E080E00E94D639809188
:10EE40001206909113060E94DB3980910F068823E9
:10EE500009F45EC0C1E040E1C42ED12C80910F06C0
:10EE60008C1708F455C0B6016C1B7109660F660F4C
:10EE7000660F5FEDE52E51E3F52E05E021E041E060
:10EE80008BE694E00E94F932CF5FE8CF81E06ECE4E
:10EE900083EF72CE27ECE22E21E3F22E05E022E092
:10EEA00042E06091CF058BE694E00E94F93255CFA5
:10EEB00094EEE92E91E3F92E08E022E047E3609119
:10EEC0000E068BE694E00E94F93258CF24E0609160
:10EED00008068BE694E00E9400356ACF425023E09A
:10EEE00060818BE694E00E9400357DCF81EDE82EB5
:10EEF00081E3F82E07E022E060910B068BE694E0B8
:10EF00000E94F93280910D06815080930D0689CFC1
:10EF1000DF91CF911F910F91FF90EF90DF90CF90F5
:10EF2000BF90AF909F908F907F906F905F9008956B
:10EF30006AE773E784E155D083E080930F068AE0A7
:10EF40008093E20510920A0696DB10920E0610924C
:10EF5000F1061092F00608958091F206882319F0C8
:10EF600082E08093100684E0809322028091110653
:10EF7000882349F0909110068FEF890F8093100637
:10EF800081E019160CF080E008950F9380919F04A2
:10EF9000853228F58091A1048B3108F160E08BE681
:10EFA00094E00E94CF3209E028E34BE164E28BE673
:10EFB00094E00E94713561E08BE694E00E94CF32CC
:10EFC0000E944C86882359F063E285E20E94D6397C
:10EFD0006FEF7FEF84E592E30F910C94303A0F913D
:10EFE0000895FB01109213061092120680931106E9
:10EFF00020E040E060E070E0CF019FD781E08093A7
:10F00000F80608951092F806CBC7809114069091E7
:10F01000160689130DC08091150690911706891761
:10F0200014F02FEF01C021E0820F8093150608C075
:10F03000891714F02FEF01C021E0820F809314068E
:10F04000891319C02091780621502093780630E06A
:10F05000832F90E0DC01AA0FBB1FAC5EB94F880F75
:10F06000991FFC01EA5EF94F808191818D939C93F9
:10F070003F5F231768F70895EF92FF921F93CF9396
:10F08000DF931091780620917F06E22E022E000C6D
:10F09000FF0830918006C32F032E000CDD0BE7E143
:10F0A000F6E040E0411709F446C0CF010397DC01C8
:10F0B0009C91BF0161507109DB018C9198131DC0B7
:10F0C000692F092E000C770B61507109C617D707FD
:10F0D00011F039132DC09081BF0162507109DB011D
:10F0E0008C91582F98170CF4592F25170CF189176C
:10F0F0000CF4892F8217E4F020C0BF01625071091F
:10F10000DB015C91652F052E000C770B61507109B6
:10F11000E616F70611F025130BC0582F98170CF4BC
:10F12000592F35172CF089170CF4892F83172CF4DD
:10F130004F5F3296B7CF80E001C081E0DF91CF9181
:10F140001F91FF90EF90089528E130E040E050E0FB
:10F1500060E070E0CB010E943838609380062AE0BE
:10F1600030E040E050E060E070E0CB010E943838D1
:10F1700060937F0681DF8111E7CF0895909181062A
:10F18000811102C08FEF01C081E0980F93709093BE
:10F190008106E0917806EF5FE0937806F0E0EE0FED
:10F1A000FF1FEC5EF94F80917C06808380917A0688
:10F1B00081830895CF9380E091E090937C068093C3
:10F1C0007B0680E095E090937A0680937906109212
:10F1D000810610927806E4E1F6E01082C5E0C18372
:10F1E00081E0CCDFC0937E061092F1061092F0060B
:10F1F00010927D06CF910895EF92FF920F931F9387
:10F20000CF93DF9380917806843008F4B1C090E00A
:10F21000FC01EE0FFF1FEE5EF94F2081EC01CC0FD9
:10F22000DD1FCC5ED94F68810297261719F0F12CAB
:10F2300031966BC0E12C219631964E2D50E0481747
:10F2400059070CF095C0BA01660F771F8B010C5E51
:10F25000194FD801FC90DB01AA5EB94F3C91F3161F
:10F26000E9F0432FF3160CF44F2D24179CF13F15B2
:10F270000CF43F2D321774F1DB01AC5EB94F1196DF
:10F280005C9141E0308153170CF040E031E068813F
:10F2900065170CF430E04317E9F06CC02F111AC069
:10F2A0006881408111965C91D80111963C91A42F00
:10F2B00064170CF4A62F732F35170CF4752F7A17DB
:10F2C0004CF046170CF4462F53170CF4352F431708
:10F2D0000CF050C0E394B1CFEA01CC0FDD1F8E01DA
:10F2E0000C5E194FD80111967C91DE01AA5EB94FD0
:10F2F00011963C911197731709F14081532F7317A1
:10F300000CF4572F45173CF4F3944F2D50E0481759
:10F31000590714F32DC037170CF4372F3417A4F303
:10F32000CC5ED94F588141E052170CF040E031E0FB
:10F3300065170CF430E0431739F31CC030813713E4
:10F34000E3CF4C91D8013C91762F26170CF4722F05
:10F35000532F34170CF4542F5717B4F2562F62174B
:10F360000CF4522F43170CF4342F53176CF202C0D5
:10F3700080E001C081E0DF91CF911F910F91FF905C
:10F38000EF900895CF92DF92EF92FF920F931F9329
:10F39000CF93DF931F92CDB7DEB7DEDD882309F46C
:10F3A00080C080917B0690917C06392F4091790630
:10F3B00050917A0620918106213061F02CF42111C0
:10F3C00016C0CA01C3970AC0223031F0233079F445
:10F3D000C39709C0C39607C0CA01C39690937A0623
:10F3E0008093790604C090937C0680937B061091ED
:10F3F0007C0600917A06311303C0051709F451C049
:10F40000183110F40A3048F01092110668E270E0EA
:10F4100080E991E00F944E5044C0E0917806F0E00E
:10F42000EE0FFF1FEC5EF94F108301838091F00611
:10F4300090917D06282F291B39F080937D0681E06D
:10F4400012160CF080E09ADE80917E06882321F06F
:10F45000815080937E0601C0D8DDCEDE8111D4CFED
:10F460008091800618131DC080917F06081319C073
:10F470006CED70E085E090E00F944E5068E171E033
:10F4800085E090E00F944E50809112069091130603
:10F490000196909313068093120682E080937E0675
:10F4A00053DE61E08BE694E00E94CF3280919F04AE
:10F4B000893050F467E080E00E94D63980911206CE
:10F4C000909113060E94DB3906E32CE749E062E0E5
:10F4D0008BE694E00E942135F12C809178062091F2
:10F4E0009F04F81608F071C0EF2DF0E0AF01440F53
:10F4F000551FDA01AC5EB94F9C91FA01EA5EF94FF3
:10F500008081981345C091811196EC901E2DE916CB
:10F510000CF4192F85E01802B0011124625F7F4FAF
:10F5200030E0621773070CF44EC09E150CF4E92E00
:10F530009E2DE5E09E0290011124265F3F4F8091B1
:10F54000A10490E028173907F4F58E2D880F880F55
:10F550008E0D7BE0780FCA018C5E994F6C011E15F1
:10F5600094F1272F072E000C330BA9014D5F5F4F3D
:10F5700080919F0490E0481759073CF08091A104C6
:10F5800090E0821793070CF04DC0E3947B5FE7CFC8
:10F5900011963C91432F440F440F340F4BE0D42E6F
:10F5A000D30E4D2D0D2C000C550BBA016D5F7F4F06
:10F5B00030E0621773073CF02091A10430E024177B
:10F5C00035070CF040C0F39488CF40917F06842F1C
:10F5D000880F880F480F455F642F042E000C770BAF
:10F5E000FB013396822F90E0E817F9073CF08091F9
:10F5F000A10490E0861797070CF044C08091110693
:10F60000811101C0C2DC0E940385882309F448C02F
:10F610000F90DF91CF911F910F91FF90EF90DF90AE
:10F62000CF90F0CCF6016081862F880F880F680F8D
:10F630006C5F04E024E0472F8BE694E079830E941E
:10F6400071357981A2CFE82E98170CF4E92EC82ED7
:10F6500089170CF4C92E1E2D110F110F1E0D50E02D
:10F660001C5FCE140CF4AFCF612F650F04E024E0D3
:10F670004D2D8BE694E059830E947135E3945981B6
:10F680005B5FEFCF60918006862F880F880F680F31
:10F690006C5F04E024E08BE694E00E942135AECF5D
:10F6A0000F90DF91CF911F910F91FF90EF90DF901E
:10F6B000CF90089562EC79E781E093DC7BDD44CD67
:10F6C0007F928F929F92AF92BF92CF92DF92EF92F2
:10F6D000FF920F931F93CF93DF9361E081E036D5C4
:10F6E0007090C906C0E08C2F870DD1F48091C806B8
:10F6F000811104C00E940385811159C080912202AA
:10F70000882309F44CC081E09091C806911180E0F3
:10F7100004E024E04AE453E36C2F0E94D7433FC047
:10F720008130E9F58091C806813021F40E9403857B
:10F73000811144C080912202882389F1D1E0809117
:10F74000C806813009F0D0E0C090BC0DD090BD0D4E
:10F75000E090BE0DF090BF0D20E030E0A901C701A0
:10F76000B6010F94185687FD05C020E030E040E058
:10F770005FE304C020E030E040E05FEBC701B6018A
:10F780000F943F550F948756CB010F94D64900E054
:10F790009C014AE353E36C2F8D2F0E940B44CF5FF3
:10F7A000C53009F0A0CF82E08093C7062CC0F8D303
:10F7B00080919506882309F4A1CF25C06091BC0DE6
:10F7C0007091BD0D8091BE0D9091BF0D0F948C5620
:10F7D0001F92812C912C8CE1A82E8DE4B82E6B0108
:10F7E0001AE0E12EF12C00E010E020E030E0A90169
:10F7F0006CEB7DE082E493E322D30F908091950639
:10F80000882309F497CFDF91CF911F910F91FF903B
:10F81000EF90DF90CF90BF90AF909F908F907F90B0
:10F8200008958091630E882359F08091750E87703A
:10F83000873031F48BEC92E30F94B13D1092630E5C
:10F8400008956F927F928F929F92AF92BF92CF92C4
:10F85000DF92EF92FF920F931F93CF93DF9300D02D
:10F860001F92CDB7DEB761E081E070D46090C90629
:10F87000712C611017C08091C806811104C00E94CC
:10F8800003858111B7C080912202882309F4AAC0A0
:10F8900081E09091C806911180E004E024E04CE200
:10F8A00053E39DC081E0681228C08091C806813072
:10F8B00021F40E9403858111A4C080912202882333
:10F8C00009F490C011E08091C806813009F010E081
:10F8D00080914F0E9091500EA091510EB091520E0A
:10F8E00089839A83AB83BC83CE0101960F94CD4D5F
:10F8F00000E09C0142E153E354C082E0681228C05A
:10F900008091C806823021F40E9403858111B1C024
:10F9100080912202882309F465C011E08091C80615
:10F92000823009F010E08091570E9091580EA0910E
:10F93000590EB0915A0E89839A83AB83BC83CE0152
:10F9400001960F94CD4D00E09C0148EF52E329C091
:10F9500083E068122BC08091C806833021F40E9496
:10F9600003858111BEC0809122028823D9F111E064
:10F970008091C806833009F010E080915F0E90916D
:10F98000600EA091610EB091620E89839A83AB8361
:10F99000BC83CE0101960F94CD4D00E09C014EED4D
:10F9A00052E3672D812F0E940B441CC084E0681233
:10F9B00019C08091C806843021F40E94038581110A
:10F9C000C1C080912202882369F081E09091C8062D
:10F9D000943009F080E000E22EE34FEC52E3672D13
:10F9E0000E94D7437394639485E0781242CF70925B
:10F9F000C706AEC0D5D280919506882309F443CFBF
:10FA0000A7C081E0F5D720E030E048EC52E46091F7
:10FA10004F0E7091500E8091510E9091520E0F9496
:10FA2000565820E030E04AEF54E40F943F550F94CD
:10FA30008C561F92E1E18E2EECE79E2EFAE3AF2E5C
:10FA4000FDE4BF2E6B0110EAE12E1FE0F12E00E075
:10FA500010E020E338EF4FEF5FEF6FE47EE08FE1DF
:10FA600093E3EDD10F9080919506882309F425CF7B
:10FA70006FC081E0BDD720E030E048EC52E46091F7
:10FA8000570E7091580E8091590E90915A0E0F9406
:10FA9000565820E030E04AEF54E40F943F550F945D
:10FAA0008C561F9231E1832E3CE7932E4AE3A42E1D
:10FAB0004DE4B42E6B0110EAE12E1FE0F12E00E0C0
:10FAC00010E020E338EF4FEF5FEF67E57EE085E081
:10FAD00093E3B5D10F9080919506882309F418CF50
:10FAE00037C081E085D720E030E048EC52E46091F7
:10FAF0005F0E7091600E8091610E9091620E0F9476
:10FB000056580F948C561F9281E1882E8CE7982EC0
:10FB10009AE3A92E9DE4B92E6B0118EEE12E13E0B5
:10FB2000F12E00E010E020E030E0A9016FE57EE07A
:10FB30008BEE92E384D10F9080919506882309F48F
:10FB400012CF06C040D480919506882309F439CF9E
:10FB50000F900F900F900F90DF91CF911F910F9109
:10FB6000FF90EF90DF90CF90BF90AF909F908F90DD
:10FB70007F906F900895FF920F931F93CF93DF9321
:10FB800061E081E0E3D2C091C906D0E0C11116C0A6
:10FB90008091C806811103C036D78111DBC08091E6
:10FBA0002202882309F43CC081E09091C80691119B
:10FBB00080E004E024E046EC52E32FC0C130B1F411
:10FBC0008091C806813019F41ED78111CAC0809176
:10FBD0002202882329F181E09091C806913009F032
:10FBE00080E003E02EE344EB52E317C0C230C1F4DF
:10FBF0008091C806823019F406D78111BCC080916B
:10FC00002202882369F081E09091C806923009F0C1
:10FC100080E003E02EE345EA52E36D2F0E94D743D4
:10FC200075D1F82E81111CC0C330E1F48091C80653
:10FC3000833019F4E8D68111A8C08091220288236C
:10FC400009F4ADC081E09091C806933009F080E0DE
:10FC500003E02EE348E952E36D2F0E94D7439FC093
:10FC600013E001C014E0C11318C08091C8068C13C2
:10FC700003C0C9D6811195C080912202882361F00A
:10FC800081E09091C8069C1380E003E02EE34CE8ED
:10FC900052E36D2F0E94D7431C2F81E0810FC813C0
:10FCA00017C08091C8068C1303C0ADD6811183C0E4
:10FCB00080912202882361F081E09091C8069C1314
:10FCC00080E000E22EE34DE752E36D2F0E94D74320
:10FCD00092E0910FF11036C0C91317C08091C80689
:10FCE0008C1303C090D681116DC0809122028823AD
:10FCF00061F081E09091C8069C1380E000E22EE361
:10FD00004FE652E36D2F0E94D74383E0810FC81363
:10FD100017C08091C8068C1303C075D6811159C0D5
:10FD200080912202882361F081E09091C8069C13A3
:10FD300080E000E22EE34EE552E36D2F0E94D743B0
:10FD400094E0910FDF5FCF5FD53009F01FCF909324
:10FD5000C70648C025D180919506882309F41FCF96
:10FD600041C081E092E50E941A488091950688235F
:10FD700009F42DCF37C08CE091E80E941A48809199
:10FD80009506882309F43BCF2DC081E29CE70E94B1
:10FD90001A4880919506882309F44FCF23C014E0B8
:10FDA0007CCF80E69BE70E941A48809195068823C5
:10FDB00009F462CF17C007D380919506882309F410
:10FDC00077CF10C003D380919506882309F48DCF97
:10FDD00009C00E94C1DD81E00BD280919506882385
:10FDE00009F49ECFDF91CF911F910F91FF9008955D
:10FDF000E0919606E63000F581E08E0F809396063E
:10FE00008091F0069091F106A0E0B0E03091C90633
:10FE10002091C70648E0E49FF0011124E956F94F0C
:10FE20004091EB065091EC0651834083828393838B
:10FE3000A483B5833683278308950D94B13D2F9213
:10FE40003F924F925F926F927F928F929F92AF926A
:10FE5000BF92CF92DF92EF92FF920F931F93CF93B7
:10FE6000DF9300D000D0CDB7DEB71C012B833C83DD
:10FE70004D835E8369837A83BBDF83E080932202B4
:10FE8000309294062092930669817A81709392064B
:10FE9000609391062B813C814D815E8120938D067C
:10FEA00030938E0640938F0650939006E092890619
:10FEB000F0928A0600938B0610938C06D092F1067E
:10FEC000C092F006B092EC06A092EB0690928806E3
:10FED000809287068C8D8093860626960FB6F894BE
:10FEE000DEBF0FBECDBFDF91CF911F910F91FF906D
:10FEF000EF90DF90CF90BF90AF909F908F907F90CA
:10FF00006F905F904F903F902F90089580918D0F4C
:10FF100090918A0F891B8F7071F49091D60992FB92
:10FF2000882780F992FD08C081E09091FC179130FC
:10FF300019F080E0089581E00895E091EB06F091DA
:10FF4000EC06E817F90721F13091FB0637FD109216
:10FF5000FB069093EC068093EB067093F10660939A
:10FF6000F0064093C9062093C7068356944821F4AF
:10FF70001092F806109296060E94FB4282E080934F
:10FF8000220281E0809395061092F3061092820679
:10FF9000089520E040E060E070E083E694E8CDCF93
:10FFA000E0919606EE2381F0E150E093960688E01A
:10FFB000E89FF0011124E956F94F2781468160E05E
:10FFC00070E080819181B9CFE4CFCF93DF93FC01C2
:10FFD000EB018091F0069091F10697FF04C010921A
:10FFE000F1061092F0064091890650918A066091C0
:10FFF0008B0670918C068091F0069091F106092E87
:020000021000EC
:10000000000CAA0BBB0B481759076A077B0724F49F
:100010005093F1064093F006809122028823D1F09C
:100020002091F0063091F10680918D0690918E0618
:10003000A0918F06B0919006BC01CD01620F731F95
:10004000811D911D1995BC01809193069091940694
:100050000E946C448091E506811108C0809186065B
:10006000882381F180912202882361F18091910699
:1000700090919206009791F02091F0063091F10650
:1000800040918D0650918E0660918F06709190067A
:10009000420F531F611D711DFE011995E0918706E6
:1000A000F0918806309741F080918606811103C057
:1000B0008091E50681111995A6D4882319F0DF9166
:1000C000CF916ECFDF91CF9108950F931F93CF9370
:1000D000DF9380912202882359F06091830670910A
:1000E000840600E010E020E041E081E00E947443DB
:1000F0008091850681111CC081E080938506C091A6
:10010000EB06D091EC0620E040E060E070E085E690
:1001100090E813DF0E9470FA1092850620E040E01C
:1001200060E070E0CE01DF91CF911F910F9105CF7C
:10013000DF91CF911F910F910895009711F484E7FB
:1001400093E39093840680938306BFCF282F109269
:10015000EA068091F0069091F1068130904820F0F7
:100160001092F1061092F0068091F206882331F089
:100170008091F0068093C806109295068091C7067C
:100180001816BCF4082E000C990B821B91092091C3
:10019000C806022E000C330B2817390754F097FFBE
:1001A00002C080E090E08093C8069093F1068093AF
:1001B000F0068091C8066623C1F09091C9068917A0
:1001C00014F48093C9062091C906022E000C330B4B
:1001D0002C5F3F4F482F082E000C550B2417350776
:1001E00034F484508093C90608958093C906089515
:1001F000882361F063E972E084E690E00F944E504A
:100200006AEB72E084E690E00D944E5068EB71E08A
:1002100084E190E00D944E50CF92DF92EF92FF92E6
:100220000F931F93CF93DF93EED3882369F00E943F
:1002300076D91092F806DF91CF911F910F91FF9020
:10024000EF90DF90CF90ACCE81E08093F806C09124
:10025000630ED1E0C111D0E00091F0061091F106DB
:100260000115110509F466C01092F1061092F0060E
:10027000B801012E000C880B990B0F94BA562091EF
:10028000130F3091140F4091150F5091160F0F94CA
:1002900056589B01AC016091350E7091360E8091DD
:1002A000370E9091380EDD2329F00F943F556B01E6
:1002B0007C010EC084E0C89FF0011124E55AF14F83
:1002C00060817181828193810F943E556B017C0125
:1002D00020E030E040E050ECC701B6010F941B581D
:1002E00087FD28C020E030E040EA50E4C701B601B5
:1002F0000F9418561816F4F0B80182E00E948DABE6
:10030000DD2349F0C092350ED092360EE092370EC2
:10031000F092380E0CC0E091630E24E0E29FF001F1
:100320001124E55AF14FC082D182E282F38282E049
:1003300080932202809122028823A1F1D11117C05B
:100340008091630E24E0829FC0011124855A914F51
:100350000F94734ABC0187E693E3DF91CF911F911D
:100360000F91FF90EF90DF90CF900C946C4485E359
:100370009EE00F94734ABC0188E593E30E946C44AD
:100380006091350E7091360E8091370E9091380E37
:10039000DF91CF911F910F91FF90EF90DF90CF9061
:1003A0000C949B45DF91CF911F910F91FF90EF909F
:1003B000DF90CF90089521E0209385060F94B63DFD
:1003C0001092850608950E94B1D912CF0E94EAE9E1
:1003D0000FCF2091F0063091F1062115310559F02B
:1003E00081E0121613060CF080E0809382061092D2
:1003F000F1061092F0068091820608954F925F9266
:100400006F927F928F929F92AF92BF92CF92DF9224
:10041000EF92FF920F931F93CF93DF931F921F9240
:10042000CDB7DEB75C014A013901280187017601A9
:1004300069837A83CEDFD82EE6D2C82E69817A818D
:10044000811104C0809122028823F9F092014D2D80
:10045000C5010E943F45CC20C1F0DD2011F0F40120
:1004600001C0F3010F900F90DF91CF911F910F9179
:10047000FF90EF90DF90CF90BF90AF909F908F90C4
:100480007F906F905F904F9019940F900F90DF9135
:10049000CF911F910F91FF90EF90DF90CF90BF9081
:1004A000AF909F908F907F906F905F904F90089546
:1004B000FC0180810895FC01849108954F925F9220
:1004C0006F927F928F929F92AF92BF92CF92DF9264
:1004D000EF92FF920F931F93CF93DF936C017B01F9
:1004E0005A012901672B31F088248394912CC0E0B4
:1004F000D0E019C0F8011182108227C03701680CC2
:10050000791C76946794E3012197A201BE01C6018C
:10051000F50119951816190654F0892BC9F04301F5
:10052000FFEF8F1A9F0AE814F90440F702C07E011A
:10053000FACFCE15DF0530F4CE0102968816990663
:1005400020F02196F801D183C0838FEF9FEF05C083
:10055000F801D183C08380E090E0DF91CF911F91BB
:100560000F91FF90EF90DF90CF90BF90AF909F9052
:100570008F907F906F905F904F9008958F929F9291
:10058000AF92BF92CF92DF92EF92FF920F931F93A1
:10059000CF93DF93EC016B017A01FB01199587FD85
:1005A00006C0082F10E020E030E0219620C1982FEF
:1005B000907E903CC1F4082F0F7110E020E030E0F5
:1005C0004801590186E0880C991CAA1CBB1C8A951D
:1005D000D1F7CE010196F60119958F73950184012B
:1005E000082B229604C1982F907F903E19F58F70AA
:1005F000882E912CA12CB12C16E0880C991CAA1CD9
:10060000BB1C1A95D1F7CE010196F60119958F738F
:10061000882A06E0880C991CAA1CBB1C0A95D1F7F5
:10062000CE010296F60119958F7395018401082B6E
:100630002396DDC0982F987F903F81F58770882E94
:10064000912CA12CB12CF6E0880C991CAA1CBB1C87
:10065000FA95D1F7CE010196F60119958F73882A84
:10066000A6E0880C991CAA1CBB1CAA95D1F7CE0148
:100670000296F60119958F73882AB6E0880C991CAA
:10068000AA1CBB1CBA95D1F7CE010396F6011995A9
:100690008F7395018401082B2496A9C0982F9C7F05
:1006A000983FE9F58370882E912CA12CB12C56E04F
:1006B000880C991CAA1CBB1C5A95D1F7CE01019637
:1006C000F60119958F73882A66E0880C991CAA1C7C
:1006D000BB1C6A95D1F7CE010296F60119958F736E
:1006E000882A76E0880C991CAA1CBB1C7A95D1F745
:1006F000CE010396F60119958F73882AE6E0880CDF
:10070000991CAA1CBB1CEA95D1F7CE010496F601F0
:1007100019958F7395018401082B259668C0982F31
:100720009E7F9C3F09F04AC08170882E912CA12C9D
:10073000B12C86E0880C991CAA1CBB1C8A95D1F7A9
:10074000CE010196F60119958F73882A96E0880CE0
:10075000991CAA1CBB1C9A95D1F7CE010296F601F2
:1007600019958F73882A26E0880C991CAA1CBB1C3B
:100770002A95D1F7CE010396F60119958F73882A31
:1007800036E0880C991CAA1CBB1C3A95D1F7CE0107
:100790000496F60119958F73882A46E0880C991CF7
:1007A000AA1CBB1C4A95D1F7CE010596F6011995F6
:1007B0008F7395018401082B269619C0982F907C81
:1007C000903849F4082F007C003871F42196CE014E
:1007D000F6011995F7CF082F0E7F0D3F28F02196CF
:1007E000CE01F6011995F7CF00E010E09801E11471
:1007F000F10429F0F7010083118322833383CE01B2
:10080000DF91CF911F910F91FF90EF90DF90CF90EC
:10081000BF90AF909F908F9008951F93CF93DF93D9
:1008200000D01F92CDB7DEB710E0AE014F5F5F4F33
:1008300068E572E8A3DE49815A816B817C81452B92
:10084000462B472B11F01F5FF0CF812F0F900F9099
:100850000F900F90DF91CF911F9108951F93CF9329
:10086000DF9300D01F92CDB7DEB710E0AE014F5F2F
:100870005F4F6BE572E882DE49815A816B817C8132
:10088000452B462B472B11F01F5FF0CF812F0F9088
:100890000F900F900F90DF91CF911F910895FC0161
:1008A000A081B1811C92A281B3818C918F5F8C93C6
:1008B0000280F381E02D80816CE0689F600D11243F
:1008C00080E00C94D6391092EA068091E5061092E9
:1008D000E506882349F020E040E060E070E084E134
:1008E00097E62BDB0C94C64220916D0230916E028C
:1008F0004091F0065091F106C901840F951F2436EE
:10090000310551F44730510514F0069720C04A3F95
:100910005F4F64F506961BC02436310524F48536F6
:10092000910524F504C08436910524F41FC08A3053
:1009300091053CF0883E43E094072CF087EE93E06D
:1009400002C08AE090E02817390731F40DC08A30E0
:10095000910584F78AE090E090936E0280936D0297
:100960001092F1061092F0060C94AB3A84E690E0F7
:10097000E1CFCF93DF931F92CDB7DEB78091870988
:10098000811103C089EC99E02FC0211103C087E8D1
:1009900099E02AC08DE0815048F0440F411DE82FB6
:1009A000F0E0E753F64F90814927F5CF8091DB06C1
:1009B0008417A9F04093DB0687E899E069832DDF6F
:1009C00090E06981861B910997FF02C080E090E06A
:1009D0008093ED061092EE0688E0809324028091C9
:1009E000EE0690E08957964F0F90DF91CF910895D2
:1009F0008093EA061092E6061092E7061092E80647
:100A00001092E90608958091E5061092E506089592
:100A10007F928F929F92AF92BF92CF92DF92EF928E
:100A2000FF920F931F93CF93DF93CDB7DEB7289735
:100A30000FB6F894DEBF0FBECDBF7C014B016A013B
:100A40005901FB0180816CE0689F600D1124F70162
:100A50008081982F990F890F880F0E94D639C11471
:100A6000D10409F496C0FE82ED8298868F8201112E
:100A700003C01C2D0D2D74C09D2C0C2D1D2DD12CB3
:100A800088248394AE014F5F5F4FB5018C2D992D63
:100A900075DDC82E992E89819A81AB81BC8177241E
:100AA00073940097A105B105C9F0712C80329105AE
:100AB000A105B10581F0AC01BD014D52510961099B
:100AC0007109423051056105710540F08B97A10510
:100AD000B10589F503C0DD2009F455C0F701208177
:100AE0008D2D90E0820F911D46972CF0253018F047
:100AF000CE010596D4DE372D3825D30EF70180813F
:100B00008D0D8083DD2089F0DA94AE014F5F5F4F59
:100B1000B501C80133DD8C0169817A818B819C81AB
:100B20004FEF5FEF0E94E139EDCF711032C00C2D15
:100B3000192DD12CA7CFD3940115110509F0A2CFFF
:100B40000C2D192D9FCF4FEF5FEF0E94E139F70178
:100B500020812F5F2083253118F0CE0105969FDE7E
:100B6000AE014F5F5F4FB501812F902F07DD182F2A
:100B7000092F69817A818B819C81611571058105BD
:100B8000910509F706C00115110589F20F5F1F4F86
:100B9000D3CF28960FB6F894DEBF0FBECDBFDF913E
:100BA000CF911F910F91FF90EF90DF90CF90BF906A
:100BB000AF909F908F907F900895AF92BF92CF9209
:100BC000DF92EF92FF920F931F93CF93DF931F92C9
:100BD0001F92CDB7DEB75C016B017A013FDE182FA3
:100BE000E114F10419F0C70139DE01C080E01A8276
:100BF0001982C114D104C1F4412F50E090E09A0150
:100C0000280F391F263131057CF425E130E0241B03
:100C1000350B281B390B37FF02C02F5F3F4F35952F
:100C200027952A8381E0898301E02BE532E8A5013D
:100C3000BE016F5F7F4FCE010296EADEC114D10480
:100C400089F08A81882321F01A8289818F5F8983C4
:100C500000E028E532E8A601BE016F5F7F4FCE01BC
:100C60000296D6DEE114F10451F000E02BE532E803
:100C7000A701BE016F5F7F4FCE010296C9DE0F90C4
:100C80000F90DF91CF911F910F91FF90EF90DF9028
:100C9000CF90BF90AF900895CF92DF92EF92FF92E6
:100CA0000F931F930E949C2D0091D7061091D80698
:100CB0002091D9063091DA066B017C01C01AD10A65
:100CC000E20AF30AF7FC13C02091D6062095209380
:100CD000D606DC01CB018A549C4FAF4FBF4F8093A7
:100CE000D7069093D806A093D906B093DA0681E090
:100CF0009091D606911101C080E01F910F91FF9055
:100D0000EF90DF90CF900895CF9393E090932202DD
:100D100081111092FA060E949C2DDC01CB018C50AF
:100D20009E4FAF4FBF4F8093F4069093F506A0936C
:100D3000F606B093F70668E873E182E090E00F945E
:100D40004E50C6E0C15049F00F94ED4F62E070E0A4
:100D500080E090E00E94CD2DF5CFCF910895AF9225
:100D6000BF92CF92DF92EF920F931F93CF93DF93B7
:100D700000D01F92CDB7DEB7809123028F3F09F4D8
:100D80004AC00E949C2D0091DD061091DE06209144
:100D9000DF063091E006DC01CB01801B910BA20B3A
:100DA000B30BB7FD38C090918A0F80918D0F8F5F84
:100DB0008F70981781F1E0912302E33019F4E090ED
:100DC000DC0602C0E090630E84E0E802F00111242A
:100DD000E056FC4F20E030E040E752E46081718152
:100DE000828193810F941F5669837A838B839C83BE
:100DF000A12CB12C65018E010F5F1F4F2FE732E050
:100E00004BE752E067E772E083E792E00F947408E3
:100E10008FEF809323020F900F900F900F90DF9130
:100E2000CF911F910F91EF90DF90CF90BF90AF9037
:100E300008950F931F930E949C2D0091F40610912A
:100E4000F5062091F6063091F706DC01CB01801BF8
:100E5000910BA20BB30BB7FD0FC08091030185FB73
:100E6000992790F981E089279091030196FF82608C
:100E7000629B84608093FA068091FA06817090915B
:100E8000FA0691FD82609091CA06891741F181307E
:100E9000A9F028F0823041F0833059F01EC0913023
:100EA00089F09230A9F019C0992361F0933081F054
:100EB00014C0913069F0923081F404C0992341F05C
:100EC000933059F49091EF069F5F9093EF0605C021
:100ED0009091EF0691509093EF068093CA061F9170
:100EE0000F910895CF93DF930E94C642E4E0F1E0B2
:100EF00080818F7D8083C5E0D1E08881809580727C
:100F0000A3E0B1E08C9380818F7B80838881809582
:100F100080748C936A98729A54985C9A82E0809359
:100F2000F90687DF1092EF06DF91CF910895CF93F6
:100F3000C09140078CEF96E070DCC81790F4809168
:100F400040078F5F21E0280FE82FF0E0E450F94FD1
:100F50009081907C903811F4822FF4CF80934007D9
:100F600002C010924007CF9108950F931F93CF9323
:100F7000DF938C01C0914007D0E0C450D94FCE011F
:100F80004CDCF8018083CE01DF91CF911F910F914E
:100F9000089581E09091FC06911101C080E00895D0
:100FA000CF93DF9320913F07211120C0FC010190D6
:100FB0000020E9F73197EF01C81BD90BC334D105E5
:100FC00034F031972081207C2038D9F3F4CFBC0154
:100FD000DD27AE018CEF96E00F94A05EC450D94F90
:100FE00018821092400783E080932202DF91CF9114
:100FF0000895CF93DF93CDB7DEB78E8190913F07F1
:10100000891790F080933F079E01275F3F4F4F81E4
:10101000588562E470E08CEF96E00F94E95E1092E0
:10102000400783E080932202DF91CF9108950F93D0
:101030001F93CF93DF938C0167FF03C010923F078C
:1010400060E080913F0790E0262F062E000C330BC6
:10105000281739071CF160933F07C8010F94025EFF
:10106000F801E80FF91FEF01C01BD10BC334D10504
:1010700034F031978491807C8038D9F3F4CFDD2728
:10108000AE01B8018CEF96E00F94235EC450D94FA7
:1010900018821092400783E080932202DF91CF9163
:1010A0001F910F9108954F925F926F927F928F924E
:1010B0009F92AF92BF92CF92DF92EF92FF920F93E7
:1010C0001F930E949C2D6B017C0149DEB2DE809152
:1010D000FA0682FF15C08091D506811113C091E0F8
:1010E0009093D50620910718211103C080918506A1
:1010F00089278093E5061092071881E005DE02C07B
:101100001092D50689B184FB992790F981E089274F
:101110001091F906811749F18093F906882309F4A3
:10112000CAC164EF71E080E090E00E9493A30E9446
:101130009B94123009F0BAC10E9472950E94C64277
:1011400083E0809322020E949C2D6B017C01DC01D4
:10115000CB018C599F4FAF4FBF4F8093D1069093D7
:10116000D206A093D306B093D4068091D106909175
:10117000D206A091D306B091D406A7019601281BF0
:10118000390B4A0B5B0B57FF05C08091F306882390
:1011900009F41DC2D701C6018C599F4FAF4FBF4FF5
:1011A0008093D1069093D206A093D306B093D40631
:1011B0006091EF06062E000C770B77FF03C0719548
:1011C00061957109062E000C770B880B990B0F9413
:1011D000BA562B013C0120E030E040E050E40F948F
:1011E0001B5887FF05C08091E50681117DC08DC029
:1011F0008091EA06882309F456C08090E606909014
:10120000E706A090E806B090E90681149104A104D5
:10121000B104E1F120E030E040E05FE3C301B2015E
:101220000F9456582B013C01C701B6016819790982
:101230008A099B090F94B8569B01AC01C301B20106
:101240000F941F5620E030E04AE754E40F945658BC
:101250004B015C0120E030E040EA52E40F941B585F
:1012600087FF0FC020E030E040EF51E4C501B4013A
:101270000F941B5887FD0AC02AE030E040E050E0A0
:1012800009C024E630E040E050E004C021E030E056
:1012900040E050E0C092E606D092E706E092E80611
:1012A000F092E90604C021E030E040E050E0A09177
:1012B000EF060091F0061091F1060A2E000CBB0B10
:1012C0000F94C15922E030E040E050E00F9484597F
:1012D000DA01C901800F911FA11DB11D9093F10684
:1012E0008093F0061092EF06D701C6018856954C00
:1012F000AF4FBF4F8093CD069093CE06A093CF06FD
:10130000B093D00681E0809322022091EB063091C9
:10131000EC0644E82336340741F480912402882304
:1013200009F4D4C08150809324022251394451F5EC
:1013300080912402882321F081508093240222C0CE
:1013400084E0809324028091EE068F5F8093EE0606
:101350009091ED06981728F41092EE068CE0809399
:10136000240281E080932202D701C6018856954C61
:10137000AF4FBF4F8093CD069093CE06A093CF067C
:10138000B093D00680916F0081FB222720F981FF66
:1013900005C080916F008D7F80936F008091830ED8
:1013A0009091840EA091850EB091860E222329F093
:1013B00020916F00226020936F003AE0B695A795C8
:1013C000979587953A95D1F7009721E0A207B10547
:1013D00020F08FEF9FEFA0E0B0E0969587952091E9
:1013E0002202211105C03091F3063111ECC051C029
:1013F000009741F04091CB065091CC064817590711
:1014000008F047C08091F306811117C0223008F020
:101410006DC08091A404811107C081E08093A40471
:101420008BE694E00E946F328BE694E00E94A63235
:1014300081E08093F2068093F30683E00E940B42E2
:1014400061E08BE694E00E94CF32E091EB06F091F0
:10145000EC0619951092F2068091F306811152C0A4
:101460001092E5060E949C2DDC01CB018C199D0990
:10147000AE09BF090091CB061091CC0620E030E008
:10148000081719072A073B0720F49093CC0680938E
:10149000CB068091EB069091EC068356944809F4B4
:1014A00083C08091F80681117FC052C060E08EEE4B
:1014B00093E3BDDD43CEEAD5123009F43FCE60E0C0
:1014C00081EE93E3B4DD0E94C97F38CE8CE0809337
:1014D00024028091CB069091CC0601979093CC0684
:1014E0008093CB0681E0809322021FCF243030F01E
:1014F000243009F08ECF109222028BCF81E08093AE
:10150000220287CF8BE694E00E94AA3291E08111FB
:1015100001C090E09093F306992309F4A1CF0E94B3
:101520009C2DDC01CB018C199D09AE09BF09C0902F
:10153000CB06D090CC06E12CF12CC816D906EA06D1
:10154000FB0608F044C09093CC068093CB063FC0C6
:101550008091CD069091CE06A091CF06B091D00695
:10156000C81AD90AEA0AFB0AF7FE0E94C97F8091CD
:10157000F30681112CC080912202813091F08330DA
:1015800031F51F910F91FF90EF90DF90CF90BF90BA
:10159000AF909F908F907F906F905F904F900C9442
:1015A000FB421092220213C048E9C40E4AE3D41E43
:1015B000E11CF11CC092CD06D092CE06E092CF067F
:1015C000F092D006D4CF009709F437CF13CF1F91F4
:1015D0000F91FF90EF90DF90CF90BF90AF909F90D2
:1015E0008F907F906F905F904F90089561E01FDD26
:1015F0000C94C97FCF93DF931F921F92CDB7DEB7B4
:1016000089839A836FDC89819A81F0DF0F900F9034
:10161000DF91CF910C94CB428091D60982FD05C019
:101620008091FC17823061F410C08091870981118C
:1016300003C089EC99E002C087E899E061E0B0CC92
:10164000813031F083EB93E305C084ED93E302C076
:1016500088EC93E36FEFEBCC109207181092940292
:101660008091D60980628093D6090E94CAB20F94F5
:101670008D5060E085EA93E3DADC0C94C97F89E958
:1016800093E30E949D8060E08CE893E3D0DC40917E
:10169000630E61E080E00E94A46682E893E30D940B
:1016A000B13DBADF10920718109294020E940667AB
:1016B000882321F08091D60982FF04C00E94C2B223
:1016C0000D9406518EE793E30F94B13DF7CF8091CF
:1016D000D60982FF2AC00E940667882319F18091EB
:1016E000910790919207A0919307B091940700976A
:1016F000A105B105B9F0BC01CD016D597F4F8F4FE8
:101700009F4F24E630E040E050E00F946259609132
:101710008D0770918E0780918F07909190070F949D
:10172000625901C020E02093FB068091FB068F7771
:10173000089583E694E89093EC068093EB06089571
:1017400061E0FC0180810E94CC2F8FEF0C94C9AA2C
:10175000CF93DF93EC018A810E948BAA60E088819D
:10176000DF91CF910C94CC2F8F929F92AF92BF922A
:10177000EF92FF920F931F93CF93DF93EC018B01B6
:101780007A010E949C2D4B015C012CE2820E21E02B
:10179000921EA11CB11C0E94A3AA8B838F3F61F4EF
:1017A0000E949C2DDC01CB0188199909AA09BB096B
:1017B000B7FDF1CF81E10DC08E3F51F4B701C801F3
:1017C0000E94AAAA0E94A3AA0E94A3AA11E003C091
:1017D0008FE0898310E0CE01B3DF812FDF91CF91BD
:1017E0001F910F91FF90EF90BF90AF909F908F90BF
:1017F0000895CF92DF92EF92FF926A017B010E94DF
:101800009C2DC60ED71EE81EF91E0E94A3AA8F3F6C
:1018100061F00E949C2DDC01CB018C199D09AE0961
:10182000BF09B7FDF2CF80E001C081E0FF90EF90EB
:10183000DF90CF900895EF92FF921F93CF93DF93A5
:1018400000D01F92CDB7DEB77C01162F29833A83D3
:101850004B835C837DDF48E552E060E070E0C701C8
:10186000C8DF812F80640E94C9AA8C810E94C9AA06
:101870008B810E94C9AA8A810E94C9AA89810E947B
:10188000C9AA112311F087E801C085E90E94C9AAFD
:101890001C3011F40E94A3AA10E00E94A3AAF70131
:1018A000838387FF04C01F3F11F01F5FF6CF0F90A7
:1018B0000F900F900F90DF91CF911F91FF90EF90BD
:1018C00008958F929F92AF92BF92CF92DF92EF9244
:1018D000FF920F931F93CF93DF93EC01162F1C827F
:1018E000198248830E949C2D6B017C0120EDC20E61
:1018F00027E0D21EE11CF11CA89561E088810E94BE
:10190000CC2F61E088810E94902F0E949CAA85E0E4
:101910008A830E948BAA0AE08FEF0E94C9AA015015
:10192000D9F7A89520E030E0A90160E0CE0183DF7F
:101930008B83813061F00E949C2DDC01CB018C19DE
:101940009D09AE09BF09B7FDEDCF81E055C0A8954F
:101950002AEA31E040E050E068E0CE016CDF8530FB
:1019600011F481E009C004E00E94A3AA8B83015016
:10197000D9F78A3A51F482E08C83A8958C81823021
:1019800081F0812C912C540111C00E949C2DDC010E
:10199000CB018C199D09AE09BF09B7FDD9CF82E0F3
:1019A0002BC0812C912CA12C80E4B82E20E030E0BB
:1019B000A90167E3CE013FDFA501940169E2CE01F1
:1019C0003ADF8B83882361F00E949C2DDC01CB01E0
:1019D0008C199D09AE09BF09B7FDE8CF8AE00CC09C
:1019E0008C818230D1F420E030E0A9016AE3CE019D
:1019F00022DF882329F088E08983CE01A1DE16C08A
:101A00000E94A3AA807C803C11F483E08C830E9416
:101A1000A3AA0E94A3AA0E94A3AACE0191DE173016
:101A200018F41A8381E003C088E1898380E0DF91A4
:101A3000CF911F910F91FF90EF90DF90CF90BF90CB
:101A4000AF909F908F9008950F931F93CF93DF9344
:101A5000EC0189018C81833039F089E0440F551FF6
:101A6000661F771F8A95D1F79A01AB0161E1CE011C
:101A7000E2DE811109C040E052E0B801CE01DF9101
:101A8000CF911F910F9170CE84E08983CE0158DEF3
:101A900080E0DF91CF911F910F910895CF93DF9355
:101AA000EC01862FBA010E94CEAA8FEF0E94C9AA2C
:101AB0008FEF0E94C9AA0E94A3AA8B83982F9F71BF
:101AC000953031F083E18983CE013ADE80E001C0B8
:101AD00081E0DF91CF9108950F931F93CF93DF9310
:101AE000EC0189018C81833039F089E0440F551F66
:101AF000661F771F8A95D1F79A01AB0168E1CE0185
:101B00009ADE81111EC0A8016EEFCE01C7DF8823C7
:101B1000E1F048E552E060E070E0CE016ADE882343
:101B200071F020E030E0A9016DE0CE0184DE81118A
:101B30000AC00E94A3AA811106C011E007C087E174
:101B400003C086E001C086E1898310E0CE01F8DDA4
:101B5000812FDF91CF911F910F910895CF93DF9344
:101B60001F92CDB7DEB72091091830910A18CE0127
:101B700001962115310519F0821B930B02C08F507D
:101B800098410F90DF91CF910895FC01238121119D
:101B90000C94DC9E089581E497E0F7CF8CE597E004
:101BA000F4CF80917707811107C00E94EAE988236A
:101BB00019F081E08093770708958091D609847F9A
:101BC0008B7F8093D60910928D0710928E0710920A
:101BD0008F0710929007109291071092920710921F
:101BE00093071092940710920208109241088EE019
:101BF00091E0E2E4F8E0DF019C011D9221503040C9
:101C0000E1F78FEF809386090895FC0120E03EE222
